:020000040800F2
:1000000000800010313F0008B9480008E9480008A6
:1000100091490008954A0008E54B000800000000DF
:100020000000000000000000000000006B610008FC
:10003000B7610008000000001F620008F5B2000868
:1000400075A9000877A9000879A900087BA900080C
:100050007DA900087FA9000881A9000883A90008DC
:10006000E765000885A9000887A90008F9B200081B
:1000700005B3000811B300081DB3000829B3000838
:1000800035B3000841B3000889A900088BA900080E
:100090008DA900088FA9000891A900083F660008F3
:1000A00093A9000895A9000897A9000899A9000834
:1000B0009BA900089DA900089FA90008A1A9000804
:1000C000A3A90008A5A90008A7A90008A9A90008D4
:1000D000ABA900084DB3000859B30008ADA900084A
:1000E000AFA90008B1A90008B3A90008B5A9000884
:1000F000B7A90008B9A90008BBA90008BDA9000854
:10010000BFA90008C1A90008C3A90008C5A9000823
:10011000C7A90008C9A90008CBA90008CDA90008F3
:10012000CFA90008D1A90008D3A90008D5A90008C3
:10013000D7A90008D9A90008DBA90008DDA9000893
:10014000DFA90008E1A90008E3A9000800000000F9
:10015000000000000000000000000000000000009F
:10016000000000000000000000000000E5A90008F9
:10017000E7A90008E9A90008EBA90008EDA9000813
:10018000EFA90008F1A90008F3A90008F5A90008E3
:10019000F7A9000800000000F9A90008FBA9000861
:1001A000FDA90008FFA9000801AA000803AA000889
:1001B00005AA000807AA000809AA00080BAA000857
:1001C0000DAA00080FAA000811AA000813AA000827
:0801D00015AA000817AA000897
:1001D800004B0000000001000100000000000000CA
:1001E8000000000000000000000000000000000007
:1001F80000000000000000000000000000000000F7
:1002080090D0030000000000000000000000000083
:1002180040420F000000000040420F0000000000B4
:100228000000000000000000FFFFFFFFFFFFFFFFCE
:1002380000D68AEAFFFFFFFF007884C9FDFFFFFFB1
:10024800DE0369000071020000401F000A0002007E
:10025800606DE06001000200C05DA861A073606D80
:1002680083FF7D0070177C153CF630F870177C15FD
:1002780054F248F4320038FF204E0700840301008E
:080288000100406A640000005F
:1002900050EC101B4FF0FF3202EB105240F2FE7395
:1002A0009A4280F09A802DE9F84F2DED028B82B0B2
:1002B00001A80AF000FC019F554B54EC105B284646
:1002C0002146002208F0EAFB81468A46514B284627
:1002D0002146002208F0E2FB43F6CE32C6F27F62EE
:1002E000AA1A4AF29E02C3F6E67274EB0202BCBF7F
:1002F00054464D46804644EC105B0E46BEBF564603
:10030000C846013F4FF0FF300CF024FC51EC100BBD
:10031000414B002208F0C2FB02460B4640463146E4
:1003200008F0EAFC05460E4602460B4603F018FEAE
:1003300083468A4641EC180B40F6B809C0F600091E
:1003400048460221B0EE480AF0EE680A0AF0CAFBFD
:1003500051EC100B314A324B08F0A0FB04468846A2
:1003600009F110000321B0EE480AF0EE680A0AF025
:10037000F2FB53EC102B2046414608F0BDFC5A46D8
:10038000534603F0EDFD2A46334603F0E9FD2A46C5
:10039000334608F083FB06468846384608F0D8FD09
:1003A00004460D461F4A204B03F0DAFD3246434611
:1003B00008F074FB064688461C4B2046294600225E
:1003C00003F0CEFD3246434608F068FB41EC100BCB
:1003D00002B0BDEC028BBDE8F88F20F000434A422A
:1003E00040F20002C7F6F07272EB030308D310422A
:1003F00007D00028BCBF002102F5002040EC101BF4
:1004000070479FED010B7047000000000000F0FFF7
:100410000000E0BF0000F0BF0000E03F9AB5B3125B
:10042000FF0750C0A80C615C10D02BBF0030E63F26
:100430002DE9F04F83B056EC107BC6F30A5001381B
:1004400040F2FE71884280F0A98043F6EF10CFF6AB
:10045000FA60C01B42F64260C4F28600B041C0F2AE
:10046000B2804BF6D240CDF67A50C01B42F22B3010
:10047000CCF28600B041C0F0898044F22320C0F65F
:10048000924026F00041381A49F6A140C3F6C73021
:1004900071EB00007DD3544D0195F00F2C4660F3B5
:1004A000DF74524A524B3846314603F059FD002260
:1004B000234608F0F3FA08F011FD029008F048FD19
:1004C000044688464B4B002203F04AFD3A46334629
:1004D00008F0E4FA06460F46474A484B2046414694
:1004E00003F03EFD32463B4608F0D8FA80460C4603
:1004F00002460B4603F034FD06460F46404A414B88
:1005000003F02EFD404A414B08F0C8FA32463B4604
:1005100003F026FDA5F58013002208F0BFFA42463D
:10052000234603F01DFD82468B46394A394B30463F
:10053000394603F015FD384A384B08F0AFFA044647
:1005400088460020294652465B4603F005FD0546D5
:100550008946304639462246434603F001FD2A4685
:100560004B4608F09BFA02460B465046594608F0A7
:10057000C3FB0022019B08F091FA41EC100B02989A
:10058000013003B0BDE8F04F0CF0E4BA9FED100B62
:1005900001E09FED130B03B0BDE8F08F26F00040A3
:1005A000794240F20001C7F6F07171EB0002F2D31C
:1005B000484038437FF46FAF002EBCBF0646074665
:1005C00046EC107BE7E79FED040BE4E700BF00BFBC
:1005D0000000000000000000000000000000F07FAC
:1005E000000000000000F03F0000E03F3CF92F9EBB
:1005F0002C15F73F0030E6BFA80C615C10D02B3FF4
:100600001CDC586FA452F13EE0F6B36FE4707C3FFF
:100610000938DE6F993F403FB35142718E71AC3F54
:100620002DE9F8432DED068BB0EE408AF0EE608A9E
:1006300058EC104B0020C3F6F07088EA000121430B
:1006400000F0A98055EC116B00F18042154200F0DA
:10065000A780C8F30A51013940F2FD73994279D855
:10066000C5F30A51A1F2FF714FF60203CFF6FF73F3
:1006700099426FD33046294608F030FC074608F00F
:1006800067FCB7F1004F40D07040694008433CD14F
:100690009FED799B002FB0EE49AAF0EE69AA25D014
:1006A0003E4648BF7E429FED74AB59EC1A4B55EC69
:1006B000188B4046294622464B4603F051FCF20770
:1006C00004BF4946204641EC1A0B4FEA5609404602
:1006D000294642462B4603F043FC012E04BF29461F
:1006E000404641EC180B5FEA0906DED151EC190BCC
:1006F00055EC1A8B42462B4608F0FEFA002F5CBFE1
:100700002946404641EC110B08E0204641460022B4
:10071000002303F0D9FC48B19FED651BB0EE410A00
:10072000F0EE610ABDEC068BBDE8F8836FF3DF786D
:1007300048EC104BFFF7ACFD53EC102B304629462C
:1007400003F00EFC41EC100BBDEC068BBDE8F8434A
:10075000FFF76EBE28F00041634272EB01031AD32B
:1007600025F00043D6F1000972EB0303D6D318EA53
:10077000020F18D088F0704383F07F63234331D099
:1007800082EA080222434FD13DA0002DA8BF0830C5
:1007900090ED001BC2E7B0EE481AF0EE681ABDE714
:1007A0009FED351BBAE73046294608F097FB074610
:1007B00008F0CEFB85EA010286EA00031A437FF4C3
:1007C00060AF37A0002DA8BF08304FEAD872D0E93B
:1007D0000010034662F3DF73FA0708BF034643ECD9
:1007E000111B9BE726A0002DA8BF0830294690EDDD
:1007F000008B304608F072FB044608F0A9FB59EC68
:10080000183B70404FEAD8764A46694066F3DF727B
:10081000084318461CBF4A461846E10704BF4A462B
:10082000184642EC110B79E700F1004202F18043D7
:100830006B40334311D188EA020020439FED0E1B29
:100840003FF46CAF4FF6FF70C3F6EF7014A2814215
:1008500088BF083292ED001B60E7814208D388EA26
:1008600002000BA1204308BF083191ED001B55E7A2
:100870009FED031B52E700BF000000000000F03FA7
:100880000000000000000000000000000000F07FF9
:10089000000000000000F07F000000000000F03FBA
:1008A000000000000000F07F0000000000000000D9
:0808B000000000000000F87FC9
:1008B800EDAF16204A62304029BD56B31544E9BF52
:1008C80077900D9CFE0B88C07E2615FA83807340B6
:0808D8000FCE674B80D541C033
:1008E00082B041F24871C1F2000145F2ED52086850
:1008F000CAF6CE42904200F040830AF0A3FD03F016
:10090000E5FE41F28070C1F200004DF6836100689F
:10091000C4F21B31A0FB0101890C4DF29F30C0F6DF
:1009200000000CF0D7F904F0B6F803F0DEFF0AF08F
:10093000BBF90AF019FA0AF05DFA03F07EFE03F043
:1009400014FF0AF0D7FA0AF0FBFA04F04CF90AF0A7
:100950001DFB0AF083FC06F070F90AF019FD0AF09D
:1009600057FD03F088FF0AF02BFC04F064FC4CF602
:100970002470C0F600000AF070F80BF0E3FF0CF0F2
:1009800029F809F09CFB0BF023FD032818D8DFE8B9
:1009900000F00209100240F20000C1F2000009F06C
:1009A000D4FB0DE040F20000C1F2000009F0F4FBBE
:1009B00006E040F20000C1F2000000210BF02AFD29
:1009C00040F20005C1F2000541F29020C1F20000A2
:1009D0000BF04AF94FF090404FF4806108F06DFA47
:1009E00098B9322000F018FB4FF090404FF480612E
:1009F00008F063FA48B94CF63370C0F600000AF00C
:100A00002CF8284601210BF005FD41F29026C1F299
:100A1000000630460BF028F904F061FC2969AA8A27
:100A2000EB8A40F68C27C1F2000740F20000C2F2C8
:100A3000000000970BF0BCFD30460BF015F902F0FA
:100A400009FD40F6645BC1F2000B0027C4F27F078A
:100A50005846394605F0BCFA40F6F840C1F20000AD
:100A6000394605F0B5FA40F68C40C1F200007F210E
:100A700005F0AEFA40F62040C1F20000394605F01C
:100A8000A7FA40F6B430C1F200007F2105F0A0FAC9
:100A900030460BF0E9F840F23421C2F2000158462A
:100AA000402207F0DAF940B172B64CF64670C0F653
:100AB000000009F0D2FF00BFFEE740F68C40C1F213
:100AC000000040F23431C2F20001032206F02BFE96
:100AD00038B172B64CF64670C0F6000009F0BDFFA2
:100AE000FEE740F62040C1F2000040F24031C2F281
:100AF0000001012206F017FE38B172B64CF64670BE
:100B0000C0F6000009F0A9FFFEE740F6B430C1F2DC
:100B1000000040F24431C2F20001042206F003FE5C
:100B200038B172B64CF64670C0F6000009F095FF79
:100B3000FEE7B34630460BF097F801F081FD3046F2
:100B40000BF092F84DF62610C0F6000009F085FF74
:100B500009F051FD288BF8B1002400BF4FF0904000
:100B6000202101220AF0F8FE4FF4AF7000F054FA91
:100B700058460BF079F84FF09040202100220AF0FF
:100B8000EBFE4FF4AF7000F047FA58460BF06CF8EC
:100B9000288B01348442E1D341F2C02AC1F2000A19
:100BA00000260196B04600BF41F29020C1F200003D
:100BB0000BF05AF8DAF80000012835D140F234245D
:100BC000C2F20004B4F8FE0002F0DEFBB4F8FC0050
:100BD00002F076FE02F096FDD5F8D800D5F8E410C4
:100BE00081FB00014FF47A72002308F0CDF9C5F8BB
:100BF0000801D5F8D800D5F8901181FB00014FF419
:100C00007A72002308F0C0F9C5F884010020CAF800
:100C1000000040F66450C1F200002146402207F077
:100C20001CF9002840F0A18141F2BC20C1F2000073
:100C30000068012806D140F23430C2F2000000689A
:100C400003F038F841F2B820C1F200000068012832
:100C500006D140F24030C2F20000006803F064F8B0
:100C600041F2B420C1F200000068012835D140F201
:100C70004434C2F20004206802F034FC606802F0E0
:100C800057FEA06803F08EFABE4F00223B4603F0E9
:100C900067F9B146BC4E0022334603F061F9DFF834
:100CA000ECB200225B4603F05BF908F017F9A5F8F7
:100CB0005001E06803F076FA00223B4603F050F959
:100CC000002233464E4603F04BF900225B4603F008
:100CD00047F908F003F9A5F8520141F2B020C1F23A
:100CE0000000006801280BD10BF02AFB02F056FC33
:100CF000A5F8980141F2B021C1F20001002008607E
:100D00000AF0D6FBB0EB0808814618BF4FF0010887
:100D10000027B5F85401002EC8BF012704281BD3B3
:100D20004DF63310C0F6000009F097FE4FF0070BA8
:100D3000A5F806B140F20044C4F6000420464FF482
:100D4000006100220AF008FEA5F806B120464FF423
:100D5000805100220AF000FE41F24420C1F200005E
:100D6000006801684068019801F00F0484422ED0A9
:100D7000D5F828010130C5F82801D5F82401013043
:100D8000C5F82401D5F820010130C5F8200141F251
:100D9000AC20C1F20000006820B94FF09040102153
:100DA00008F0C1F801F0E4FF02F0DCFF09F02CFCD0
:100DB0000BF0CCFC02F0DAFE04F077FB02F0F0FE60
:100DC000A5F89C0102F0C8FBA5F816010194688BF8
:100DD000002840F20004C2F2000400F0798094F888
:100DE0002600002840F07480688B40F2F131884280
:100DF0000DDC01380A2821D8DFE800F006363A2F4A
:100E000020B64E3F33435900284600215BE0B0F541
:100E10007D7F1ADB52D040F2D241884251D041F25C
:100E2000525188420AD141F24870C1F2000045F2A5
:100E3000ED51CAF6CE4101600AF058FC4DF6C8608B
:100E4000C0F6000009F009FE40E00131884231D0CF
:100E500001318842F2D101202DE0284609F09CF9A9
:100E600034E00BF049FA31E0284609F06EF92DE044
:100E7000284601210BF0CEFA28E0284609F002F9B5
:100E800024E0284601F0A8FA40F23030C2F2000017
:100E9000008802F0DDFC19E0284609F0DCF840F299
:100EA0003030C2F2000000880BF07AFB0EE001F057
:100EB00029FB0BE0002004F0E4FF07E00AF010F942
:100EC00004E02846012109F044FA00BF00206883AD
:100ED00008EA0700361A4FF090404FF4806107F09F
:100EE000ECFF002808BF002E18D020460BF0FEFBB8
:100EF0000028C8463FF458AE204609F02BFB0228D4
:100F000020D141F2AC20C1F20000006800287FF43B
:100F10004BAE204609F039FB46E600BF0A2000F040
:100F20007BF84FF090404FF4806107F0C6FF002837
:100F3000DBD141F2AC21C1F20001086848B10E607A
:100F40000FE000BF40F6AC30C1F20000222101608A
:100F50002AE6012008604FF09040102101220AF09B
:100F6000FBFC4FF4FA76C0E7FEE772B64CF646702B
:100F7000C0F6000009F071FDFEE70020086000F0F7
:100F800007F800BF0070A740000035400000F03EA9
:100F900082B04EF28010CEF2000072B64FF0FF31F8
:100FA000082200BF40F8041B013AC0F8FC10F9D138
:100FB0000020C1F6FF7003C880F3088841F260008A
:100FC000C4F202000123026842F0010202600068DC
:100FD00000F00100019001980020C4F201000268B5
:100FE00063F30202026062B688474DF64C14C0F605
:0C0FF000000400BF204609F030FDFBE7C4
:100FFC00C012001000000000000000000000000003
:0C100C00BC120010B8120010B41200104A
:1010180038B504460AF048FA054641F27070C1F244
:101028000000611C006818BF044400BF0AF03CFAC5
:08103800401BA042FAD338BDB1
:10104000000000000100000002000000030000009A
:10105000000000000500000006000000070000007E
:0810600000000000090000007F
:10106800BFF34F8F4EF60C50CEF2000004220168F9
:1010780001F4E061C0F2FA5211430160BFF34F8FEF
:0410880000BFFDE7C1
:10108C0010B55FEA920E0ED0D0F800C00B4600BF30
:10109C0053F8044B24BABEF1010ECCF80040F7D142
:1010AC0022F0030300E0002302F00302DFE802F069
:1010BC001702060E0268C95C117010E0CA18C95CF0
:1010CC005278036842EA0121198008E0CA18C95C09
:1010DC005378046843EA01212180917821700068DB
:0410EC00006810BDCB
:1010F00070B5416842F22002C4F2020204294FF0A6
:10110000060C1ED803291CD04FF0070C0429C0F888
:1011100000C016D802F10C03DFE801F00B03061340
:10112000090002F1100304E002F12C0301E002F1D6
:101130003003196801F07F0181601968C1F306412D
:10114000C1601168C9B2AA290B4618BFBB23CC29BC
:1011500008BF0B4603611168C3695E1E012E21F0B2
:10116000FF01816163D847F2E056C1F6FF760021A6
:10117000C0F604010CF1080C0025C4F20105C0F80A
:1011800000C02D683488ED054FF6FF7508D4AC42D9
:101190004FF0006E0FD03468714664F358210AE0B6
:1011A000AC4205D031684FF0006E61F3582E00E07C
:1011B0008E464FF00061146864020DD4012B4FF687
:1011C000F071C0F2070117D1566801EA061606F160
:1011D00000660662966816E0012B4FF6F874C0F2BE
:1011E000030415D1516804EAC10171440162916898
:1011F00004EAC101714414E0566A01EA061606F1D8
:1012000000660662966A01EA061101F1006108E0D3
:10121000566A04EAC6060E440662966A04EAC606E0
:1012200031444162916801F000411943C1610CF100
:1012300010010160136DC16A4E1E012E03F480334C
:1012400083620AD80CF1300C012914BF54215021BB
:0C125000C0F800C05158C9B2016370BD65
:10125C002DE9F04F85B0044600F138404FEAB0203C
:10126C00029007280D4606D34CF6CB70C0F6000052
:10127C00A92109F097FF2868010C01D1000406D1BF
:10128C004CF6CB70C0F60000AA2109F08BFF686801
:10129C00B0F5881F80F20081122800F2178101211D
:1012AC0001FA00F00F21C0F20601084200F00E8195
:1012BC002868002800F0ED8040F2004AC4F2010AD0
:1012CC0004F12001019141F20041C4F60001062213
:1012DC008C4208BF05220299052938BF0A460392A1
:1012EC004FF00009032700BF012101FA09FB10EAA6
:1012FC000B0800F0C780686800F003014A1E012A41
:10130C0020D8E868042807D34CF6CB70C0F6000050
:10131C00BB2109F047FFE8684FEA49018840A26801
:10132C0007FA01F122EA01010843A06061686868CC
:10133C0021EA0B01C0F3001202FA09F211436160B9
:10134C0000F00301032915D0A868032807D34CF635
:10135C00CB70C0F60000CC2109F024FFA8684FEA3E
:10136C0049018840E26807FA01F122EA01010843C9
:10137C00E060686800F00301022929D1029807286F
:10138C0006D34CF6CB70C0F60000D92109F00AFF49
:10139C002869102807D34CF6CB70C0F60000DA2170
:1013AC0009F000FF28696FF0030101EA59011C22C2
:1013BC0002EA8902019E904073580F2707FA02F245
:1013CC0023EA020210437050686800F003010327FF
:1013DC0010F4403F4FEA490001FA00F1226807FA85
:1013EC0000F022EA000040EA010020604AD041F2FD
:1013FC006001C4F202014FF60846086840F0010093
:10140C000860086800F001000490049829F00300BB
:10141C005044CFF6FF760C22815902EA89020F2341
:10142C0093409943039B03FA02F211438151DAF87A
:10143C000800696840EA0802CB0258BF20EA08029B
:10144C0040F20C46C4F20106CAF80820306840EAA3
:10145C0008028B0258BF20EA08023260DAF8040056
:10146C0040EA08028B0358BF20EA0802CAF804209D
:10147C00DAF8000040EA0802C90358BF20EA080263
:10148C00CAF80020286809F1010930FA09F17FF443
:10149C002BAF05B0BDE8F08FB0F5081F0CDAB0F536
:1014AC00881F3FF405AFB0F5901F3FF401AFB0F5C6
:1014BC00041F3FF4FDAE09E03FF4FAAEB0F5441F53
:1014CC003FF4F6AEB0F5481F3FF4F2AE4CF6CB70DD
:0C14DC00C0F60000AB2109F065FEE9E657
:1014E800F8B5044600688069800719D415460E4689
:1014F8004F1C00BF204631462A4600F021F8E8B9C3
:1015080057B109F0D1FF216816B1401BB04204D988
:101518008869800701D405E0216888698007E9D5D2
:101528000020F8BD606C40F020006064202084F842
:101538004100002084F8420084F840000120F8BDF2
:10154800F8B5036804469869C00623D4002500202E
:1015580038E000BF596894F842009A6912040BD524
:1015680011F4804108D1202806D0586840F4804002
:10157800586009F099FF06462368986980061AD4CE
:1015880009F092FF801B1928F6D923682425986949
:10159800012017E01020D861986980060ED41646FD
:1015A8000D464F1C3FB109F07FFF2368002DD1D0B5
:1015B800801BA842CED898698006F3D52020D86130
:1015C800012004259969CA0504D501354FF48070B6
:1015D800D86101204A0503D4890507D450B9F8BD5C
:1015E800083588054FF48060D86103D502354FF47B
:1015F8000070D86120460AF0C9F920684EF600024A
:101608004168CFF6006211404160606C2843606415
:10161800202084F84100002084F8420084F840002B
:041628000120F8BDE8
:10162C0038B5040054D0206843F20001C4F2000124
:10163C00884206D04DF22A00C0F60000B52109F010
:10164C00B1FD6068072806D34DF22A00C0F60000F1
:10165C00B62109F0A7FDA068B0F5805F06D34DF266
:10166C002A00C0F60000B72109F09CFDE068B0F537
:10167C00805F06D34DF22A00C0F60000B82109F0B5
:10168C0091FD94E807004CF6CC43036045F25553AA
:10169C0003604160826009F005FF2168CA68520747
:1016AC000CD0054609F0FEFE401B3228216802D3FF
:1016BC00C86840070ED1C8684007F3D10A69E068D2
:1016CC00824206BF4AF6AA2008600861002038BD95
:0816DC00012038BD032038BDD8
:1016E4002DE9F04704007DD0884620680F2802D8F1
:1016F40010F00F0007D14DF23D60C0F6000040F23B
:101704000B3109F053FDB8F1100F07D34DF23D60D2
:10171400C0F600004FF4437109F048FD42F200079F
:10172400C4F20207386800F00F0080450AD938680F
:1017340020F00F0040EA08003860386800F00F001D
:1017440040454FD12068C107A7F6F87503D181073A
:1017540040F195807AE06068411E032908D34DF278
:101764003D60C0F6000040F2233109F01FFD6068BF
:1017740055F8081C022833D0032836D1880131D506
:10178400686869686A6800F00300C1F303110131F5
:10179400C2F30622032842F20040C0F2F40004BF60
:1017A40047F64000C0F27D10B0FBF1F06968504389
:1017B400C1F34161022202EB4101B0FBF1F04BF2B3
:1017C4000041C0F2C441884208D9286810F0F00FE3
:1017D40015D02078800701D5A06880B1002614E0D8
:1017E400880304D40120BDE8F0874805FAD508F041
:1017F40088F94BF20041C0F2C4418842EED928680E
:10180400082161F30710286001262868616820F028
:1018140003000843286009F049FE814641F2883AF2
:101824002868616800F00C00B0EB810F06D009F065
:101834003DFEA0EB09005045F2D93CE02068810749
:1018440004D4E6B1286820F0F00017E0410742BF55
:10185400296841F4E0612960000704D5286807215C
:1018640061F30D202860A0686FF0070101EB3011CF
:10187400082976D2296821F0F001084328603868E5
:1018840000F00F00804519D2386820F00F0040EABC
:101894000800386009F00AFE814641F2883A00BF28
:1018A400386800F00F00404508D009F0FFFDA0EBB8
:1018B40009005045F4D90320BDE8F08720684107AA
:1018C40018D5E0686FF0030101EB302104290BD334
:1018D4004FEA302141B14DF23D60C0F600004FF4B3
:1018E400677109F063FCE068296821F4E06108434A
:1018F40028602068000718D520696FF0030101EB08
:10190400302104290BD34FEA302141B14DF23D601F
:10191400C0F6000040F2A33109F048FC20692968B0
:1019240021F4605141EAC000286008F0EAF829680F
:10193400C1F303114EF22412C0F60002515C01F00F
:101944001F0120FA01F141F26C70C1F2000041F272
:101954008072C1F2000200681160BDE8F04709F02E
:101964007DBD4FEA301100293FF484AF4DF23D6054
:10197400C0F6000040F27A3109F018FCA06879E75B
:101984002DE9F04182B004460068010307D14DF609
:10199400CB30C0F60000832109F008FC2068000366
:1019A40041F20C06C4F2020601D400256BE0206D5E
:1019B4004FEA3020042806D34DF6CB30C0F60000A1
:1019C4008B2109F0F3FBF06C5FEAC00808D4F06CDB
:1019D40040F08050F064F06C00F080500190019869
:1019E40047F20007C4F20007386840F4807038609A
:1019F40009F05CFD054600BF3868C00506D409F04F
:101A040055FD401B0228F7D9032535E0D6F884009C
:101A140010F44071206D26D0814225D0D6F8841070
:101A2400D6F8842042F48032C6F88420D6F8842084
:101A340022F48032C6F8842021F44072C6F884204F
:101A4400C907014610D009F031FD054641F2883737
:101A5400D6F88400800700F11F8209F027FD401B9F
:101A6400B842D1D8F4E70146D6F8840020F4407097
:101A74000843C6F884000025B8F1000F5EBFF06C7F
:101A840020F08050F0642068C10710D060680428FA
:101A940007D34DF6CB30C0F60000E02109F086FBF9
:101AA4006068F16F21F003010843F0672068810743
:101AB40012D5A0684FEAB001042907D34DF6CB3004
:101AC400C0F60000EA2109F071FBA068F16F21F073
:101AD4000C010843F0672068410712D5E0684FEA1B
:101AE4003011042907D34DF6CB30C0F60000F6219F
:101AF40009F05CFBE068F16F21F030010843F06706
:101B04002068010713D520694FEAB011042908D3CE
:101B14004DF6CB30C0F6000040F2031109F046FB4D
:101B24002069F16F21F0C0010843F0672068C10605
:101B340013D560694FEA3021042908D34DF6CB3020
:101B4400C0F600004FF4887109F030FB6069F16F52
:101B540021F440710843F0672068810613D5A06919
:101B64004FEAB021042908D34DF6CB30C0F600006B
:101B74004FF48E7109F01AFBA069F16F21F44061F2
:101B84000843F067206841060CD5E069002818BFB7
:101B9400B0F5805F40F02081F16F21F4405108439B
:101BA400F067206801060CD5206A002818BFB0F53C
:101BB400804F40F01F81F16F21F440410843F067EA
:101BC4002068C1050CD5606A002818BFB0F5803FB5
:101BD40040F01E81F16F21F440310843F067206822
:101BE400810313D5A06A032808D34DF6CB30C0F681
:101BF40000004FF4A47109F0D9FAA06AD6F8901045
:101C040021F003010843C6F890002068810513D52C
:101C1400E06A4FEAB041042908D34DF6CB30C0F650
:101C240000004FF4AA7109F0C1FAE06AF16F21F4DF
:101C340040210843F0672068400519D5206B4FEA1E
:101C44003051042908D34DF6CB30C0F6000040F2E1
:101C54005F1109F0ABFA206BF16F21F440110143DD
:101C6400B0F5801FF16702BF306840F48010306027
:101C74006078000719D5606B4FEAB051042908D386
:101C84004DF6CB30C0F600004FF4B97109F08EFA6E
:101C9400606BF16F21F440010143B0F5800FF167EF
:101CA40002BF306840F4801030606078C00612D5FE
:101CB400A06B002818BFB0F1807F40F0B780F16FAF
:101CC40021F040710143B0F1807FF16702BF3068B9
:101CD40040F480103060607880061AD5E06B40F0E4
:101CE4000061B1F1006F08D04DF6CB30C0F60000B2
:101CF40040F2971109F05AFAE06BF16F21F040615C
:101D04000143B0F1006FF16702BF306840F4801006
:101D14003060607840061AD5206C40F00061B1F163
:101D2400006F08D04DF6CB30C0F600004FF4D371ED
:101D340009F03CFA206CF16F21F040610143B0F1ED
:101D4400006FF16702BF306840F480103060607843
:101D5400000611D5606C002818BFB0F1805F73D104
:101D6400F16F21F040510143B0F1805FF16702BF90
:101D7400306840F480303060A078C00711D0A06C87
:101D8400B0F1004F18BF00286CD1F16F21F0404131
:101D94000143B0F1804FF16702BF306840F48030F6
:101DA4003060A078400713D5E06C002818BFB0F568
:101DB400801F64D1D6F8901021F440110143B0F58E
:101DC400001FC6F8901002BF306840F480103060E5
:101DD400284602B0BDE8F081B0F5005F3FF4DCAE08
:101DE4004DF6CB30C0F600004FF4937109F0DEF9E4
:101DF400E069D1E6B0F5004F3FF4DDAE4DF6CB30EF
:101E0400C0F600004FF4987109F0D0F9206AD2E6C8
:101E1400B0F5003F3FF4DEAE4DF6CB30C0F6000027
:101E240040F23B1109F0C2F9606AD3E6B0F1007FD9
:101E34003FF445AF4DF6CB30C0F6000040F28511BB
:101E440009F0B4F9A06B3AE7B0F1005F3FF488AF52
:101E54004DF6CB30C0F600004FF4DA7109F0A6F964
:101E6400606C7DE7B0F1804F8FD04DF6CB30C0F67B
:101E7400000040F2C51109F099F9A06C85E7B0F5AE
:101E8400001F97D04DF6CB30C0F600004FF4EC7134
:0C1E940009F08CF9E06C8DE7216DE5E5AC
:101EA00038B504460068C168490615D4C16841F0D8
:101EB0008001C16009F0FCFA2168C96849060BD4A9
:101EC000054600BF09F0F4FA401BB0F57A7F05D84B
:101ED0002068C0684006F5D5002038BD032084F88E
:081EE00025002168C96838BD26
:101EE80038B5044600685F21C0F20101C16009F0FD
:101EF800DBFA05462068C068800607D409F0D4FAE2
:101F0800401BB0F57A7FF5D9032038BD002038BDD5
:101F18002DE9F0411E460446806815460F4638B143
:101F28004DF2F960C0F600004FF49F6109F03CF9EA
:101F380009F0BAFA94F85D100129804606D101200B
:101F4800002F18BF002D0DD1BDE8F0816068B0F5F5
:101F5800827F0DD102200429F6D1A1680029EED094
:101F6800BDE8F081002EEFD094F85C00012802D182
:101F78000220BDE8F081012084F85C0094F85D003F
:101F880004281CBF052084F85D0000202066256415
:101F9800A4F84660A4F84460A763E687A687C4E966
:101FA80013002068E168426822F48055B1F5E06FBB
:101FB8002B4698BF03F58053721E88BF2B4643609B
:101FC80003685B065EBF036843F040030360B1F536
:101FD800E06F6168069EB2FA82F2B1FA81F14FEAC7
:101FE800521242EA51113DD931B137F8021BC16092
:101FF800A763E08F0138E0870127751CE08F20B9BF
:10200800B4F84600002800F0A1802068816889079C
:102018000ED5E18F002918BF002F09D0A16B00272A
:1020280031F8022BC260A163E18F0139E18700BF5B
:102038008168C9070DD0B4F8461051B1C068216C49
:10204800012721F8020B2164B4F846000138A4F8EE
:10205800460009F029FA002DD0D0A0EB0800B042C4
:10206800CCD36AE091B1E18F02294FF6FE7103D318
:1020780037F8022BC26005E03A780273A06B471C60
:102088004FF6FF71A763E08F0844E0870127751CAE
:10209800E08F18B9B4F84600002857D02068816846
:1020A800890719D5E18F002918BF002F14D0E18FB7
:1020B8000229A16B06D331F8022BC260A163E18F1C
:1020C800023907E009780173A16B20680131A16327
:1020D800E18F0139E18700278168C90725D0B4F865
:1020E800461011B3B4F84610022912D3C168226C05
:1020F80022F8021B2264B4F846100239A4F84610EC
:10210800B4F8461001290FD8416841F48051416064
:102118000AE0007B216C0870206C01302064B4F860
:1021280046000138A4F84600012709F0BDF9002D42
:10213800AED0A0EB0800B042AAD3012084F85D001D
:10214800002084F85C000320BDE8F0812046314679
:10215800424607F048FD38B120202066002084F868
:102168005C000120BDE8F081012084F85D000020BA
:1021780084F85C00206E002818BF0120BDE8F081BB
:1021880038B504460020C4F8900009F08DF921689C
:1021980005460A6812071AD56FF07E4C20464FF4A0
:1021A800001100222B46CDF800C005F0E3FD68B110
:1021B800206850E8000F216820F0800041E8000204
:1021C800002AF5D103202021882232E021680868FE
:1021D800400725D56FF07E4C20464FF48001002241
:1021E8002B46CDF800C005F0C5FDC8B1206850E801
:1021F800000F216820F4907041E80002002AF5D110
:102208002068083050E8000F216820F001000831EC
:1022180041E80002002AF3D1032020218C2208E0A3
:102228002020C4F88800C4F88C000021E1667022E0
:0C2238000020A150002184F8841038BD63
:1022440010B50446D0F8880020282FD1012061B3AE
:1022540013002AD02165A4F85430A4F856304FF066
:10226400000CC4F890C02120C4F88800E06FF8B1D5
:1022740047F61962C0F60002C26249F63B62C0F634
:102284000002026349F64162C0F60002426322681A
:10229400C0F838C0283209F05BFA48B11020C4F8FD
:1022A40090002020C4F88800012010BD022010BD39
:1022B40020684021016200BF2068083050E8000F08
:1022C400216840F08000083141E80002002AF3D17F
:0422D400002010BD19
:1022D80010B5134604468165A0F85C204FF0000C49
:1022E800C0F890C02220C4F88C00D4F88000F0B167
:1022F8000A4648F26D41C0F60001C16249F69B6189
:10230800C0F60001016349F64161C0F6000141636E
:102318002168C0F838C0243109F018FA38B1102003
:10232800C4F890002020C4F88C00012010BD20695A
:1023380050B100BF206850E8000F216840F4807059
:1023480041E80002002AF5D12068083050E8000F63
:10235800216840F00100083141E80002002AF3D169
:102368002068083050E8000F216840F0400008312C
:0C23780041E80002002AF3D1002010BD53
:10238400016851E8001F026821F0C00142E800130F
:10239400002BF5D10168083151E8001F026821F4CF
:1023A4000001083242E80013002BF3D12021C0F8C9
:0423B40088107047D6
:1023B8000100000004000000020000000800000006
:1023C80000000000040000000200000008000000F7
:1023D8002DE9F04104464DF2B970C0F600000AF04C
:1023E80075FCD4F89C0000287CD0D4F89C0006F03A
:1023F800ABFD404E0022334606F07AFC40F2E04244
:10240800C1F20002D2E900582A46434606F070FCA1
:10241800394F00223B4601F09FFD01F0ADFEC4F8A4
:102428009400B4F8CE00A4F89800B4F8CC00A4F84E
:102438009A004DF68D40C0F600002A4643460AF041
:1024480045FCD4F89C0006F07FFD0022334606F0D8
:102458004FFC02464DF2E800C0F600000B460AF0B9
:1024680035FCB4F9980006F06FFDA6F55915002261
:102478002B4606F03DFC02464DF2F700C0F6000080
:102488000B460AF023FCB4F99A0006F05DFD002221
:102498002B4606F02DFC02464DF2CB70C0F600002C
:1024A8000B460AF013FCD4F8940001F077FE0022E2
:1024B8003B4601F051FD02464DF6CC70C0F60000D7
:1024C8000B460AF003FC4DF2D570C0F600000AF086
:1024D800FDFB40F20000C1F200000021BDE8F04120
:1024E80007F033BF4DF6AA40C0F60000BDE8F04142
:0C24F80008F0AFBA00408F4080842E41F5
:102504002DE9F0474DF20210C0F600000AF0E0FB9E
:1025140040F20009C1F20009B9F8CE00A9F8A00000
:10252400B9F9A00006F012FD414F00223B4606F027
:10253400E1FB02464DF21910C0F600000B460AF00A
:10254400C7FBB9F9CE00B9F99810401A06F0FEFCA1
:102554008246884600223B4606F0CCFB02464DF2FA
:10256400EB70C0F600000B460AF0B2FB40F2D0401C
:10257400C1F2000030C84DF22810C0F60000224617
:102584002B460AF0A5FBD9F89C0006F0DFFC07F502
:1025940059160022334606F0ADFB02464DF2F9709F
:1025A400C0F600000B460AF093FBD9F89C0006F035
:1025B400CDFC0022334606F09DFB22462B4606F056
:1025C40099FB1C4B002206F067FA5246434606F07C
:1025D40091FB194C0022234601F0C0FC06F07CFC60
:1025E400C9F8A400D9F8A40006F0B0FC00222346E0
:1025F40006F080FB00223B4601F0B0FCA7F5D203B5
:10260400002206F049FA02464DF25B10C0F60000C3
:102614000B460AF05DFB4DF6E070C0F600000AF0D0
:1026240057FB48460021BDE8F04707F090BE00BFC5
:0C263400000059400000F0BF65CDCD4112
:102640002DE9F04F89B040F60004C4F6000420469E
:102650000121012209F080F99620FEF7DDFC41F20C
:102660009025C1F20005284609F0FEFA2046022115
:10267000002209F071F99620FEF7CEFC284609F0F9
:10268000F3FA20460221012209F066F99620FEF7AE
:10269000C3FC284609F0E8FA20460121002209F08F
:1026A0005BF940F6462006904FF47A7640F6D05417
:1026B000C1F20004204606A906AA02230096FFF7ED
:1026C0002BFC26208DF81800204606A906AA032315
:1026D0000096FFF721FC9DF81A000A285DD196208C
:1026E000FEF79AFC41F29020C1F2000009F0BCFA1A
:1026F0002046202105F07CFF4FF023088DF818803C
:10270000204606A906AA03230096FFF705FC9DF8BC
:102710001A00009600F0EF008DF8190043278DF89D
:102720001870204606A906AA0223FFF7F5FB8DF8CC
:102730001880204606A906AA03230096FFF7ECFBA3
:102740008DF81880204606A906AA03230096FFF7F5
:10275000E3FB9DF81A008DF8187000F09F00203000
:102760008DF81900204606A906AA02230096FFF755
:10277000D3FB8DF81880204606A906AA03230096ED
:10278000FFF7CAFB9DF81A0080060ED44DF299108F
:10279000C0F6000008F061F9FEE74DF6FC70C0F6E7
:1027A000000008F05AF900BFFEE743F25140ADF8CF
:1027B00018004FF000088DF81A803746204606A909
:1027C00006AA02230096FFF7A7FB31208DF8180018
:1027D000204606A906AA03230096FFF79DFB9DF855
:1027E0001A00342805D04DF60300C0F6000008F0AA
:1027F00034F94EF62549A246052400BFCDF81890BD
:102800008DF81280ADF81080504606A904AA032363
:102810000097FFF781FB9DF81000FF2805D19DF878
:1028200011009DF8181088420BD0013CE6D100BF82
:102830004FF09040202106F076FBC820FEF7ECFB1D
:10284000F6E79DF8120040F0600800274FF04509B8
:102850004FF47A7540F6D056C1F20006052400BF49
:102860008DF818908DF81980ADF81070304606A9D3
:1028700004AA02230095FFF74FFB9DF81000FF28E4
:1028800005D19DF811009DF8181088420BD0013C2D
:10289000E6D100BF4FF09040202106F044FBFA2023
:1028A000FEF7BAFBF6E705A8029000264EF625458E
:1028B00041F26C28C1F200084FF47A7440F6D05906
:1028C000C1F20009052700BFCDE90656404606A91A
:1028D000022203F04BFC8DF81A00ADF81460049648
:1028E000484606A904AA06230094FFF715FB9DF8A5
:1028F0001000FF2822D19DF811009DF81810884281
:102900001CD19DF812009DF81910884216D19DF82F
:1029100013009DF81A10884210D19DF815000390FD
:1029200040460299012203F021FC0399884205D117
:102930009DF8140000F0600060280BD0013FC3D167
:102940004FF09040202106F0EEFA4FF49670FEF71B
:1029500063FBF5E741F29020C1F2000009F084F931
:1029600000274EF6F24941F26C2BC1F2000B4FF4F6
:102970007A7540F6D058C1F200080526CDF81890B7
:10298000584606A9022203F0F1FB8DF81A000497BD
:10299000404606A904AA04230095FFF7BDFA9DF856
:1029A0001000FF2811D19DF811009DF818108842E1
:1029B0000BD19DF812009DF81910884205D19DF8A1
:1029C00013009DF81A1088420CD0013ED6D100BFEA
:1029D0004FF09040202106F0A6FA4FF4AF70FEF7BA
:1029E0001BFBF5E705A8029000264EF6214541F2B3
:1029F0006C28C1F200084FF47A7B40F6D059C1F23E
:102A000000090527CDE90656404606A9022203F033
:102A1000ADFB8DF81A00ADF814600496484606A97F
:102A200004AA0623CDF800B0FFF776FA9DF810004F
:102A3000FF2820D19DF811009DF8181088421AD166
:102A40009DF812009DF81910884214D19DF81300CA
:102A50009DF81A1088420ED19DF81500039040464B
:102A60000299012203F082FB0399884203D19DF968
:102A7000140000280BD4013FC4D14FF09040202116
:102A800006F051FA4FF4C870FEF7C6FAF5E741F2C6
:102A90009024C1F20004204609F0E6F89620FEF7E3
:102AA000BBFA204609F0E0F809F042FC204609F0A4
:082AB000DBF809B0BDE8F08F6E
:102AB8002DE9F04387B042F66450C0F600000DF1EE
:102AC800100890E88C0088E88C0041F26C20C1F274
:102AD80000004146022203F045FB8DF81200002059
:102AE8008DF80C00CDE901004FF47A7740F6D0500C
:102AF800C1F20000414601AA09230097FFF708FA2E
:102B08009DF80400FF2840F27805C1F2000533D192
:102B18009DF805009DF8101088422DD19DF80600FB
:102B28009DF81110884227D19DF807009DF81210D2
:102B3800884221D19DF80C8002A941F26C20C1F293
:102B48000000042203F00EFB404515D19DF8080053
:102B580000F0CC0084280FD19DF909009DF80B10D6
:102B68009DF80A20002860F3174141EA022000F18D
:102B78007F4109D5481C07E0B5F80A010130A5F8DE
:102B88000A01FFF759FD002041F21431C1F200019A
:102B98006FF000430A689A4201D1012606E0002638
:102BA800132A02F101020A60C8BF012641F2183156
:102BB800C1F200010A68104402EBD272A0EB620075
:102BC800086000EBD0704110C5F810112968C1EBFE
:102BD800600841F2DC20C1F20000C0F80080E86D16
:102BE800A9682A69401A504306F0AEF9544C0022ED
:102BF800234606F07DF806F06DF9C5F81401A8EB38
:102C0800000741F2E420C1F200000760B5F9540062
:102C1800B5F90610401A06F097F98046A869894662
:102C280006F092F942464B4601F096F900222346F7
:102C380006F05EF806F04EF941F2E021C1F200011B
:102C4800381A086006F080F93E4B002201F084F93A
:102C58003D4B002201F080F900224FF07A5301F039
:102C68007BF9044641EC100B40F2E040C1F2000051
:102C7800884680ED000BE86901F090FA334B00229A
:102C880006F036F82246434601F066F9044641EC60
:102C9800100B40F2D040C1F20000884680ED000BD6
:102CA800B5F95600B5F92010401A06F04DF98146DD
:102CB800E86A0F4606F048F9254B002206F018F896
:102CC8004A463B4601F048F9224B002205F0E2FE55
:102CD8002246434601F040F9044641EC100B40F20D
:102CE800D840C1F20000884680ED000B6FF3DF7119
:102CF800194B2046002201F0C7F910B1D5F8180188
:102D080007E00F4B20464146002201F025F906F066
:102D1800E1F8E8665EB1E86E296F8842C4BFE86EE4
:102D28002867E86E696F8842BCBFE86E686741F241
:102D3800B020C1F200000121016007B0BDE8F083B6
:102D480000408F40000008400000494080842E4128
:0C2D580065CDCD410000F03F002061403F
:0C2D640012EC0000000000000000000065
:102D70002DE9F84F2DED028B88B040F20004C1F22E
:102D8000000440F2F846C1F20006D4F85CB0D6E97F
:102D9000002352EA03004EF68061C0F2360106D1EC
:102DA000D4F82C0100FB01F20023C6E9002340F215
:102DB0000059C1F20009D9E900A55AEA0500CDE998
:102DC000063206D1D4F8300100FB01FA0025C9E92A
:102DD00000A5D4F8E400B4F97010B0EB010823D4D6
:102DE000B4F8520001F0DEF9DFF8909500224B466E
:102DF00005F082FF06460F46404601F0D3F9324601
:102E00003B4601F0ADF80646B4F9D6010F4606F090
:102E10009FF800224B4605F06FFF324640F2F8461D
:102E2000C1F200063B4636E0E06DB4F86810B0FB36
:102E3000F1F778428045404635DA06F089F8CDF85A
:102E400014B083468946384606F082F802460B469F
:102E500089F00041584605F04FFF41EC180BB4F8DB
:102E6000500001F09FF9DFF81835002205F044FF0B
:102E7000DFF81035002205F011FE41EC110BB0EE29
:102E8000480AF0EE680A09F085FE51EC100B5A462C
:102E9000DDF814B04B4601F063F806F01FF840F27D
:102EA0000059C1F20009C4F8F000D4F8E40000238E
:102EB00000280EDB1AEB080045EBE871C9E90001B8
:102EC0004EF68062C0F2360206F040F9C4F83001D6
:102ED00019E0C8F10001DDE90620401842EBE1717C
:102EE00003C64EF68062C0F2360206F02FF9C4F82F
:102EF0002C01D4F82C01E26D4FF47A714843B0FBF9
:102F0000F2F0A4F83C01D4F8F000D4E93E1209181C
:102F100042EBE070C4E93E10D4F8F000D4E9581256
:102F2000091842EBE070C4E95810D4E958014FF495
:102F300061694A46002306F027F8C4F84001D4F836
:102F40000001002841F2A425C1F2000501DC286837
:102F500078B1D4E9700110EB080041EBE871C4E9E5
:102F60007001D4E970014A46002306F00DF8C4F858
:102F7000C801D4F8E400D4E97812091842EBE070F3
:102F8000C4E97810D4E97801ABFB09974FF461628A
:102F9000002305F0F9FFC4F8D801D4F8D8010028BF
:102FA0004FF47A7006D0D4F84011D4F8D8214843B1
:102FB00090FBF2F0A4F8D601D4E93E01B9EB000091
:102FC00077EB0100B8BFC4E93E97D4E95801013856
:102FD00071F1000008DB0020C4E95800C4F840018A
:102FE000C4E97800C4F8D801E06DB4F85410D4F8FE
:102FF000D820B4F858309A4241F23436C1F2000673
:103000001ADD484301F0CEF8DD4B002205F074FED6
:1030100001F076F8D4F8E420101A4FEAE270884103
:103020000ADA308801303080B4F8561002B28A4291
:1030300004DDB4F8560000E000203080B4F85610EB
:1030400000B288424EDBC4E93E970020C4E9580034
:10305000C4F8400107F07BFC2868002804BF012069
:10306000286041F2A820C1F200000168012932D194
:1030700000210160D4F8E801D4E970234EF680699C
:10308000C0F23609A0FB090105F07EFFA4F8440157
:10309000D4F8EC01D4E96E23A0FB090105F074FF1C
:1030A000A4F84601D4F82811D4F8C821D4F8243162
:1030B000B4F94401B4F94671D4F8D860D4F8E49076
:1030C000CDE90007CDE902694EF22000C0F600000C
:1030D00009F000FE06E00020C4E97000C4F8C80151
:1030E000C4E96E00D4E93E014FF46162002305F0AB
:1030F0004BFFC4F8F400B4F8B80000285FD0B4F86F
:103100005001B0F57A7F40F2C880B4F85201C0088F
:103110007C2800F2C28041F23230C1F20000018806
:1031200001318AB20A2A0180C0F0BD8029680A22D2
:103130000129028040F0A080D4F82001B0F5616F31
:10314000C0F09A80D4F8200142F60071C0F20D015F
:10315000884200F29180D4F84001D4F84011002850
:1031600048BF4942C4F80C1109F042FCD4E970018F
:103170004FF2F019CFF6FF794A464FF0FF3305F0D2
:1031800003FFC4F8E801D4E96E014A464FF0FF336B
:1031900005F0FAFEC4F8EC01D4F82811D4F80C219B
:1031A000D4F8E831D4F82001D4F8D870D4F8E46029
:1031B000CDE900074DF2F710C0F6000059E0D4F851
:1031C000D800B4F88011884267DAD4F8D800B0F596
:1031D0007A7F62DD41F23230C1F2000001880131B4
:1031E0008AB20A2A01805ED329680A220129028054
:1031F00042D1D4F82001B0F5966F3DD3D4F8200128
:103200004FF68041C0F20A01884235D8D4F8400117
:10321000D4F84011002848BF4942C4F80C1109F005
:10322000E7FBD4E970014FF2F019CFF6FF794A4677
:103230004FF0FF3305F0A8FEC4F8E801D4E96E01B1
:103240004A464FF0FF3305F09FFEC4F8EC01D4F876
:103250002811D4F80C21D4F8E831D4F82001D4F89E
:10326000D870D4F8E460CDE900074DF2B410C0F690
:103270000000029609F02EFD0020C4F82401286009
:1032800041F2A821C1F2000101220A60C4E97000E4
:10329000C4F8C801C4E96E0005E041F23230C1F261
:1032A000000000210180B4F86400042848F2A069FD
:1032B000C0F201091ED8DFE800F0031A141711004C
:1032C000E26DD4E93E01A0FB09034FF4616701FB05
:1032D0000931A2FB072305F057FE0CE009F0F8FBCB
:1032E00009E009F0B1FB06E009F0C8FB03E009F0D2
:1032F00029F800E00020C4F80001E26DD4E93E01A5
:10330000A0FB090301FB09314FF46163A2FB032316
:1033100005F03AFE48F21F59C5F2EB1950FB09F0CF
:10332000410901EBD070A4F8CC0109F00BF850FB77
:1033300009F0410901EBD070A4F8CE0109F084FB3B
:1033400050FB09F0410901EBD070A4F8D00109F05D
:1033500095FB50FB09F0410901EBD070A4F8D201B4
:1033600009F0B6FB50FB09F0410901EBD070A4F85D
:10337000D40108B0BDEC028BBDE8F88F00408F404F
:08338000000059400000F0BFFD
:1033880038B541F20C31C1F200016FF000430A6810
:103398009A42044601D1012506E0501C0025B2F5E9
:1033A800A07F0860A8BF012541F21030C1F20000DB
:1033B8000168A1EB51112144016048F20000CFF6E9
:1033C800FF7000EB511005F0BFFD1D4B002200F00F
:1033D800C3FD1C4B002200F0BFFD00224FF07C53C0
:1033E80000F0BAFD05F076FD002D40F2D805C1F2D7
:1033F800000528600BD0286869688842C4BF28681F
:1034080068602868A9688842BCBF2868A860204608
:1034180005F09AFD0C4B002205F03CFB084B0022FE
:1034280000F09AFD074B002200F096FD00224FF0B5
:103438007C5300F091FD05F04DFDC5F8BC0038BD8A
:0C3448000070A740000026400000E0C01B
:1034540080B547F2A850C1F6FF709FED1E1A01888F
:103464009FED1D2A00EE101AB8EE400A20EE010A64
:1034740020EE020ABCEEC00A41F2D421C1F20001DE
:10348400408C81ED000A03EE100AB8EE433A23EEB5
:10349400011A10EE100A21EE020ABCEEC00A41F233
:1034A400D821C1F2000181ED000A10EE101A081AA9
:1034B40041F2D021C1F20001086000F071FE074B17
:1034C400002205F017FC40F2C842C1F2000203C218
:1034D40008BD00BF00803B45000080390000544017
:1034E40038B540F6B8314843000C00F059FE0446A4
:1034F40041F2D420C1F200000D46006800F050FEF5
:1035040002460B462046294600F024FD40F2C842FC
:10351400C1F200020CCA05F0EDFB094B002205F0D4
:10352400BBFA084B002200F019FD05F0D5FC40F26F
:10353400CC01C1F200010880BDE8384006F0D8BDD6
:0835440000003E400000594068
:0C354C0021D800083AD2000803DD000876
:1035580038B540F23415C1F200052889A0B12868B1
:1035680000F01CFE044668680D4600F017FE02468F
:103578000B462046294605F0BBFB054B002200F010
:10358800EBFC05F0A7FC00E0C04300B238BD00BF6B
:043598000000594096
:10359C002DE9F84F40F20009C1F2000941F208345C
:1035AC00C1F20004D9F828012168401AA9F89A013F
:1035BC0040F6E40AC1F2000A0AF104005146FC226A
:1035CC0006F016FA40F2E47BC1F2000B0BF104009A
:1035DC005946FC2206F00CFAD9F8E4C0CAF800C02F
:1035EC00D9F8D800CBF800006FF00040002240233F
:1035FC00D0460027064600BF58F8045B002D48BF94
:10360C006D42B54238BF2E465BF8041BBD4288BFE5
:10361C002F46002948BF4942814238BF0846914293
:10362C0088BF0A46013BE7D1BD1B48BF6D42101A4B
:10363C0048BF4042D9F85C10B9F86820B1FBF2F1F0
:10364C0046F26762C6F2666251FB02F1CA1002EBE7
:10365C00D1718D4202DA4FF0FF3047E0192802D2C7
:10366C004FF6FE7042E00027DA4313467E1C5AF8F0
:10367C002610B1EB0C0848BFC8F100089845C4BF30
:10368C0043463A463F2E8C463746EFD1202A2CD162
:10369C0000F082FD80460E46284600F07DFD024675
:1036AC000B464046314605F021FB124B002200F040
:1036BC0051FC05F00DFCA9F81C01D9F8280120607B
:1036CC00002040F23421C2F2000100BFC0F13F03E0
:1036DC0009EB430331F8042BA3F8F42131F8022C45
:1036EC00A3F8742201304028F0D1002000B2BDE8CC
:0836FC00F88F00BF0088C340F5
:103704002DE9F0416FF000400023591E40F23428A7
:10371400C2F200080E46002238F82350A84228BFFF
:10372400284688BF1E46AA429CBF2A461946013332
:10373400402BF1D108EB810108EB860349885B88B3
:10374400101ACF1A05F002FC3B4B002200F006FCD5
:1037540005F0C2FB05F0FAFB40F20005C1F20005DA
:103764000446D5F894000E4600F01AFD334B0022AF
:1037740005F0C0FA2246334600F0F0FB05F0ACFB3E
:103784000446384605F0E2FB2D4B002200F0E6FB30
:103794002C4B002200F0E2FB00224FF07C5300F09F
:1037A400DDFB05F099FBE96DB5F86820B1FBF2F19A
:1037B40046F26762C6F2666251FB02F18A1002EBBE
:1037C400D171220048BF62428A4202DA4FF0FF31CF
:1037D4002EE04FF6FE71020048BF42420A2A27D368
:1037E40005F0B4FB07460E46204605F0AFFB024643
:1037F4000B463846314605F07DFA134B002200F0A3
:10380400ADFB05F069FBA5F81E01D5F828014020A1
:1038140038F8041B81F40041A5F8F41238F8021CAE
:1038240081F40041A5F8741302350138F0D1002168
:1038340008B2BDE8F08100BF804F124080842E4161
:0C3844000070A740000026400088C34030
:1038500070B540F29C06C1F200067169401AA0F5ED
:10386000004005F075FB114B002200F079FB0022AF
:103870004FF07C5300F074FB0D4B002205F03CFA36
:103880000C4A0D4B05F038FA044630680D4605F039
:103890005FFB22462B4605F02FFA084B002200F072
:1038A0005FFB00F06DFCB06170BD00BF0070A74011
:1038B00000004440FCA9F1D24D62403F80842E417B
:1038C00070B540F2B006C1F200063168401AA0F5AA
:1038D000004005F03DFB114B002200F041FB0022AF
:1038E0004FF07C5300F03CFB0D4B002205F004FA36
:1038F0000C4A0D4B05F000FA044670680D4600F0C6
:1039000051FC0A4B002205F0F7F922462B4600F045
:1039100027FB05F0E3FAC6F8E00070BD0070A74091
:1039200000004440FCA9F1D24D62403F80842E410A
:1039300010B540F2C804C1F2000440F6B83121804D
:1039400000F030FC074B002200F00AFB064B00227F
:1039500000F006FB054B002200F002FB05F0BEFA6A
:10396000608010BD0070A740000008400000F03EDD
:1039700070B516460D460446049821604A6033B17E
:10398000012B09D14FF480524FF4C06106E04FF48F
:1039900080524FF4806101E000210022013818BFFD
:1039A00001204003C5E902202961284608F090FB68
:1039B00038B14DF67C50C0F6000007F04EF800F02C
:1039C00051FF284608F000FCB6F5964F0AD8059836
:1039D00000F0E8FB154B002200F0C2FA00F0D0FB2B
:1039E00001460BE040F2D66070434DF68361C4F2AD
:1039F0001B31A0FB0101012000EB9141284608F09A
:103A0000C7FB28684FF48072016841F08061016053
:103A100054F8270B214604F0C9FA30B14DF63700AF
:103A2000C0F6000009F056F9FEE770BD00000C403A
:103A30004FF6FF72A1B100B54AF2010C10F8013B3C
:103A40005A4008235FEAC27E8CEA520E08BF4FEA52
:103A5000520E013B7246F5D10139EFD15DF804EB0E
:043A600090B2704769
:103A640030B540F2000EC1F2000EBEF81850002B23
:103A740018BF9D420CD10B794C7944EA0325A5F17A
:103A84007E0313F17E0F07D883218154032110E0B4
:103A9400862181540B210CE049884BBA05EB030CB9
:103AA400ACF2FD11851811F5FE7F07D28321297030
:103AB400022110444170911C084630BD911C6200E3
:103AC40003242C706A7008440EEB4302557800F806
:103AD400025B12F8025B00F8015C013302316345BA
:043AE400F4D3E9E747
:103AE800F0B540F20006C1F20006002B358B18BF76
:103AF800AB420BD10D794B7943EA0525A5F17C043E
:103B080014F17C0F05D84FF4647110E040F686314B
:103B18000DE091F802C091F803E04EEA0C24254428
:103B2800A5F2FD1717F5FE7F05D24FF424718152D7
:103B380002201044F0BD073106EB440611F8027B61
:103B4800777011F8017C06F8027B0134AC42F5D39A
:103B580010218154104480F801C0A0F802E00371DC
:043B68000520E6E767
:103B6C0040F2BA00C1F200000088032803D8DFE855
:103B7C0000F0020F0B0D40F60000C4F600004FF4ED
:103B8C000051002207F0E2BE08F094BE06F03CBEE5
:043B9C0006F0E7BD8B
:103BA000F8B540F2E404C1F2000434F88C0C00F0E3
:103BB000F9FA3C4A3C4B00F0D3F905F08FF941F299
:103BC000F425C1F2000534F88C1C2E68A4F8BA6004
:103BD00054F80C7C874204DD41F2EC20C1F2000075
:103BE0000EE0084600F0DEFA304A314B00F0B8F93A
:103BF00005F074F9874241F2EC20C1F2000006DAC8
:103C00000021016029604FF0FF3000B2F8BD01686B
:103C1000002904BF0760394601F10A02974202DC1D
:103C20000A398F4205DA0021016029606FF0010036
:103C3000EBE7216834F9742C914205DA0021016028
:103C400029604FF6FD70E0E7701C42F63121884292
:103C5000286004D3206834F8741C401AA086B4F994
:103C6000340001281CDB606C44F20751CCF22E2199
:103C7000A0FB010141F2F020C1F20000090C026832
:103C80008A420DD0016041F2F820C1F200000168C3
:103C9000B4F93420A1EB9111114401608809E08648
:103CA0000020B2E77B14AE47E17AF03F0AD7A37059
:043CB0003D0AEF3F9B
:103CB40080B505F04BF9164B002200F04FF9154B77
:103CC400002200F04BF9144B002204F0E5FE134BE4
:103CD400002205F00FF8124B002200F03FF905F026
:103CE400FBF840F2CE01C1F200010880B1F90000F6
:103CF400B1F902209042B1F9000001DD488008BD0D
:103D0400B1F904209042BCBF0888888008BD00BF78
:103D14000070A7400000F03E00C082C000002440B4
:043D24000000594002
:103D280080B5A0F5004005F00FF90A4B002200F01D
:103D380013F9094B002200F00FF900224FF07C53D1
:103D480000F00AF900F018FA40F2D401C1F20001BB
:0C3D5800086008BD0070A7400000264075
:103D64002DE9F84F40F2E842C1F2000240F20004AB
:103D7400D2E9001B51EA0B00C1F200044EF6806048
:103D8400C0F2360006D1D4F8341141434FF0000B91
:103D9400C2E9001B009140F2F042C1F20002D2E9F4
:103DA400009A59EA0A0107D1D4F8381101FB00F945
:103DB4004FF0000AC2E9009AB4F87250D4F8E40053
:103DC400B4F97010461A21D4304600F0E9F980465F
:103DD4000F46284600F0E4F94E4D00222B4604F02D
:103DE40089FF42463B4600F0B9F88046B4F9D60153
:103DF4000F4605F0ABF800222B4604F07BFF424649
:103E04003B4600F0ABF805F067F801E0D4F8F000A9
:103E1400C4F87C01D4F87C01D4F8D81081FB0001EB
:103E24004FF47A72002305F0ADF8226ED4E95C37C2
:103E34001B184F41C4E95C37D4E95A37C01879419B
:103E4400C4E95A01D4F800014FF461610128A2FBCE
:103E540001580EDBD4F8D80080FB06014FF47A72C7
:103E6400002305F08FF8D4E96E2380185941C4E982
:103E74006E01D4E95C01281A78EB0100B8BFC4E9EB
:103E84005C58D4E95A01013871F10000A4BF002044
:103E9400C4E95A00D4E95A014FF46162002305F0E1
:103EA40071F8C4F84801D4E95C014FF4616200235D
:103EB40005F068F8C4F87801D4F80801D4F80811BA
:103EC4000023002812DB19EB010040F2F042C1F29A
:103ED40000024AEBE17103C24EF68062C0F2360280
:103EE40005F032F9C4F83801BDE8F88F494200986A
:103EF400401840F2E842C1F200024BEBE17103C208
:103F04004EF68062C0F2360205F01EF9C4F83401A0
:083F1400BDE8F88F00408F406A
:103F1C00034C206804348047FBE7FCF7DBFCFEE72E
:043F2C0000E20008A7
:103F300006F072FD4EF60850CEF200000549016011
:103F40004EF68850CEF20000016851F47001016015
:083F5000FFF7E4FF0000000888
:083F580083F0004304F09EBD5C
:103F6000F0B540F2FF7681EA030C16EA115E1EBF3F
:103F7000B64516EA1355B54252D021EA465141F4EE
:103F80008011A1FB024723EA465343F48013AE4459
:103F9000A0FB03650CF0004C36197D41A1FB0347E3
:103FA00047F10003A0FB0217F619654153F1000326
:103FB000094218BF46F0010640F2FE74B3F5007FD7
:103FC00013D2AEF5806EA64523D24CEA0331280306
:103FD00041EA155140EA16503203450872F1004299
:103FE00050F1000051EB0E51F0BDAEF2FF3EA64580
:103FF0000FD24CEAC321E80241EA555140EA56503B
:10400000F202450872F1004250F1000051EB0E51EE
:10401000F0BD1EEA0E0F2DD50CF000410020F0BDC2
:1040200016EA115F04BF01F000410020004218BFF2
:1040300041F0010116EA135F04BF03F000430022C0
:10404000124218BF43F0010306EA1354B44218BFEA
:10405000B64503D00CF000410020F0BD21F0004136
:1040600023F00043B1EB065F0CD8B3EB065F09D831
:1040700041B13BB10CF0004141F0FE4141F470010F
:104080000020F0BD40F20001C7F6F8710020F0BD3D
:104090004FF4001C1CEB410F98BF1CEB430F11D8D1
:1040A00051EA030C50EA4C0C5CEA020C0AD004D230
:1040B00082428B4180414042704790429941804109
:0840C0004042704700207047E8
:1040C8004FF4001C1CEB410F98BF1CEB430F11D899
:1040D80051EA030C50EA4C0C5CEA020C0AD004D2F8
:1040E8009042994180414042704782428B418041D1
:0840F8004042704700207047B0
:10410000C1F30A5240F21E439A1A15DA203225DD15
:10411000CB17C90241EA5051C00241F00041D141E0
:10412000D04048409140D14048405B1C18BF704788
:10413000404263EB01017047CB17C90241EA50517D
:10414000C00241F00041202A28BF202231FA02F0AB
:10415000190008BF70474042894170474B00004238
:1041600018BF43F0010313F5001F88BF21F0004181
:10417000002011F000415CBF6FF00041C043704768
:104180000B0D40F21E42D21A09DBCB0243EA50501B
:1041900040F00040202A28BF2022D040704749002C
:0441A00080417047A3
:1041A40050B140F21D42B0FA80F1521A8840C30A5D
:0C41B400400503EB02517047010070470A
:0841C000004870477C17001055
:1041C8005AB3844690EA01039B071FD1830707D09F
:1041D80011F8013B00F8013B521EF7D11CE0844660
:1041E800203A09D32DE9F007B1E8F807A0E8F80765
:1041F800203AF9D2BDE8F0071C3205D451F8043B47
:1042080040F8043B121FF9D2043205D011F8013BE3
:0C42180000F8013B521EF9D160467047CF
:1042240000220B0011001A0084465AB3830704D0FD
:1042340000F8011B521EF9D124E0C9B241EA012160
:1042440041EA0141202A11D3203A2DE9F0030B461B
:104254000C460D460E460F4688468946A0E8FA03EA
:10426400203AFBD2BDE8F00320320BD0042A05D358
:1042740040F8041B121F05D0042AF9D200F8011BD0
:08428400521EFBD16046704799
:10428C0000B50549FFF796FF4158044A002908BFBD
:10429C008118084600BD00BF080000000C0000009B
:0C42AC00F5D80008D8420008B84200080D
:1042B800B5CE0008D5CE0008E1CE0008EDCE000846
:1042C8000DCF000819CF00089BAC000869AC0008A6
:1042D800F7D80008A0DE0008A0DE0008A0DE00086D
:1042E800A0DE0008A0DE0008A0DE0008A0DE0008AE
:1042F800A0DE0008A0DE0008FFFFFFFFFFFFFFFFB2
:10430800FFFFFFFFFFFF0000BBD8000852DE0008D8
:1043180032D300086FDE000889D3000840DE0008A9
:0843280049DE000890D30008F3
:1043300070B59CB0044617A81421FFF773FF02A8BC
:104340005421FFF76FFF206800F130404FEA302022
:10435000062800F27081DFE810F0070089006E0186
:104360006E014600D50018014FF4004002904FF056
:104370008050139002A8FDF705FB002818BF00F03D
:1043800071FA41F20430C1F2000001684A1C026077
:1043900041F24C00C4F2020041B9016841F40051FD
:1043A0000160016801F4005101910199016841F037
:1043B00001010160006800F00100019001980320F4
:1043C000CDE917000026199617A94FF09040FCF789
:1043D00045FF41F23C15C1F200050820C4F202007D
:1043E0002860052081E04FF4803002904FF080403B
:1043F000149002A8FDF7C6FA002818BF00F032FAA0
:1044000041F20030C1F2000001684A1C026041F232
:104410004C00C4F2020041B9016841F480410160DE
:10442000016801F4804101910199016841F00201A4
:104430000160006800F002000190019842F2030060
:10444000179003200026CDE9180640F20040C4F67C
:10445000000017A9FCF702FF41F27C05C1F200053C
:104460003020C4F2020028602520CEE04FF4004046
:1044700002904FF08050139002A8FDF783FA0028B5
:1044800018BF00F0EFF941F20430C1F200000168FA
:104490004A1C026041F24C00C4F2020041B90168BA
:1044A00041F400510160016801F40051019101994A
:1044B000016841F001010160006800F00100019015
:1044C0000198C020179003200026CDE9180617A9EF
:1044D0004FF09040FCF7C2FE41F2DC05C1F200054E
:1044E0001C20C4F2020028602420C5E901068020B7
:1044F000C5E903604FF4007068614FF40060C5E9DE
:1045000006068FE04FF4803002904FF08040149008
:1045100002A8FDF737FA002818BF00F0A3F941F20E
:104520000030C1F2000001684A1C026041F24C00F8
:10453000C4F2020041B9016841F4804101600168A0
:1045400001F4804101910199016841F0020101608B
:10455000006800F00200019001984FF4404017906D
:1045600003200026CDE9180640F20040C4F6000002
:1045700017A9FCF773FE41F21C05C1F200054420A7
:10458000C4F20200286026203FE04FF48030029001
:104590004FF08040149002A8FDF7F4F9002818BFEE
:1045A00000F060F941F20030C1F2000001684A1CDD
:1045B000026041F24C00C4F2020041B9016841F4CA
:1045C00080410160016801F4804101910199016815
:1045D00041F001010160006800F0010001900198C4
:1045E0004FF44070179003200026CDE9180617A954
:1045F0004FF09040FCF732FE40F6BC75C1F200056A
:104600005820C4F2020028602720C5E90106802056
:10461000C5E903604FF4807068614FF40060A861E1
:104620002020E8612E62284604F021F808B100F04D
:0A46300019F96565AC621CB070BD9D
:10463A0070B588B068462021FFF7EFFD40F62044A8
:10464A00C1F2000440F20050C5F200002060201DB3
:10465A001421FFF7E2FD002501200426A6614FF48C
:10466A008071A183206284F82450C4E90B5584F830
:10467A003800E56384F840001C2161648021C4E9A4
:10468A0012152065204600F0DEFA002818BF00F057
:10469A00E4F81020C1F2C000009006200190072023
:1046AA0002900020C4F27F00CDE90306059520465A
:1046BA00694600F050FF002818BF00F0CEF808B095
:0246CA0070BDC1
:1046CC0020B594B005A83821FFF7A6FD6846142143
:1046DC00FFF7A2FD4FF4007002F09EFC05F0FBF911
:1046EC0041F29000C4F202000325016821F0180188
:1046FC0001602D2005904FF480300690012007902A
:10470C00CDE90A0002200C90CDE90D5010210F913B
:10471C000821CDE91010129005A802F007FD40B158
:10472C0072B64CF64670C0F6000006F090F900BF69
:10473C00FEE70F20CDE900050020CDE90200049032
:10474C0068460321FCF7C8FF38B172B64CF64670C8
:0E475C00C0F6000006F07BF9FEE714B020BDA9
:10476A0030B589B001A82021FFF757FD40F6B430D3
:10477A00C1F200000024012140F20062C5F20002E9
:10478A00C0E90024C0E90244C0E904410822826168
:10479A004FF4807282830425056280F82440C0E9C0
:1047AA000B4480F83810C46380F840101C2242641D
:1047BA008022C0E91224016500F045FA002818BFDA
:1047CA0000F04BF81020C9F2C000019006200290B8
:1047DA00072003907F20CDE90405069440F6B43003
:1047EA00C1F2000001A900F0B6FE002818BF00F0CF
:1047FA0034F80020CCF2527001900C20029040F65E
:10480A00B430C1F2000001A900F0A5FE002818BFCB
:10481A0000F023F805F1066001901220029040F69C
:10482A00B430C1F2000001A900F095FE002818BFBB
:10483A0000F013F80220C0F23040019018200290D4
:10484A0040F6B430C1F2000001A900F084FE00284D
:0A485A0018BF00F002F809B030BDED
:1048640072B64CF64670C0F6000006F0F4F800BFCD
:02487400FEE75D
:1048760080B541F26C20C1F2000043F20001C4F29F
:104886000201016040F2011181800721816010213F
:10489600C160FF2101610021C0E90511012101620A
:1048A60003F026FE002814BFBDE8084008BDFFF748
:0248B600D6BF6B
:0248B800FEE719
:1048BA00006843F20001C4F2020188420ED181B0BD
:1048CA0041F24800C4F20200016841F480510160DB
:0E48DA00006800F480500090009801B0704714
:0248E800FEE7E9
:1048EA0000B583B041F24800C4F202000022016818
:1048FA0041F004010160016801F00401029102998A
:10490A00016841F001010160006800F001000190B6
:10491A0001980B20002103F06FFB0B2003F0D8FB5A
:10492A000C200021002203F067FB0C2003F0D0FBCF
:10493A000D200021002203F05FFB0D2003F0C8FBCD
:10494A000E200021002203F057FB0E2003F0C0FBCB
:10495A000F200021002203F04FFB0F2003F0B8FBC9
:10496A0010200021002203F047FB102003F0B0FBC7
:10497A0011200021002203F03FFB03B011205DF853
:06498A0004EB03F0A5BBE5
:02499000FEE740
:1049920010B59CB0044617A81421FFF742FC02A8E8
:1049A2005421FFF73EFC206846F60041C4F20001A4
:1049B200884231D0A1F58061884268D14FF480509D
:1049C20002904FF00070109002A8FCF7DAFF002866
:1049D20018BFFFF746FF41F2FC20C1F20000016858
:1049E2004A1C026041F24C00C4F2020041B9C168A3
:1049F20041F00071C160C16801F00071019101993B
:104A0200016841F002010160006800F002000190BB
:104A12000198092060212CE04FF4805002904FF061
:104A22000070109002A8FCF7ACFF002818BFFFF737
:104A320018FF41F2FC20C1F2000001684A1C02602A
:104A420041F24C00C4F2020041B9C16841F0007168
:104A5200C160C16801F0007101910199016841F0E2
:104A620002010160006800F00200019001980B2031
:104A720018211791022118910021CDE919111B90DB
:104A820040F20040C4F6000017A9FCF7E6FB1CB098
:024A920010BD55
:024A9400FEE73B
:104A96002DE9F04687B001A81421FFF7C0FB41F2CB
:104AA6004C00C4F2020040F20049016841F00401E2
:104AB6000160016801F0040100910099016841F06C
:104AC60020010160016801F0200100910099016850
:104AD60041F001010160016801F0010100910099B6
:104AE600016841F002010160016801F002010091D4
:104AF6000099016841F008010160006800F00800B3
:104B060000900098C4F6000909F5806642F2030495
:104B1600304621460022002706F01BFF4FF090404A
:104B260030210022302506F014FF48464FF4E051AC
:104B360000228A4606F00DFF01940124CDE90247C2
:104B46000497304601A9FCF786FBCDE90154CDE96F
:104B560003774FF0904001A9FCF77DFBCDE901A456
:104B6600CDE90377484601A9FCF775FB4FF4806051
:104B7600CDE9010703944FF0904001A9FCF76BFBC8
:104B8600042001904FF40416CDE9026409F5006093
:104B960001A9FCF760FB8020CDE901060394484695
:104BA60001A9FCF758FB4FF40070CDE90107039704
:104BB600484601A9FCF74FFB08200021002203F01C
:104BC6001DFA082003F086FA17200021002203F0C0
:0E4BD60015FA172003F07EFA07B0BDE8F0864E
:024BE400FEE7EA
:104BE60010B541F2F014C1F2000447F60000C4F219
:104BF6000000206041F22E20C0F2E200606000203A
:104C0600A0600120E06004F110001421FFF707FB0B
:104C1600204604F0CDF9002818BFFFF720FE2046F5
:104C2600002106F0A4FF002818BFFFF718FE204653
:104C3600002104F0F1FE002818BFFFF710FE4FF424
:0A4C46008000BDE8104006F0E2BF58
:104C500070B582B004004FF0000001901DD02068B4
:104C600000F130404FEA3020062837D8012101FA00
:104C700000F010F0730F31D06068B0F5801F0EDBCC
:104C8000B0F5001F18DAB0F5C01F35DAB0F5801F97
:104C900043D0B0F5A01F38D13FE0012657E2B0F570
:104CA000403F13DBB0F5002F21DAB0F5403F34D0A0
:104CB000B0F5802F29D130E0B0F5201F21DAB0F512
:104CC000001F2AD0B0F5101F1FD126E028B3B0F581
:104CD000803F22D0B0F5003F17D11EE04DF2674073
:104CE000C0F6000040F29B1106F062FAC4E714D04F
:104CF000B0F5402F09D110E00FD0B0F5E01F04D17E
:104D00000BE00AD0B0F5301F07D04DF26740C0F677
:104D100000004FF4CE7106F04BFAA0684FEAF000A5
:104D2000042807D34DF26740C0F6000040F29D1101
:104D300006F03EFAE06840F40040B0F5004F07D0BE
:104D40004DF26740C0F600004FF4CF7106F030FA24
:104D5000206944F20A01884207D34DF26740C0F649
:104D6000000040F29F1106F023FA6069022807D381
:104D70004DF26740C0F600004FF4D07106F018FA0B
:104D8000607F022807D34DF26740C0F6000040F272
:104D9000A11106F00DFA206B4FEAB020042807D3CA
:104DA0004DF26740C0F600004FF4D17106F000FAF2
:104DB000E06AA0F588614FEA71111C2900F2CA81EE
:104DC000012202FA01F14DF6E572C1F6010211422B
:104DD00000F0C081606B002818BFB0F1806F40F018
:104DE000DB8094F83800022807D34DF26740C0F604
:104DF000000040F2A51106F0DBF9A069042809D0F3
:104E0000082807D04DF26740C0F600004FF4D37178
:104E100006F0CEF9E06B40F48050B0F5805F07D02B
:104E20004DF26740C0F6000040F2A71106F0C0F94D
:104E3000207F022807D34DF26740C0F600004FF4F0
:104E4000D47106F0B5F994F84000022807D34DF26A
:104E50006740C0F6000040F2A91106F0A9F96069A8
:104E600038B3206A0138102807D34DF26740C0F6E6
:104E7000000040F2AD1106F09BF994F824000228DE
:104E800009D34DF26740C0F600004FF4D77106F029
:104E90008FF994F8240001280BD1A06A0138082862
:104EA00007D34DF26740C0F600004FF4D97106F009
:104EB0007FF994F8240001280AD1607F012807D1E6
:104EC0004DF26740C0F6000040F2B71106F070F9ED
:104ED000E06D30B92046FFF72BFA0020206684F8F9
:104EE00058002068816889004FF6C071C5F6FF71CF
:104EF00042BF82680A4082608268D2001CD4826805
:104F000001F18051114041F08051816041F2807186
:104F1000C1F2000142F6635209688909C0F23E52AB
:104F2000A1FB02129109022202EB410101910199B8
:104F300011B101990139F9E78168C90009D4E16D1E
:104F400041F01001E165216E41F001012166012669
:104F500000E000268168E26D02F0100201F0040119
:104F60008918E16D14D121F481710231E165816804
:104F7000C9073ED140F4807140F20012C5F2000230
:104F80009142A2F1F80114D10A68D1F8003118E079
:104F900041F010000126D9E0B0F1006F3FF421AFDD
:104FA0004DF26740C0F600004FF4D27106F000F9F0
:104FB00017E7D1F800C4D1F80035D1F8002643EA4C
:104FC0000C031A43D20714D101F1F802904214BF26
:104FD0004FF4E0624FF44072B0F1A04F08BF4FF4BD
:104FE0004072D4F804C08B5823F47C1343EA0C03BA
:104FF0008B50617FE26BD4E9023542EA41312943AB
:1050000094F824201943012A41EA024106D1A26AF8
:105010000023CFF6FE7303EB42421143E26A22B152
:10502000236B02F478721A431143C26844F20703F7
:10503000CFF6F0731A401143C1600169626B21F031
:105040004061114301618168090771D494F83810F7
:10505000227F490041EA8231C26844F202039A4346
:105060001143C1602169026941B142F48032026199
:10507000D0F8C0206FF30D02114306E022F4803116
:105080000161D0F8C0106FF30D01C0F8C01094F8A2
:105090004010012948D1606C4FEAB000082807D3BE
:1050A0004DF26740C0F6000040F2762106F080F82D
:1050B000A06C4FEA7010092807D34DF26740C0F684
:1050C000000040F2772106F073F8E06C40F40070C5
:1050D000B0F5007F07D04DF26740C0F600004FF4F6
:1050E0001E7106F065F8216D41F4806040F20142C6
:1050F000904208D04DF26740C0F6000040F279219E
:1051000006F056F8216D2068D4E911CEE56C0269ED
:1051100040F2FD739A4342EA0C0242EA0E022A432D
:10512000114341F0010102E0016921F00101016137
:105130006169026B012922F00F0102BF226A013A64
:1051400011430163E06D012161F30100E065304628
:1051500002B070BD216801F130426FF0030303EB30
:105160003223032B0ED2B0F58C6F1EDBB0F5986F97
:1051700033DAB0F58C6F3FF42DAEB0F5946F3FF499
:1051800029AE4FE04FEA3222012A48D8B0F5986F95
:1051900017DAB0F58C6F27DAB0F5806F3FF41AAEEE
:1051A000B0F5846F3FF416AE2BE000283FF412AE4A
:1051B000B0F5806F3FF40EAEB0F5846F3FF40AAEE9
:1051C00030E0B0F5CC6F16DAB0F5986F3FF402AE70
:1051D000B0F5BC6F3FF4FEAD13E03FF4FBADB0F5AE
:1051E000BC6F3FF4F7AD1DE03FF4F4ADB0F5946F44
:1051F0003FF4F0AD05E03FF4EDADB0F5D06F3FF416
:10520000E9AD40F20042C5F200029142ABD002F596
:1052100000729142A7D0A2F580729142A3D00028DB
:105220003FF4D8AD4DF26740C0F6000040F2A31144
:0652300005F0BEFFCEE513
:1052360080B541F29020C1F2000043F20001C4F2B1
:1052460000010160032141604FF47A71C0E9021147
:10525600FCF7E9F9002814BFBDE8084008BDFFF7D0
:02526600FEBA8E
:1052680038B5016804468A688868C0074FF00000AE
:1052780017D012F0020214D1886800F00D0001283E
:105288001FD1886820F0004020F03F00023088607D
:105298000320086006F008F921688968C90701D168
:1052A800002038BD054600BF06F0FEF8401B032865
:1052B800206802D38168C90703D18068C007F3D189
:1052C80038BDE06D40F01000E065206E40F0010050
:0652D8002066012038BD34
:1052DE0038B541F24420C1F20000012104F06DFC0A
:1052EE004BF6BE6188426FD14DF2B930C0F6000068
:1052FE0005F0ACFB41F24424C1F200042046022129
:10530E0004F05BFC40F20005C1F200050321C5F874
:10531E002C01204604F051FCC5F830012046042132
:10532E0004F04BFCC5F834012046052104F045FC81
:10533E00C5F838012046062104F03FFCC5F82801C7
:10534E002046072104F039FCC5F80C01204608213F
:10535E0004F033FCC5F810012046092104F02DFCA1
:10536E00C5F8400120460A2104F027FCC5F8480183
:10537E0020460B2104F021FCC5F8F40020460C2138
:10538E0004F01BFCC5F8780120460D2104F015FC35
:10539E00C5F8D801D5F840014FF4616180FB0102D8
:1053AE00C5E95802D5F8D80180FB0102C5E978029B
:1053BE00D5F8480180FB0102C5E95A02D5F8F40080
:0A53CE0080FB0101C5E93E0138BD76
:1053D80070B582B004460020019021688A68D2071F
:1053E80044D14FF6C076C7F6FF76886806F17F028B
:1053F800104209D0E06D40F01000E065206E40F0EA
:1054080001002066012031E0886830400130886062
:1054180040F20010C5F200004FF4C162814208BF9B
:105428004FF40272B1F1A04F08BF4FF40272105846
:1054380000021DD406F038F821680A68D20714D192
:10544800054600BF8868C00703D18868304001302E
:10545800886006F029F8401B0328216802D30868F1
:10546800C007C7D00868C007ECD0002002B070BDE4
:1054780041F28070C1F2000042F663510068800971
:10548800C0F23E51A0FB0101880900EB40000C214D
:1054980001EB8000019001980028CBD001980138D9
:0254A800F8E723
:1054AA0038B540F20C15C1F2000541F2E821C1F20B
:1054BA000001E8690A68904200D138BD086004F02A
:1054CA000BFB41F24424C1F20004204601214BF6B1
:1054DA00BE6206F0B0FC2A6A2046022106F0ABFC46
:1054EA006A6A2046032106F0A6FCAA6A204604211D
:1054FA0006F0A1FCEA6A2046052106F09CFCEA694E
:10550A002046062106F097FC2A682046072106F065
:10551A0092FC6A682046082106F08DFC6A6B2046D8
:10552A00092106F088FCEA6B20460A2106F083FC72
:10553A0055F8182C20460B2106F07DFCEA6E204611
:10554A000C2106F078FCD5F8CC2020460D21BDE8C8
:06555A00384006F070BCB1
:105560002DE9F843044600200090206800F1304007
:105570004FEA302006280D4600F2DB80012101FAB7
:1055800000F010F0730F00F0D4806868B0F500717F
:1055900019DAA0F58071182908D8012202FA01F160
:1055A00041F24102C0F20412114219D1182800F24E
:1055B000D280012101FA00F041F24001C0F2041151
:1055C00008420DD1C7E0182900F2BC80012202FA7E
:1055D00001F141F24102C0F20412114200F0B28026
:1055E000A86806286BD2E8687F2840F20008C4F259
:1055F0007F0809D0404507D04DF26740C0F6000053
:1056000040F6D52105F0D4FD2869052807D34DF2D1
:105610006740C0F6000040F6D62105F0C9FD2068BD
:105620006969C068062202EA900040F6FF7222FA19
:1056300000F0814207D94DF26740C0F6000040F605
:10564000D72105F0B5FD286904280BD094F8400057
:10565000012807D14DF26740C0F6000040F6DB217B
:1056600005F0A6FDE9682868414540F2FF11C2F245
:10567000B05110D1884233DC7F21C1F650518842AD
:1056800072DC0221C0F23041884200F0AE8040213D
:10569000C1F6201184E0884234DC3F21C1F620119C
:1056A000884269DC012800F0A0800221C0F230416C
:1056B000884200F09A800421C0F6600192E0B0F1C7
:1056C000004F90D020F0010006283FF48CAF4DF23F
:1056D0006740C0F6000040F6D42105F069FD82E77E
:1056E00040F2FF71C2F63061884252DC40F2002184
:1056F000C2F2B051884200F0788040F20041C2F618
:1057000000214DE040F6FF71C3F2602188425CDC6D
:1057100040F20021C2F2B051884266D040F200410E
:10572000C2F60021884260D040F60001C2F6306126
:1057300058E04DF26740C0F6000040F6D22105F077
:1057400037FD22E7B0F5407F3FF44AAF40F2063123
:1057500088423FF445AF4DF26740C0F6000040F686
:10576000D32105F025FD3BE7013188423DD040F2D1
:105770000011C2F2801113E00131884235D080213E
:10578000C1F65051884230D040F20011C2F280116F
:1057900028E00131884228D044F20001C3F6C0213C
:1057A000884222D0216801F130414FEA3122062A95
:1057B00040F6E42100F25E83DFE812F09302420239
:1057C0005C035C0331025B027402013188420CD03D
:1057D00044F20001C3F6C021884206D048F200011D
:1057E000C3F6F061884240F0A88094F85800012880
:1057F00002D10220BDE8F8830121206884F8581006
:105800008168490734D4D5E90012C1F38461C2F339
:10581000012300EB830302F01F0291401F271E6B40
:1058200007FA02F226EA02021143196381688268CC
:1058300001F0040102F00802891840F0ED802F68A1
:10584000AB6800F114010422C7F3406602EAD752A4
:1058500051F82690C7F304560727B740B3F1004F1D
:1058600029EA07070AD18F50096841F000410BE08F
:10587000E06D40F02000E06501209FE2B3403B4333
:105880008B50096821F000414161D5E90431C268BB
:10589000042B0CD1016E016E2A685303C1F384619D
:1058A0006FD092FAA2F22068B2FA82F26BE000EBBB
:1058B0008300062303EA92022B68914003F0F8422A
:1058C0001143026E4FF20003C0F2FF331A4011433E
:1058D00041F000410166A86940F08070B0F1807F1E
:1058E00007D04DF26740C0F6000040F61C3105F0CD
:1058F0005FFC287F022807D34DF26740C0F6000006
:1059000040F61D3105F054FC2068296900F1600360
:10591000AA6953F8217027F080773A4343F8212091
:1059200029692A7F53F8217027F00077012A08BFE0
:1059300007F1007743F821706EE0216801F13041F2
:105940004FEA3122062A4FF42E6100F29382DFE8FB
:1059500012F00700E90191029102D301FE01150244
:105960004FF6FF71CCF6833188424FF42E6140F33D
:105970003B820F22C1F2C002904240F356820132B4
:10598000F5E1C2F3846291424FF6FF71C0F2070164
:1059900002BF026E22F000420266426E426E2B6827
:1059A0000B42C2F3846205D093FAA3F32068B3FAE2
:1059B00083F301E0C3F384639A4202BF426E22F094
:1059C00000424266826E826E2B680B42C2F3846292
:1059D00005D093FAA3F32068B3FA83F301E0C3F38D
:1059E00084639A4202BF826E22F000428266C26ED7
:1059F000C36E2A680A42C3F3846105D092FAA2F208
:105A00002068B2FA82F201E0C2F38462914202BFDE
:105A1000C16E21F00041C16681682B68C90740F062
:105A20008780EA68D0F8B06042454FF6FF71C0F257
:105A3000070102F0180221FA02F202EA03071A46ED
:105A40006FF3DF4226EA020647EA0607C0F8B070A5
:105A50006ED122B193FAA3F2B2FA82F200E09A0E6A
:105A6000013202F01E032A68092B02EA01030BD857
:105A700013B192FAA2F22A680A4211D092FAA2F362
:105A80002A68B3FA83F30CE013B192FAA2F22A68FF
:105A90000A4215D092FAA2F32A68B3FA83F310E00F
:105AA000930E0A4203F1010101F01F014FF00103BF
:105AB00003FA01F114D092FAA2F2B2FA82F210E0E3
:105AC000930E0A4203F1010101F01F014FF001039F
:105AD00003FA01F10DD092FAA2F2B2FA82F209E0D1
:105AE000920E013202F01F0202EB420241EA025121
:105AF0000DE0920E013202F01F0202EB420200237F
:105B0000CFF6206303EB0252114341F00071C1F361
:105B1000406200EB8200AA684769C1F304518A40E1
:105B2000072303FA01F127EA0101114341612B68C0
:105B30000020C8F20800034200F03F81266840F2CE
:105B40000011C5F200014FF4C1608E4208BF4FF44E
:105B50000270B6F1A04F08BF4FF402700022455802
:105B6000CCF22132934205F0E07204D01027C9F242
:105B7000C007BB422CD12B0200F11F8101F5A063AD
:105B80009E4203D0B6F1A04F40F017810B5823F08E
:105B9000E0731A4342F400020A5041F28070C1F2ED
:105BA000000042F6635100688009C0F23E51A0FB3C
:105BB0000101880900EB40000C2101EB800000BFCF
:105BC00000900098002800F0F98000980138F7E76D
:105BD0000027CCF25277BB4208BF5FEA126716D0AB
:105BE0000020CCF6843083424FF0000008BF15F44B
:105BF000800340F0E380B6F1A04F00F0D5808E42E4
:105C000000F0DC8000F0D08001F5C060CEE00B58E1
:105C100023F0E0731A4342F080720A50CDE00F2166
:105C2000C1F2C001884240F6E42161DD1022C1F2D8
:105C3000C00290423FF4D9AD2022C1F2F0420FE100
:105C40001F21C1F2F041884240F6E42142DD2022CA
:105C5000C1F2F04290423FF4C8AD41F20002C3F2FB
:105C6000602290423FF4C1AD42F20002C3F2906262
:105C7000FDE01F21C1F2F041884240F6E42129DD18
:105C800041F6FF72C3F29062904200F3E880202256
:105C9000C1F2F04290423FF4A8AD41F20002C3F2DB
:105CA0006022E4E041F20001C3F2602188423FF447
:105CB0009CAD42F20001C3F2906188423FF495AD81
:105CC00048F20001C3F6F06188423FF48EAD40F621
:105CD000E421CFE00422C0F6600290423FF485AD9B
:105CE00016E00F21C1F2C001884240F6E4213BDCFE
:105CF0000422C0F660029BE00721C0F69041884272
:105D00004FF42E615FDD1F22C1F2F042904243DC6E
:105D10000822C0F6904290423FF467AD1022C1F2D3
:105D2000C002A4E00F21C1F2C00188424FF42E61ED
:105D30006BDD41F6FF72C3F29062904214DD0132D6
:105D400090423FF452AD0022C4F252728FE00F2114
:105D5000C1F2C00188424FF42E6160DD41F6FF724E
:105D6000C3F29062904217DC1022C1F2C00290424E
:105D70003FF43BAD2022C1F2F04278E04FF6FF71D4
:105D8000CCF2517188424FF42E6158DD41F6FF721A
:105D9000C3F2906290421DDD013290423FF425AD86
:105DA0000022C4F2213262E001F50070816821F026
:105DB000E071114341F4800181600020002184F8EA
:105DC0005810BDE8F88342F20002CBF2986290428C
:105DD0003FF40BAD0022CCF2527290423FF405AD7D
:105DE0000022CCF6843242E042F20002CBF2906212
:105DF00090423FF4FAAC0022CCF2213290423FF4C0
:105E0000F4AC0022CCF2527231E00022CCF2293202
:105E100090423FF4EAAC0022CCF68C3208E000223B
:105E2000CCF25A7290423FF4E0AC0022CCF68432BD
:105E300090423FF4DAAC0822C0F6904217E0082204
:105E4000C8F6904290423FF4D0AC1022C9F2C00292
:105E500090423FF4CAAC2022C9F2F04207E001327E
:105E600090423FF4C2AC48F20002C3F6F0629042A6
:105E70003FF4BBAC4DF26740C0F6000005F098F966
:025E8000B3E489
:105E820010B58EB0044668463421FEF7CAF968465A
:105E9200FBF72DF98CB34DF6F460C0F6000004F068
:105EA200DBFD0498AA2837D102200090BB20049081
:105EB20005F031FD28B14CF65570C0F6000004F033
:105EC200CBFD02F0D5FD28B14DF2E930C0F600005D
:105ED20004F0C2FD4DF61470C0F6000004F0BCFDE3
:105EE200684600F0AEFBE0B14DF6D110C0F60000FE
:105EF20004F0B2FD02F0F0FE4BE00498BB2826D17C
:105F020002200090AA20049005F005FD08B34CF68B
:105F12005570C0F600003AE04DF6B410C0F600002D
:105F220013E002F0D9FE4DF62470C0F6000004F032
:105F320093FD05F004FD4DF2FF30C0F6000004F0C1
:105F42008BFD4DF63C70C0F6000004F085FD01208B
:105F520020E04DF2D730C0F6000004F07DFD02F0E3
:105F620087FD20B14DF2E930C0F600000FE04DF69A
:105F72005D10C0F6000004F06FFD684600F061FBA2
:105F820050B102F0A9FE4DF69310C0F6000004F0E5
:105F920063FD00200EB010BD4DF6D860C0F60000C3
:105FA20004F05AFD02F098FE4DF62470C0F600008F
:105FB20004F052FD05F0C3FC4DF2FF30C0F60000C4
:0E5FC20004F04AFD4DF67210C0F60000BDE777
:105FD00038B5044600200090206800F130404FEAB8
:105FE000302006280D4649D8012101FA00F010F0B2
:105FF000730F43D07F2D0BD00020C4F27F00854269
:1060000006D04DF6E610C0F60000852105F0D0F868
:1060100094F85800012801D1022038BD012084F8ED
:1060200058002046FFF720F9E16D10B141F0100152
:1060300030E041F2021291430231E165216805F03E
:1060400080438A6822F0404222F03F021A4402F163
:1060500000428A604DF60262C0F204028B68002B97
:1060600014DA009B01330093009B9342F6D3E06D5A
:1060700040F0100020F0020101200BE04DF6E61088
:10608000C0F60000842105F093F8B3E7E16D01222A
:0E60900062F30101E165002184F8581038BD6B
:10609E00F0B587B0044602A81421FEF7BCF82068BC
:1060AE0043F60041C4F2000188423AD141F24C005D
:1060BE00C4F202000225C16841F40041C160C1680A
:1060CE0001F4004101910199016841F00101016063
:1060DE00016801F0010101910199016841F004018B
:1060EE000160006800F00400019001984FF4004038
:1060FE00CDE902050026CDE90466062706974FF086
:10610E00904002A9FBF7A3F84FF4E05002A961C139
:10611E00CDE9056740F60000C4F6000002A9FBF7C2
:06612E0096F807B0F0BD79
:1061340030B55FEA520C03680ED08E46604600BF4D
:106144003EF8044B01383EF8025C45EA04441C6006
:10615400F6D14FEA8C0000E00020D2071CBF085A99
:066164001880186830BD30
:02616A0070477C
:10616C0038B505460220687728682B6A846844F0A5
:10617C000104012B846010D0022B0AD0032B10D108
:10618C002AB100BF51F8043B0360013AFAD1006810
:10619C0008E02846FFF7C8FF04E02846FAF770FF2E
:0A61AC0000E000200121697738BDF2
:0261B600704730
:1061B800F8B514460D464FEAF207042F064606D3F3
:1061C8004DF6A820C0F600005F2104F0EDFFE807B7
:1061D80001D10120F8BD1F20013805D300F01F01AF
:1061E80025FA01F1C907F7D0032FF2D8DFE807F045
:1061F8000A0205080F28ECD804E00728E9D801E0CE
:106208000628E6D830684561816821F018012143E5
:0662180081600020F8BDCA
:02621E007047C7
:1062200070B5040000F0FC80206846F20046C4F21D
:106230000006B04210D006F5806188420CD001F50E
:106240008061884208D04DF65C70C0F600004FF4C3
:10625000987104F0ADFF2068B0420AD16068102840
:1062600007D34DF65C70C0F6000040F2331104F025
:106270009FFFA068002818BFB0F5807F40F0EA803B
:10628000E068052807D34DF65C70C0F600004FF4B7
:106290009B7104F08DFF207C022807D34DF65C70C3
:1062A000C0F6000040F2371104F082FF607C022843
:1062B00007D34DF65C70C0F600004FF49C7104F0FB
:1062C00077FFA07C022807D34DF65C70C0F6000073
:1062D00040F2391104F06CFF60690138B0F5007FBD
:1062E00007D34DF65C70C0F600004FF49D7104F0CA
:1062F0005FFFA0690138802807D34DF65C70C0F6B7
:10630000000040F23B1104F053FFE0690138FF2820
:1063100007D94DF65C70C0F600004FF49E7104F092
:1063200047FF206A0138802807D34DF65C70C0F61D
:10633000000040F23D1104F03BFFA068B0F5407F43
:106340002FD1606A0138202807D34DF65C70C0F663
:1063500000004FF4A07104F02BFFA06A0138102850
:1063600007D34DF65C70C0F6000040F2411104F016
:106370001FFFE06A0138202807D34DF65C70C0F695
:1063800000004FF4A17104F013FF206B01381028B6
:1063900007D34DF65C70C0F6000040F2431104F0E4
:1063A00007FF606B1D2807D34DF65C70C0F6000038
:1063B00040F2451104F0FCFEA06B092807D34DF60E
:1063C0005C70C0F600004FF4A37104F0F1FEE06BC6
:1063D00040F08070B0F1807F07D04DF65C70C0F661
:1063E000000040F2471104F0E3FE94F85C0020B98D
:1063F00084F85D002046FEF7CCFA2068816921F020
:106400001001816105F054F8054600BF20688169DC
:10641000090707D505F04CF8401B0B28F6D312E00E
:10642000012070BD816941F00101816105F040F8F2
:10643000054600BF20688169C90718D105F038F802
:10644000401B0B28F6D3206E40F00100206601208F
:106450000321C5E0B0F5407F3FF412AF4DF65C700C
:10646000C0F6000040F2351104F0A2FE08E7816991
:1064700041F00201B042816104BF6168C6F80011B9
:10648000217C826922F04002012918BF40328261DA
:10649000617C826922F48042012908BF02F58042B2
:1064A0008261A17C826922F48052012918BF02F521
:1064B000805282618369D4E9021223F440730B4352
:1064C0008361836923F0A4038361036923F01003CC
:1064D00003619AB1012A0DD0022A09D0836943F0E1
:1064E000800383610369032A43F01002026105D12E
:1064F000202200E0042283691A438261B1F5407FC3
:1065000004F118010EC9A1F10105A3F101036FF017
:10651000FF0101EB022242EA456243EA0203656998
:10652000A1F57F4202EB054543EA0503C36110D1A3
:10653000636A02EB0342D4E90A5301EB03216B1EA9
:106540001943236B6FF00F0505EB03131943114338
:10655000C160D4E90D23E16BD0F8C0502943C0F8E5
:10656000C01006F5806506F58041A84204BF4AF2D6
:106570005071C4F2000106F500664AF25075C4F28B
:106580000005B04208BF05F554712164D0F8806061
:1065900026F4F81646EA0242C0F8802001F17002A3
:1065A0006264D0F8802022F0706242EA0362C0F890
:1065B000802001F1B000A06401F5C470E06401F531
:1065C0001870206501F51E70606501F55470002299
:1065D00041F8042B8142FBD30020A06520660121F5
:0665E00084F85C1070BDA0
:0665E600042002F0C3BC1A
:1065EC0070B5044642F21006C4F2020604F05AFFDB
:1065FC00054600BF3068C00306D504F053FF401BAE
:10660C00A042F7D9032070BD30684CF2FA3101403A
:10661C0008D041F24C70C1F2000042680A4342605B
:10662C00012004E03068C0070846ECD0012131603D
:02663C0070BD2F
:06663E00802002F097BC71
:106644002DE9F04F83B004460068402807D34CF688
:106654006870C0F6000040F23B1104F0A7FD41F25F
:106664004C7BC1F2000B9BF80000012801D10224ED
:10667400DDE242F21405C4F2020501208BF80000A9
:106684004FF0000ACBF804A0206847F2E058C1F6A6
:10669400FF78C1074FF6FF7600F07A80271D97E850
:1066A4008006042F4ED8032F4CD0B8F80000B04217
:1066B40002D1802031460FE0B8F80020B2F5007F07
:1066C40001D1802007E02020B242314604D0B2F547
:1066D400807F08BF40201146814509D34CF668707D
:1066E400C0F600004FF42A7104F060FDB8F8001001
:1066F400B14208D0B8F80000B0F5007F03D0B04232
:1067040029D1202000E08020824507D34CF6687010
:10671400C0F6000040F2A92104F048FD4FF47A705D
:10672400FFF762FF10B14FF0010A30E0042F21D8C7
:1067340005F11800DFE807F01B03161E190005F128
:106744001C0014E04CF66870C0F6000040F2A7216B
:1067540004F02CFDA9E7B0F5807F4FF02000D3D1E1
:106764004020D1E705F1380001E005F13C0049EA99
:106774000A410160286840F4003028604FF47A70C0
:10678400FFF732FF5FEA000A18BF4FF0010A2068E2
:10679400800701D4D1461BE02669AA2E18BFBB2E60
:1067A40037D14FF47A70FFF71FFF4FF0010978B922
:1067B400E86820F0FF003043E860286840F40030C7
:1067C40028604FF47A70FFF70FFF002808BFD14606
:1067D4002078400740F1C280D4E9056A701E4FF664
:1067E400FF71C0F20101884207D34CF66870C0F60D
:1067F400000040F2193104F0D9FC4FF47A70FFF72D
:10680400F3FE10B14FF00109A8E0F0070CD1804667
:1068140019E0CC2EC5D04CF66870C0F600004FF4D9
:106824003A7104F0C3FCBCE70AF4E068B8F5A06F61
:1068340007D34CF66870C0F6000040F22F3104F024
:10684400B5FC4FF4E06006F0060140EAC121700790
:106854000AEAC62000F480500AF4005248BF1044EB
:1068640016F4805241EA82010AF4804218BF1044AF
:1068740006F0780241EA423132070AF4803248BF16
:106884001044F2060AF4003248BF1043B2060AF478
:10689400802248BF104372060AF4002248BF104306
:1068A40016F0800241EA42310AF4801218BF104304
:1068B400B2050AF4000248BF104372050AF0807260
:1068C40048BF104332050AF0007248BF1043B204B7
:1068D4000AF0806248BF104372040AF0006248BFA5
:1068E400104340EA08074FF0607000EA863006F46F
:1068F400C04240EA4230320401EB000811D51AF0DC
:10690400405507D14CF66870C0F6000040F2BB3128
:1069140004F04CFC2F4348F0405842F21405C4F2F2
:10692400020516F480300AF0804118BF0F43E9686D
:1069340048EA803021EA00003843E860286840F4DF
:10694400003028604FF47A70FFF74EFE002818BF1D
:106954004FF0010947F2E058C1F6FF7820780007AC
:1069640040F1E380D4E9086A564500F0DE804746EA
:10697400E069019000F0030002900138022807D377
:106984004CF66870C0F600004FF47D7104F00EFC04
:106994000025C0F60405B6F1006F05F580280CD378
:1069A40038884FF6FF71884240461EBF39684FF061
:1069B400006061F39920864207D34CF66870C0F6F4
:1069C400000040F2F63104F0F1FBBAF1006F0BD392
:1069D40038884FF6FF7188421EBF38684FF0006850
:1069E40060F39928C24507D34CF66870C0F60000DE
:1069F40040F2F73104F0DAFB4FF47A70FFF7F4FD5C
:106A0400B84630B14FF0010942F21405C4F2020550
:106A14008BE0C4F201000068C0053888029A4FF682
:106A2400FF7108D488424FF000610DD038680D46DC
:106A340060F3582508E0884229464FF000651EBFE0
:106A44003868294660F3582142F21400C4F2020067
:106A5400C0684002019800F0004013D4012A24D1F8
:106A640042F21403C4F2020306F1784219696FF387
:106A74000E0141EA121119610AF17841090903F181
:106A8400140238E0012A24D1721A42F21407C4F223
:106A94000207AAEB01013B69C9086FF30E0343EA3D
:106AA400D2023A6107F1140225E0022A28D142F207
:106AB4001403C4F2020306F17842196B6FF30E015A
:106AC40041EA121119630AF17841090903F1340208
:106AD40011E0022A14D1721B42F21407C4F2020715
:106AE400AAEB05013B6BC9086FF30E0343EAD2021C
:106AF4003A6307F1340213686FF30E03194311600C
:106B040042F21405C4F20205696921F00041084308
:106B14006861286840F4003028604FF47A70FFF709
:106B240063FD002818BF4FF001092078800650D576
:106B3400D4E90B6A701E022807D34CF66870C0F6BD
:106B4400000040F2654104F031FBB8F800004FF654
:106B5400FF71884208D0B8F80000B0F5007F03D078
:106B640088421BD1202000E08020824507D94CF6C2
:106B74006870C0F6000040F2664104F017FB4FF461
:106B84007A70FFF731FD10B14FF0010921E0012EB9
:106B94000BD0022E11D105F1600008E0B0F5807F22
:106BA4004FF02000E1D14020DFE705F15C000168EF
:106BB40021F0FF0141EA0A010160286840F4003035
:106BC40028604FF47A70FFF70FFD002818BF4FF0CC
:106BD40001092078C00601D44C4625E0D4F828A049
:106BE4006FF480301AEA000F07D04CF66870C0F6D4
:106BF400000040F29A4104F0D9FA4FF47A70FFF79A
:106C0400F3FC012480B9E86D20F4803040EA0A00E6
:106C1400E865286840F4003028604FF47A70FFF784
:106C2400E3FC002808BF4C4600208BF800002046F7
:066C340003B0BDE8F08F83
:106C3A0010B540F62034C1F2000443F60000C4F255
:106C4A00010020604FF4964060600020C4E9020011
:106C5A004FF4806020610C20606104F11800142157
:106C6A00FDF7DBFA204605F02EFA002818BFFDF7DB
:106C7A00F4FD2046002105F0D0FA002818BFFDF7E0
:106C8A00ECFD2046002103F07DF9002818BFFDF72E
:106C9A00E4FD204603F035F9002814BFBDE8104092
:066CAA0010BDFDF7DABD8C
:106CB0002DE9F8430446006880690840401AB0FA9C
:106CC00080F0B2EB501F26D191460E461F46DDF8EC
:106CD00020805D1C204639464246FAF735FC48BB09
:106CE00085B104F0E5FB21681FB1A0EB0800B842B4
:106CF00009D988693040801BB0FA80F0B9EB501F89
:106D000001D10BE0216888693040801BB0FA80F027
:106D1000B9EB501FDED00020BDE8F883606C40F076
:106D200020006064202084F84100002084F84200A4
:0A6D300084F840000120BDE8F8835C
:106D3A002DE9F0419CB0044617A81421FDF76DFA1D
:106D4A0002A85421FDF769FA206844F20041C4F20E
:106D5A00000188423BD001F57441884240F0A68088
:106D6A000120029002A8FAF708FE002818BFFDF7D2
:106D7A0074FD41F25800C4F20200816841F4804176
:106D8A008160806800F48040019001986C20C4F210
:106D9A000200D0F8E01F41F00401C0F8E01FD0F86B
:106DAA00E00F00F0040001900198302017900220B3
:106DBA0018900020CDE9190007201B9040F600002A
:106DCA00C4F6000017A9FAF744FA252466E002255A
:106DDA00029502A8FAF7D1FD002818BFFDF73DFD7C
:106DEA0041F25800C4F2020040F26C08016841F412
:106DFA0000310160006800F400300190C4F202081A
:106E0A000198D8F8E00F40F00100C8F8E00FD8F870
:106E1A00E00F00F00100019001980C20CDE9170560
:106E2A000027CDE9197707201B9017A94FF090404A
:106E3A00FAF70FFA40F65C75C1F200051A20C5E9A7
:106E4A000080AF608026C5E90376C5E90577C5E904
:106E5A000777284601F006FC002818BFFDF7FDFC5D
:106E6A00C4F88050AC6240F6FC65C1F2000508F136
:106E7A00140028601B2068601020C5E90207C5E9D4
:106E8A000467C5E906772F62284601F0EBFB002864
:106E9A0018BFFDF7E2FCE567AC6226242046002114
:106EAA00002201F0A9F8204601F012F91CB0BDE851
:026EBA00F08165
:106EBC0070B5044600688069800614D415460E46E9
:106ECC00204631462A46FAF739FBD0B904F0EAFAE3
:106EDC00216816B1401BB04202D98869800604D5DE
:106EEC0088698006ECD5002070BD606C40F02000F5
:106EFC006064202084F84100002084F8420084F86B
:066F0C004000012070BDF1
:106F120010B596B0044602A85021FDF782F9206808
:106F220045F60041C4F20001884216D14FF40050E8
:106F3200019001A8FAF725FD002818BFFDF791FC82
:106F420041F25800C4F20200016841F400010160FC
:0E6F5200006800F400000090009816B010BD1A
:106F600038B505004FD0286845F60041C4F200014D
:106F7000884206D04DF2DF50C0F60000872104F0B1
:106F800017F995F8910220B985F890022846FFF785
:106F9000C0FF032085F89102286805F0A3F928793D
:106FA00000B305F110010022012300244B7001F809
:106FB000284B013401F8252C41E90622844241F88E
:106FC000102CF3D105F5A871002200234A7001F8B6
:106FD000283B013301F8252C41E90622834241F880
:106FE000102CF3D195E8070003F028F8002028734F
:106FF000012185F89112A97A012903D1284602F0CE
:0A7000005BFD002038BD012038BD03
:10700A0041F27070C1F2000041F2A021C1F2000108
:0A701A0000680A681044086070471F
:1070240010B547F20004C4F20004E8B3B0F5007FE1
:1070340010D0B0F5806F06D04DF66A30C0F600006F
:107044009D2104F0B3F82068022161F34A202060F6
:10705400002010BD2068D4F8801000F4C060B0F5A2
:10706400806F41F48070C4F88000F1D12068012160
:1070740061F34A20206041F28070C1F200003222A4
:10708400006850434DF68362C4F21B32A0FB020237
:1070940001EB9240002100BF6369013841F1000215
:1070A4005B052BD552B3F7E72068D4F8801000F4C1
:1070B400C060B0F5806F21F48070C4F88000C7D13F
:1070C4002068012161F34A20206041F28070C1F2FE
:1070D40000003222006850434DF68362C4F21B3232
:1070E400A0FB020201EB9240002100BF636901385A
:1070F40041F100025B0501D5002AF7D16069400522
:06710400A6D5032010BD1A
:10710A0010B504466FF00200044207D04DF20D405C
:10711A00C0F6000040F2A22104F045F83020C4F283
:0E712A000100016821F002012143016010BD47
:107138002DE9F04182B0040000F00381206858B1C5
:1071480010F02F0108D14DF23D60C0F6000040F26A
:10715800451104F029F82068C00741F20006C4F27E
:10716800020642D12078800768D42078000700F111
:10717800A6802078400740F18981A068052805D8B5
:10718800012101FA00F010F0230F07D14DF23D6004
:10719800C0F600004FF4FA7104F006F8B06D5FEA2B
:1071A800C00808D4B06D40F08050B065B06D00F0F4
:1071B80080500190019847F20007C4F20007386830
:1071C800C00500F1CD80386840F48070386004F064
:1071D8006BF905463868C00500F1C28004F064F90F
:1071E800401B022800F27C82F4E76068002818BF80
:1071F800B0F5803F40F0A780B06800F00C01F0685F
:10720800082900F07F8081F00C01032222EA0000A7
:107218000844B0FA80F0400974D161683068B1F56B
:10722800803F07D0B1F5A02F40F0C08040F4802007
:107238003060306840F480303060C0E0E06840F48E
:107248008070B0F5807F07D04DF23D60C0F6000039
:107258004FF4C07103F0A8FF2069802807D34DF2CE
:107268003D60C0F6000040F2811103F09DFFB06858
:10727800F16800F00C0004284DD001F0030180F003
:107288000C0081F002010844B0FA80F0400942D1B4
:10729800E0680028306800F09F8040F4807030601B
:1072A80004F002F9054600BF3068400500F1A580EA
:1072B80004F0FAF8401B022800F21282F4E7606931
:1072C800022808D34DF23D60C0F600004FF4E47187
:1072D80003F06AFF60690028D6F8940052D040F0A5
:1072E8000100C6F8940004F0DFF80546D6F89400CB
:1072F80080073FF53EAF04F0D7F8401B022800F2A4
:10730800EF81F3E7306880037FF52CAF60680028D1
:107318007FF428AF15E03068400501D5E06880B1FA
:107328007068216920F0FE4040EA0160706041F217
:107338006C70C1F20000006804F08EF800283FF479
:1073480014AF0120CDE1B0F5A02F3FF455AF4DF2B9
:107358003D60C0F6000040F24B1103F025FF4BE7FB
:10736800A168D6F89000012907D005294DD140F031
:107378000400C6F89000D6F8900040F00100C6F866
:1073880090004DE020F00100C6F8940004F08CF85D
:10739800054600BFD6F8940080077FF5EAAE04F0F2
:1073A80083F8401B022800F29B81F3E720F4803029
:1073B8003060306820F480200029306041D004F02B
:1073C80073F80546306880033FF5CCAE04F06CF8DE
:1073D800401B6428F6D983E120F48070306004F003
:1073E80063F80546306840057FF5BFAE04F05CF8E9
:1073F800401B022800F27481F4E77068216920F0CC
:10740800FE4040EA01607060AFE620F00100C6F877
:107418009000D6F8900020F00400C6F89000F1B172
:1074280004F042F8054641F2883700BFD6F89000CC
:10743800800724D404F038F8401BB84200F2508189
:10744800F4E704F031F80546306880037FF58AAE2A
:1074580004F02AF8401B642800F24281F4E704F0A3
:1074680023F8054641F28837D6F89000800706D5FC
:1074780004F01AF8401BB84200F23281F4E7B8F180
:10748800000F5EBFB06D20F08050B0652078800698
:107498004FD4E069032808D34DF23D60C0F60000E0
:1074A8004FF4197103F080FEE069002800F0238191
:1074B800B16801F00C010C295DD1012800F011819F
:1074C800F068216A00F003028A427FF43AAF616AE9
:1074D8006FF00F0202EB011100F0F0028A427FF414
:1074E80030AFA16A00F4FE42B2EB012F7FF429AF5E
:1074F800E16A00F07842B2EBC16F7FF422AF216BF2
:107508000022CFF6E07202EA0151A1F5001100F461
:10751800C0028A427FF415AF00F0C060616B4FF083
:107528007E4202EA016101F17E4188427FF409AF9F
:10753800E1E0A069022808D34DF23D60C0F60000E2
:1075480040F23B2103F030FEA0690028D6F89800ED
:107558006BD040F00100C6F8980003F0A5FF05467F
:10756800D6F89800800794D403F09EFF401B0228A9
:1075780000F2B680F4E7022869D1206A032801D80E
:10758800012807D14DF23D60C0F6000040F26E219F
:1075980003F00AFE606A0138102807D34DF23D60F7
:1075A800C0F6000040F26F2103F0FEFDA06A083823
:1075B800782807D34DF23D60C0F600004FF41C71E7
:1075C80003F0F2FDE06A02381E2807D34DF23D6051
:1075D800C0F6000040F2712103F0E6FD206B082898
:1075E80000F28B80012101FA00F010F4AA7F00F06C
:1075F8008480606B082800F28980012101FA00F07C
:1076080010F4AA7F00F08280306820F0807030602B
:1076180003F04AFF054600BF3068800127D503F014
:1076280043FF401B02285BD8F6E720F00100C6F8AC
:10763800980003F039FF0546D6F8980080077FF5D3
:1076480028AF03F031FF401B022849D8F4E730681F
:1076580020F08070306003F027FF04463068800116
:1076680042D503F021FF001B022839D8F6E7F0685D
:10767800226A48F20C01C0F29F1108401043616A67
:107688006FF00F0202EB0111A26A084340EA0220E0
:10769800216B0022CFF6E07202EA0151A1F5001138
:1076A800E26A084340EAC260616B4FF07E4202EA38
:1076B800016101F17E410843F060306840F080705C
:1076C8003060F06840F08070F06003F0EDFE044632
:1076D800306880010FD403F0E7FE001B0228F7D9B9
:1076E800032002B0BDE8F081F0684FF6FC71CFF6D8
:1076F800EE610840F0600020F3E74DF23D60C0F60F
:10770800000040F2722103F04FFD72E74DF23D6038
:0E771800C0F6000040F2732103F046FD74E756
:107726002DE9F04190460446006840F20017C5F284
:1077360000074FF4C162B84208BF4FF40272B0F1BD
:10774600A04F08BF4FF402720E46D55900F13042E1
:107756004FEA3222062A2ED80121914011F0730FEA
:1077660029D08168490703D494F85810012902D119
:107776000220BDE8F08105F01F05012107F5A06292
:1077860084F85810904218BF002D1ED12046FDF7F0
:1077960020FEF0B92168E06D40F60172904300F5D5
:1077A6008070B942E0651AD007F5806081421CD12D
:1077B60007F5407015E04DF26740C0F6000040F254
:1077C600DB7103F0F2FC2068CBE7052DDED0092D36
:1077D600DCD0002084F858000120BDE8F0814FF08D
:1077E600A040884218BF002D03D1E06D20F4801020
:1077F600E065E06D0022C004104644BF206E20F014
:1078060006002066606D4BF2CD43C0F60003C362EE
:1078160047F63F13C0F60003036347F6EF13C0F6BF
:10782600000343631C230B6084F858204A6842F027
:1078360010024A60CA6842F00102CA60403132460C
:10784600434603F084FF21688A6822F0004222F052
:0A7856003F0204328A60BDE8F081B1
:107860002DE9F04F83B09A4690460D460646002417
:107870008DF8074003F01CFEAAEB000000EB080B9C
:1078800003F016FE41F28071C1F200013768096809
:1078900023225143090D01FB0BF10291B9682942E2
:1078A00049D0824608F10109384600BFB5F5C06FDE
:1078B00002BF397B8DF807109DF80710B9F1000F52
:1078C0000DD003F0F5FDA0EB0A0058450CD202994B
:1078D0000298013800290290306808BF8B46816801
:1078E0002942E3D1002426E0D6E90001B1F5827FE8
:1078F000426822F0E00141600AD1B168B1F5004F61
:1079000002D0B1F5806F03D1016821F04001016020
:10791000B16AB1F5005F07D1016821F4005101603F
:10792000016841F400510160012086F85D000020EB
:0E79300086F85C000324204603B0BDE8F08F0B
:06793E00806A00F069BA46
:10794400F8B515460E46044603F0B0FD281A87190B
:1079540003F0ACFD41F28071C1F200010968C1F38A
:10796400CB317943009121688A68120613D5054604
:10797400013600BF66B103F099FD401BB8420CD23A
:1079840000980099013900280091216808BF074632
:1079940088680006EED40020F8BDD4E90001B1F5F2
:1079A400827F426822F0E00141600AD1A168B1F50A
:1079B400004F02D0B1F5806F03D1016821F040017E
:1079C4000160A16AB1F5005F07D1016821F400519B
:1079D4000160016841F400510160012084F85D00F8
:0A79E400002084F85C000320F8BDC9
:1079EE00806AC16D41F04001C165016E41F0040134
:0679FE00016600F0BBB9B8
:107A0400F8B50446406841F63121C0F21E1188429F
:107A140007D34DF28900C0F6000040F6DD3103F0D3
:107A2400C5FBA068002818BFB0F5805F40F0BB809C
:107A3400206848F20007C4F20007B842E06814D096
:107A44004FEA3030042807D34DF28900C0F6000015
:107A540040F6E53103F0AAFB206A40F40060B0F57B
:107A6400006F0FD040F6E63106E040F40050B0F568
:107A7400005F07D040F6E1314DF28900C0F6000006
:107A840003F094FB2069002818BFB0F5806F40F024
:107A94009780606910B130F00C0007D04DF2890076
:107AA400C0F6000040F6EA3103F080FBA0694FEA1B
:107AB4003020042807D34DF28900C0F6000040F6B8
:107AC400EB3103F073FBE06940F40040B0F5004F84
:107AD40007D04DF28900C0F6000040F6EC3103F007
:107AE40065FB606A0C2807D34DF28900C0F60000DC
:107AF40040F6ED3103F05AFB206804F108012EC969
:107B0400194341EA0503E169056846F6F316CCF624
:107B1400FF762E4033430B430360436823F4405302
:107B24001A434260A269B8421CBF236A1A4383689D
:107B340023F06E4323F430631A438260C36A626A9B
:107B440023F00F031343C36244F6FF73C4F200032C
:107B540098424FF0100312DCA7F57056B0423CD0A7
:107B640006F58066B04246D006F58066B04257D12D
:107B740041F28803C4F202031B689B0948E0A7F59D
:107B84004056B04230D0B8423CD006F56846B042C8
:107B940046D141F28803C4F2020342F2B8351B68AD
:107BA400C0F6000538E0B0F1805F3FF441AF4DF21C
:107BB4008900C0F6000040F6DE3103F0F7FA37E73B
:107BC400B0F5C06F3FF465AF4DF28900C0F6000018
:107BD40040F6E93103F0EAFA5BE741F28803C4F2C4
:107BE40002031B689B0813E041F28803C4F20203FA
:107BF4001B681B0A0CE041F28803C4F202031B68F1
:107C04001B0905E041F28803C4F202031B689B0AC6
:107C140042F2C835C0F6000503F0030355F82330DB
:107C2400B84242F20040C0F2F40011D0B1F5004F66
:107C34004FF001011AD1082B00F29580DFE803F020
:107C440005293B932F939393390001F091FF28E08A
:107C54000121082B00F28780DFE803F005856285A7
:107C640015858585600001F083FF0EE0082B00F286
:107C74007A80DFE803F005113C78197878783A00C7
:107C840001F076FF12E001F03CFF002844D0626A64
:107C940046E001F082FF04E001F07FFF06E001F01E
:107CA40030FFC8B3626A06E001F02BFFA0B3626A3A
:107CB4001DE04FF400404CF20C21C0F6000131F8F5
:107CC40012106268B0FBF1F0510801EB4000B0FB08
:107CD400F2F0A0F110014FF6EF72914242D8511C1C
:107CE4000140C0F34200084414E04FF400404CF259
:107CF4000C21C0F6000131F81210B0FBF1F06168FC
:107D040000EB5100B0FBF1F0A0F110014FF6EF725F
:107D1400914227D82168C860002124E04FF4004034
:107D24004CF20C21C0F6000131F812106268B0FB6D
:107D3400F1F002EB42018842012114D3B0EB023F7F
:107D440011D8010E000210EB520041F10001002392
:107D540001F0FAF9A0F540714FF60052C0F20F029B
:107D64009142D7D301214FF00110A0660022C4E94B
:067D74001D220846F8BDC7
:027D7A00704750
:107D7C002DE9F84F804600689146C2690E461140C5
:107D8C00891BB1FA81F1B9EB511F27D19A46A6F1A3
:107D9C00400131F0400B0A9D18BF4FF0010B6F1CD6
:107DAC00032400BF97B103F07DFBC5B1A0EB0A0023
:107DBC00A84214D8D8F8000001681BEA910105D03C
:107DCC00C16909070ED4C16909050FD4C1693140D5
:107DDC00891BB1FA81F1B9EB511FE3D00024204685
:107DEC00BDE8F88F01240821894604E003244FF0F4
:107DFC0020094FF400610162404600F039F9C8F8DF
:0A7E0C009090002088F88400E9E758
:027E16007047B3
:107E18000168806A0968890619D40021A0F85610FB
:107E28000168083151E8001F026821F0800108321A
:107E380042E80013002BF3D1016851E8001F0268E3
:107E480041F0400142E80013002BF5D1704702F0E1
:027E58006DBB00
:107E5A002DE9F0419CB004460068154640F4806064
:107E6A0040F20047C5F20007B8420E4607D04DF669
:107E7A00E610C0F6000040F2653103F094F9607F25
:107E8A00022807D34DF6E610C0F6000040F266312C
:107E9A0003F089F9206B4FEAB020042807D34DF686
:107EAA00E610C0F6000040F2673103F07CF994F85E
:107EBA003800022807D34DF6E610C0F600004FF44A
:107ECA005A7103F070F920688168490703D494F85D
:107EDA005810012903D102201CB0BDE8F08101210C
:107EEA0084F85810002118911991B0F1A04FA7F504
:107EFA00407804D0B84210D108F5806000E04046CE
:107F0A0001902046FDF763FA18B901A8FDF75FFA58
:107F1A0058B1002184F85810DEE7E06D40F02000E7
:107F2A00E06584F858100120D6E72268606DE16D9B
:107F3A0008F5037340F60177B94301F58071E165ED
:107F4A00002121664BF2CD47C0F60007C76247F60B
:107F5A003F17C0F60007076347F6EF17C0F600079A
:107F6A0047631C274245176084F8581019461CBFFE
:107F7A0040F20C71C5F20001B2F1A04F576808BF78
:107F8A00194647F01003536032462B4603F0DDFBD7
:107F9A0021688A6822F0004222F03F0204328A6095
:027FAA009AE754
:107FAC00D0F88C30202B23D10123002918BF002AB4
:107FBC001FD00023C366D0F800C048F20003C4F2FF
:107FCC0000039C4512D000B5DCF804301B020BD525
:107FDC00036853E800CFD0F800E04CF080634EE823
:107FEC00003CBCF1000FF3D15DF804EBFAF76EB96D
:067FFC0002231846704745
:1080020070B515460E46102A044606D34DF6472093
:10801200C0F60000BE2103F0CAF8102E06D34DF6BA
:108022004720C0F60000BF2103F0C1F84EF60C5005
:10803200CEF200004FF0FF330168C1F3022181F05C
:108042000702042A28BF0422033938BF002103FA99
:1080520002F226EA02028B4002FA01F125EA030249
:1080620011430901002C03D4A0F60C10215470BD59
:0A80720004F00F021044017270BD0B
:10807C00016851E8001F026821F4907142E8001376
:10808C00002BF5D14FF6FE7CCEF6FF7C0268083251
:10809C0052E8002F036802EA0C02083343E800217F
:1080AC000029F3D1C16E01290AD100BF016851E842
:1080BC00001F026821F0100142E80013002BF5D1DB
:0E80CC002021C0F88C100021C166416770476A
:1080DA0000280DDB00F01F01012202FA01F11C2227
:1080EA0002EAD0004EF20012CEF20002815070472E
:0E80FA004DF64720C0F60000D22103F054B826
:1081080070B501680446CA6908688E6840F62F038E
:108118001340202B0BD100F0200306F080555B198B
:1081280016D0616F69B32046BDE87040084740F635
:108138000F031A420CD00123C1F2000306EA030C14
:1081480040F22013C0F20043034013EB0C0326D186
:10815800E36ED50616D5012B14D110F0100311D0FB
:10816800102008628868400600F1A380B4F85C001B
:10817800B4F85E10B4F85E20002A18BF884240F0B8
:10818800F88070BDD30272D516F480036FD04FF417
:10819800801220460A62BDE8704001F087BED3070E
:1081A80018BF10F4807307D001230B62D4F8903005
:1081B80043F00103C4F89030930706F0010E0AD586
:1081C800BEF1000F07D002230B62D4F8903043F0C1
:1081D8000403C4F8903053070AD5BEF1000F07D046
:1081E80004230B62D4F8903043F00203C4F89030B3
:1081F80013070CD500F0200353EA0C0307D008231B
:108208000B62D4F8903043F00803C4F8903013059B
:108218000BD510F0806308D04FF400630B62D4F8DC
:10822800903043F02003C4F89030D4F89030002BFD
:10823800A7D092060AD500F0200006F080528018D8
:1082480004D0626F12B1204690472168D4F890009C
:10825800896801F0400100F028004018204640F0ED
:10826800B98004F0C3F90020C4F8900070BD11066D
:1082780006D500F0800106F40003C91840F0CD804F
:1082880051066CD510F0400169D000BF206850E855
:10829800000F216820F0400041E80002002AF5D1D3
:1082A8002020C4F888002046A267BDE8704002F08C
:1082B8003DB9D4F8800000684268B4F85C3091B2E7
:1082C800002944D0994242D2A4F85E200068800672
:1082D80034D400BF206850E8000F216820F4807073
:1082E80041E80002002AF5D12068083050E8000F64
:1082F800216820F00100083141E80002002AF3D18A
:108308002068083050E8000F216820F0400008314C
:1083180041E80002002AF3D12020C4F88C00E2666C
:10832800206850E8000F216820F0100041E80002A2
:10833800002AF5D1D4F8800000F017FB022020674E
:10834800B4F85C00B4F85E10401A81B23DE08B428C
:108358007FF417AF006880067FF513AF33E0110292
:1083680062D510F080415FD02046BDE8704001F032
:108378009FBD401A216851E8001F226821F49071BE
:1083880042E80013002BF5D14FF6FE71CEF6FF71CF
:108398002268083252E8002F23680A40083343E86D
:1083A8000026002EF4D12021C4F88C10E6666667FA
:1083B800216851E8001F226821F0100142E80013EB
:1083C800002BF5D181B2022222672046BDE8704019
:1083D80001F05BBDFFF74EFE2068806840061ED5A1
:1083E8002068083050E8000F216820F0400008316C
:1083F80041E80002002AF3D1D4F8800078B14CF2A9
:108408008511C0F60001816303F0F8F900283FF4F4
:10841800B8AED4F88000816B86E6A16F82E620466C
:10842800BDE8704004F0E2B8D1017FF5AAAE00289B
:0E843800BFF6A7AE2046BDE8704001F038BD8B
:108446000138010E01D0012070474EF21001CEF224
:108456000001486001F61350F02202700020886087
:0684660007220A607047C6
:10846C000168806A0968890634D40021A0F85E107E
:10847C00016851E8001F026821F4807142E8001382
:10848C00002BF5D10168083151E8001F026821F07A
:10849C000101083242E80013002BF3D101680831C6
:1084AC0051E8001F026821F04001083242E8001335
:1084BC00002BF3D12021C0F88C10C16E012909D1F9
:1084CC00016851E8001F026821F0100142E8001316
:1084DC00002BF5D100210167C16E012903D1B0F841
:0A84EC005C1001F0D0BC01F0D0BC20
:1084F60010B5040027D0206843F20001C4F202013F
:10850600884206D04DF2C540C0F60000702102F048
:108516004CFE607F18B920772046FCF7CBF9022085
:1085260060772079022807D34DF2C540C0F60000D7
:108536007E2102F03AFE207938B1D4E902122046B3
:10854600FDF737FE58B1012010BD206841F6B7513E
:10855600C0F2C1414161816821F0180181606079F2
:10856600022807D34DF2C540C0F60000902102F064
:108576001CFE6079002814BF2269421E61692068CA
:108586004FEA7113042B026108D34DF2C540C0F6C1
:1085960000009C2102F009FE20686169826822F0D1
:1085A600600211438160A16941F08002802A08D0EF
:1085B6004DF2C540C0F60000A02102F0F6FD20688D
:1085C600A169826822F0800211438160206A013825
:1085D600032806D34DF2C540C0F60000A52102F0DF
:0A85E600E4FD01206077002010BDC5
:1085F0002DE9B04183B00C46804622258DF8055008
:108600004FF47A770DF105010DF105020323009770
:10861000F9F782FC9DF80700009700F0070020435F
:108620008DF8060042208DF8050040460DF1050149
:108630000DF105020223F9F76FFC8DF80550404655
:108640000DF105010DF1050203230097F9F764FC14
:108650009DF807002040A04202D103B0BDE8B081E0
:0E8660004DF27E10C0F6000002F0F7F9FEE7C2
:10866E0010B5040000F0B980206840F20741C4F252
:10867E0002018842D4BFA1F56C7150318842D4BF3B
:10868E00283928318842CCBF01312739884203D09E
:10869E001431884240F0D380A068002818BF1028FB
:1086AE0040F0A980E06840F04000402806D04DF22E
:1086BE002350C0F60000A52102F073FD206940F0A2
:1086CE008000802806D04DF22350C0F60000A6216F
:1086DE0002F067FD6069002818BFB0F5807F40F09A
:1086EE009680A069002818BFB0F5806F40F09B807F
:1086FE00E06940F02000202806D04DF22350C0F64D
:10870E000000A92102F04DFD206A4FEA3030042806
:10871E0006D34DF22350C0F60000AA2102F041FD0F
:10872E006068742806D34DF22350C0F60000AC21C9
:10873E0002F037FD40F20041C4F20201206801F15F
:10874E00080290424FF6F832CBF6FD723CBF02F5AE
:10875E008062A1F5806102444CF6CD43CCF6CC4349
:10876E00A2FB03236FF0030202EA930204F1080353
:10877E0093E80850C4E91012022184F8251001680C
:10878E006FF30E11194341EA0C0141EA0E01D4E9CF
:10879E00052311431943D4E90723114319430160FB
:1087AE00204600F085F8A068B0F5804F06BF002087
:1087BE0060606068411E032904F148010EC9C0B211
:1087CE00086053600BD8204602F08BFF04F1540072
:1087DE0007C8002303604A6005E0012010BD002099
:1087EE00C4E91500E0650020E063012184F825103E
:1087FE0084F8240010BDB0F5804F3FF453AF4DF216
:10880E002350C0F60000A42102F0CBFC4AE7B0F5DD
:10881E00007F3FF466AF4DF22350C0F60000A72153
:10882E0002F0BFFC5DE7B0F5006F3FF461AF4DF2B3
:10883E002350C0F60000A82102F0B3FC58E74DF219
:0E884E002350C0F60000A32102F0ABFC24E78B
:10885C002DE9F04F83B01D469246064658188709FD
:10886C0000204FF47A7941F2F018C1F2000800BFF1
:10887C0041EA861211FA85F3402B2C4628BFC1F130
:10888C0040041FFA80FB1AFA80F00090A0B2CDE9E8
:10889C00010992B24046A021022303F083F801366D
:1088AC002D1B1BFA84F00021013FE1D203B0BDE87F
:0288BC00F08F3B
:1088BE0000B5016801F0FC02083A4CF6CD43CCF647
:1088CE00CC43A2FB032C40F6000EC4F2020EAEF512
:1088DE007E73426C994222F003010EF1200238BFE2
:1088EE007246114481640EF18001C164CCF304110F
:0A88FE00012202FA01F1016500BD3C
:108908002DE9F04F83B01F469246834658188609D2
:10891800002541F2F018C1F2000800BF41EA8B10AF
:1089280011FA87F2402A3C4628BFC1F140041FFAD9
:1089380085F91AFA85F10091A1B2019182B24046F7
:10894800A02102234FF47A75029500F078FF0BF10D
:10895800010B3F1B19FA84F50520F8F759FB002194
:0A896800013EDBD203B0BDE8F08F42
:10897200014690F82500022827D100B50868D1E900
:1089820010CE8A6C036823F00E030360136823F48D
:1089920080731360026822F0010202600EF01F0071
:1089A200012202FA00F0CCF80400D1E91320506051
:1089B200486D38B1026822F480720260D1E9160271
:1089C200426000205DF804EB02E00420C86301204D
:0E89D200012281F82520002281F82420704720
:1089E00041F20800C4F202000168C1F3810241F2C1
:1089F0008071C1F20001DFE802F0022B04090A686D
:108A00002BE043F20062C0F26E1225E04268436838
:108A100002F00302C3F3031303F1010C022A43F231
:108A20000062C0F26E1204BF42F20042C0F2F402D1
:108A30004368B2FBFCFCC3F30623426803FB0CFC57
:108A4000C2F34162022303EB4202BCFBF2F203E0F9
:108A500042F20042C0F2F4020A600068C0F3031060
:108A60004EF22413C0F60003185C22FA00F00860EE
:028A700070474D
:108A720042F20C00C4F202008168490001D40020D5
:108A8200704742F63B21C0F61901016001F1443101
:0A8A920001608068C0F38070704737
:108A9C0030B591EA030F00F18280841A71EB030C5C
:108AAC0005D2121953EB0C03001B71EB0C0140F2B5
:108ABC00000CCFF6E07C1CEA430F52D0BCEB410F0C
:108ACC005FD90C0DA4EB135E5FF0010C6CF31F511E
:108ADC006CF31F53DEF1200C2AD303FA0CF540196A
:108AEC0041F1000122FA0EF5401923FA0EF5694105
:108AFC0012FA0CF2CD0208D349085FEA30005FEAA3
:108B0C00320228BF42F00102641C641E5FEA500C62
:108B1C0072F1004250F1000051EB04514FF400137C
:108B2C0013EB410F38BF30BD6FF31301002030BD84
:108B3C00BEF1200EBEF1200F1ED223FA0EF5401905
:108B4C0041F10001CEF1200C124218BF012203FAB0
:108B5C000CF52A43CEE711EA5C0F04BF002000217C
:108B6C0030BD1CEA410F04BF01F00041002030BDB4
:108B7C0001F00041002030BD21F4801101EB0451C3
:108B8C0030BD004218BF41F00101BCEB410F08BFE2
:108B9C0030BD4FF0FE4141F47801002030BD83F030
:108BAC000043841A71EB030E07D28EF0004E001BAB
:108BBC0071EB0E01121953EB0E0340F2000CCFF6C1
:108BCC00E07C1CEA430FC6D0BCEB410F72D90C0DF4
:108BDC00A4EB135EC90241EA5051C00241F00041BE
:108BEC00DB0243EA5253D20243F00043DEF1200C85
:108BFC0041D312FA0CF522FA0EF203FA0CF542EA02
:108C0C00050218BF42F0010223FA0EF3801A9941B3
:108C1C00E30AC4F30A0411F0404F03D418D0641EC5
:108C2C0040004941641E23D44205C00A40EA415029
:108C3C00C90A51EAC3715FEA500C72F1004250F15B
:108C4C00000051EB045130BD01002FD00020203C1E
:108C5C000029F9D0B1FA81FCDCF1200E11FA0CF1EB
:108C6C0030FA0EF510FA0CF02943A4EB0C04D9E7FA
:108C7C000020D90730BDAEF1200EBEF1200F0DD271
:108C8C00CEF1200C03FA0CF533FA0EF32A4318BF7D
:108C9C0043F00103C01A61F10001B9E721F0004172
:108CAC00C00A40EA4150C90A01EB045130BD002012
:108CBC00002130BD004218BF41F00101BCEB410F57
:0E8CCC007FF467AFBCEB430F3FF463AF30BDE6
:108CDA0042F21400C4F20200016841F080410160CE
:0E8CEA00006800F08040012181EA9070704720
:108CF8002DE9F04391EA030E0EF0004E40F2000712
:108D0800CFF6E07717EA41051EBFBD4217EA4305D3
:108D1800BD4200F09F807F0D17EA135623EA4753A0
:108D280043F4801317EA115521EA475141F48011A1
:108D3800AD1B05F2FD354FEAD31C1CF1010C4FF0B9
:108D48000047B7FBFCF77F01A2FB079C0024E3FB6D
:108D580007C4D9F100096CEB4C0CA0FB076200209A
:108D6800E1FB072000275FEAC628E0FB0987760DAC
:108D780046EAC226520DF61900277A41E0FB0C623A
:108D88005FEAC823E2FB09375FEA585848EAC62871
:108D9800760D18EB070800214E41E2FB0C8602EB2A
:108DA800C020DA02E6FB09215B0D43EAC8235FEA2B
:108DB80058585B18002758EB0708E6FB0C38D10217
:108DC800E8FB0917520D42EAC3225B0DD2190027AE
:108DD8007B41E8FB0C2308EBC6265FEAC128E3FBCE
:108DE8000987490D41EAC221520DC91942F1000211
:108DF800E3FB0C12470019EB08095CEB010C72EB62
:108E0800040453EBC62047EB56530026B3F5000F76
:108E18007641AD19B61CD6F1200910FA09F4F040D4
:108E280013FA09F21043F340E40F001943F1000369
:108E3800B3F5001F24BF5B086D1C40F2FE77BD42EE
:108E480004D24EEA05511944BDE8F0832D4224D5D9
:108E5800714626E0004218BF41F00101124218BFD6
:108E680043F00103B7EB410F2CBFB7EB430F1BE0F7
:108E7800B7EB410F04BFB7EB430F15E017EA410FFB
:108E880004BF17EA430F0FE017EA410FE0D017EAD3
:108E9800430F02D0B7EB430FDAD04EF0FE4141F456
:108EA80070010020BDE8F08340F20001C7F6F871B8
:028EB800F7E7DA
:108EBA0038B50C00054607D14CF6CB70C0F6000059
:108ECA004FF4BD7102F06FF92869204018BF0120E4
:028EDA0038BDA1
:108EDC00C1F30A5340F21E42D21A0EDD202A0AD8E0
:108EEC00CB0243EA505040F00040D04090EAE17091
:108EFC00B0EBE1707047002070474B00004218BF88
:108F0C0043F0010313F5001F88BF21F0004111F05D
:0A8F1C00004058BF6FF0004070479E
:108F260038B50C00054607D14CF6CB70C0F60000EC
:108F360040F2B31102F039F9686900EA040124EA43
:0A8F4600000040EA0140A86138BDB8
:108F500010F0004160B148BF40420A0D02F21D42CC
:108F6000B0FA80F3D21A9840C30A400503EB0251CD
:028F7000704748
:108F720040F21441C4F201010A68024214BF0860BF
:068F8200704702F0EEB999
:108F880070B5CC1760406140001BA141DD176A40F5
:108F98006B40521BAB4100F0D5F862406340121B96
:0E8FA800A3416C4060406140001BA14170BDC0
:108FB60010B504000FD0206847F2FF71C4F200011B
:108FC600884214DC45F20041C4F2000188421DD0FB
:108FD60001F5806110E0012010BD4CF40441022A25
:108FE600816040F08A80416841F4006188E0013187
:108FF60088420BD001F54061884207D04DF281507E
:10900600C0F600004FF4087102F0CFF8A068B0F582
:10901600806F07D34DF28150C0F6000040F2212147
:1090260002F0C3F8E0680138022807D34DF28150F8
:10903600C0F6000040F2222102F0B7F8206940F4A1
:109046000040B0F5004F07D04DF28150C0F6000049
:1090560040F2232102F0A9F86069FF2807D94DF2F2
:109066008150C0F600004FF4097102F09EF8A06925
:10907600082807D34DF28150C0F6000040F22521A2
:1090860002F093F8E06940F40020B0F5002F07D015
:109096004DF28150C0F6000040F2262102F085F81C
:1090A600206A40F40030B0F5003F07D04DF2815001
:1090B600C0F6000040F2272102F077F894F841004C
:1090C60020B984F84000204601F08FFF242084F860
:1090D600410094E80910E268016821F0010101608D
:1090E60023F070610161816821F40041012A8160E9
:1090F6007FF473AF4CF400418160416821F4006154
:109106004160416841F0007141F400414160C1682D
:1091160021F40041C16004F110010EC9114341EA76
:109126000321E269C160216A11430160016841F0CF
:109136000101016000206064202184F84110206351
:0691460084F8420010BD98
:10914C00002B35D129B9B0FBF2FC0CFB12026046A6
:10915C007047914215D22DE9F041B2FA82F39A4050
:10916C009940D3F1200C30FA0CFC51EA0C019840D8
:10917C0000F04EF8280036FA03F200210023BDE877
:10918C00F081F0B5B1FBF2FC0CFB1211B2FA82F3D8
:10919C009A409940D3F1200630FA06F631439840B4
:1091AC0000F036F8614628003200DA400023F0BDAA
:1091BC00F3B5B3FA83FC49085FEA300013FA0CF3F9
:1091CC00DCF1200432FA04F423430CB41A0000F04E
:1091DC001FF80CBC33FA0CF3DCF11F0C35FA0CF550
:1091EC0018BF6D1E03BCA5FB026705FB0377801B34
:1091FC00B941904271EB030C05D3821A71EB030356
:10920C00681C0021F0BD02000B0028000021F0BDFD
:10921C00940D4FF6C2752D02B5FBF4F4D60A761CEC
:10922C0004FB04F5A5FB0656F64306EB041655089D
:10923C0032BF002777086D1C05FB1677A6FB074786
:10924C007F0807EBC63714001500E7FB02457F1BB0
:10925C004D1C0400E7FB014505FB1206A64284BF2A
:0E926C006D1EB618964224BF6D1CB61A7047D0
:10927A002DE9F0411D4690460446006847F2FF7208
:10928A00C4F2000290420F4608DC45F20041C4F2E3
:10929A000001884211D001F5806104E0511C884226
:1092AA000BD001F54061884207D04DF28150C0F6DB
:1092BA00000041F6714101F076FF069E002D18BFAD
:1092CA00B5F1807F33D143F6FF70C8F200008642C1
:1092DA000ADC42F20000C8F20000864210D000F513
:1092EA008060864204D10BE00130864208D03EB14C
:1092FA004DF28150C0F6000041F6734101F053FF70
:10930A006FF39F2747EA084028433043216820F03B
:10931A0000404A684FF4806303EA565383F07C4363
:10932A0083F41C431A4010434860BDE8F081B5F14C
:10933A00007FC8D04DF28150C0F6000041F672415C
:06934A0001F031FFBFE756
:109350002DE9F04F89B01546894682460020CAF8AB
:1093600000000DF10E0819F8011B252906D000296F
:1093700000F04F82504603F00FFCF4E72C46002724
:109380004A4619F8010BA0F12003102B0DD88021BB
:10939000DFE803F0091B1B191B1B1B151B1B3018D7
:1093A0001B101B1B120040210DE05E280DD14FF455
:1093B000805108E0102106E04FF4007103E04FF403
:1093C000004100E020210F43DAE7A0F13001C9B2EB
:1093D00009294FF000010BD801EB810100EB41019D
:1093E00019F8010BA0F13002D2B230390A2AF3D3B6
:1093F00025460CE0254655F8040B010048BF4142C4
:10940000102303EAD060074302F1020950782E28A6
:109410000BD14A4612F8010B2A2809D155F804BB92
:1094200099F8010009F1020218E04FF0000B1EE06C
:10943000A0F13003DBB2092B4FF0000B14D80BEB7B
:109440008B0300EB430312F8010BA0F130095FFA24
:1094500089F9B9F10A0FA3F1300BF0D3BBF1000F7A
:1094600004D447F4807701E047F480779146A0F177
:109470006802D3B2D20142EA5302D2B2092A22D8F8
:10948000DFE802F0050E122121210F21210F4A46AB
:1094900012F8010B682812D199F8010008370BE087
:1094A000023719F8010B0EE04A4612F8010B6C283E
:1094B00007D199F80100023709F1020903E00437E6
:1094C00000E001379146622821EAE17620DDA0F133
:1094D000630115293FF647AFDFE811F038001700A8
:1094E00016001600160016001700160016001600CB
:1094F00016009A0044000601160016002900160006
:109500004E001600160022002DE747F4804737E092
:10951000252800F08A80582840F08C8147F40057B5
:1095200043F2580278281ED143F278021BE00195DD
:109530002D68002D04BF4DF22B35C0F60005F8054F
:10954000284600F1458103F079FC44E12C78013E86
:1095500050463946324603F071FB5046214603F02F
:109560001BFB4AE13022390602EAE1710291F9055A
:1095700008D527F4007705E0F90548BF27F4007700
:109580000021029179044FEA8771009604D40029E2
:1095900009D4291D00240CE0002913D4294651F8D0
:1095A000045BEC1714E0E91D21F0070505F1080143
:1095B0006C687A072D6814D417F0080F13D00024B4
:1095C000EDB210E0E91D21F007014C6851F8085B8D
:1095D0000191790709D439070AD545F3C0146DB252
:1095E00006E0ADB20024019126E045F3C0342DB26F
:1095F000002C07DBB9061DD47906029A48BF202249
:10960000029219E000216D4261EB04042D2112E069
:1096100055F8040B3907DAF8001000F1F880BA07A2
:1096200052BF0160002206C09DE65046252103F08E
:10963000B3FA98E62B210291F90548BF27F4007789
:10964000F90558BF4FF0010B00266E2821DD6F3859
:10965000092800F27980DFE800F005567777777700
:109660002277775655EA04006ED0E80840EA447045
:10967000062262F3DF0508F80650013650EAD401ED
:109680004FEAD4044FEAD001054641EA4470F0D1D4
:109690005AE0582837D0642818BF692854D155EAB1
:1096A000040051D0380407D506F00300032802BF98
:1096B0002C2008F806000136284621460A220023FD
:1096C000FFF744FD00EB8002A5EB4202D5F1090350
:1096D0000023A34142F0300208F8062006F10106FB
:1096E00005460C46DED32FE02846009650F8045B72
:1096F00001903806232101EAE070029047F4807758
:1097000000244FF0080B002655EA04001CD04EF24E
:109710003C10C0F60000B9045CBF4EF24C10C0F61D
:109720000000290941EA047105F00F020D46825C30
:1097300008F80620013651EA14114FEA14144FEAD2
:10974000151141EA0471EFD1ABEB060020EAE07B92
:1097500006EB0B000099029D0C1A4FF0FF30FF2D15
:1097600088BF0138002D18BF0444B80505D4504601
:109770003946224603F062FA0024FF2D04D9290A53
:10978000504603F009FA00E01DB15046294603F0A7
:1097900003FA50463946224603F050FA504630212B
:1097A0005A4603F03BFA012E08DB751E504618F8A6
:1097B000051003F0F1F9012E2E46F6D8F806019DAA
:1097C0007FF5D1AD50462021224603F027FACAE5A5
:1097D000594603F049FB044627F40077361A5046F1
:1097E0003946324603F02AFA34B115F8011B5046C7
:1097F00003F0D2F9013CF8D1019D0435F8067FF55C
:10980000B2AD50462021324603F008FAABE50170B4
:10981000A9E5DAF80C0028B1DAE9001291423CBF60
:1098200000224254504601F0B9F9DAF8000009B0BC
:10983000BDE8F08F00287FF496AD504601F0AEF9F8
:069840004FF0FF30F3E7DA
:109846002DE9F84F1E4693468A46591E89B20229CB
:10985600044607D34DF28150C0F6000040F6E111F0
:1098660001F0A3FC94F8410020280AD10A9F57B1C1
:10987600DDF82C80B8F1000F05D094F840000128DF
:1098860006D1022514E04FF40070606401250FE054
:10989600012584F8405001F008FE814620464FF429
:1098A600004101221923CDF80090FDF7FEF910B111
:1098B6002846BDE8F88F0C99212084F84100402005
:1098C60084F84200002565646762A4F82A80884609
:1098D600656342F20007C8F20007F2B2204651461D
:1098E6004FF080730097FFF7C5FC204641464A4675
:1098F600F7F7F7FDC0B9012E206809D04FEA1B2102
:109906008162204641464A46F7F7EBFD60B920687A
:109916005FFA8BF181622046802100224346CDF812
:109926000090FDF7C2F910B184F84050AEE7608DA3
:10993600FF2804D9FF20FF224FF0807303E0608DDB
:10994600C2B24FF000732085204651460095FFF7BE
:1099560091FCFF26204641464A46F7F7C2FD0028FD
:1099660094D1606A216810F8012B8A626062608D6A
:1099760001386085208D01382085618DF1B10004A4
:109986001CD12046802100224346CDF80090FDF7E9
:109996008CF900287FF47AAF608DFF2804D92685DC
:1099A600FF224FF0807304E0608D2085C2B24FF035
:1099B6000073204651460095FFF75CFC608D002839
:1099C600C8D1204641464A46FDF775FA00287FF47D
:1099D6005DAF20682021C16142684EF60003CFF6D4
:1099E60000631A40426084F84110002584F8425012
:0699F60084F840505CE71C
:1099FC004AB1884207D007D28018891852428B5C32
:109A0C008354521CFBD17047521E8B5C8354FBD188
:029A1C00704791
:109A1E0038B50446006847F2FF72C4F20002904265
:109A2E000D4608DC45F20041C4F20001884210D018
:109A3E0001F5806104E0511C88420AD001F54061B5
:109A4E00884206D04DF60930C0F60000912101F093
:109A5E00A8FB102D06D34DF60930C0F6000092215A
:109A6E0001F09FFB94F84100202803D194F84000A8
:109A7E00012801D1022038BD242084F8410020683D
:109A8E00016821F001010160016821F4706141EA71
:109A9E0005210160016841F001010160202084F878
:0A9AAE004100002084F8400038BD9C
:109AB80001680122C0F8D022002280F8C822B1F83B
:109AC800540040F00100A1F85400B1F8540040F0EF
:0A9AD80002020020A1F8542070479C
:109AE20047F20000C4F20000016841F48071016095
:029AF2007047BB
:109AF40047F20800C4F20000016841F480410160AB
:029B04007047A8
:109B060041F20801C4F2020142F200420868C0F2C2
:109B1600F40200F00C000428104625D0086800F076
:109B26000C00082847F64000C0F27D101CD00B68D8
:109B360003F00C030C2B18D14B6803F00303032B23
:109B46004B6808BF0246C3F303100130B2FBF0F0C6
:109B56004A684968C2F306225043C1F341610222B2
:0E9B660002EB4101B0FBF1F0704700207047A8
:109B740041F28070C1F2000041F20801C4F2020116
:109B840000680968C1F302214EF23412C0F60002E3
:0A9B9400515C01F01F01C84070474A
:109B9E0041F28070C1F2000041F20801C4F20201EC
:109BAE0000680968C1F3C2214EF23412C0F60002F9
:0A9BBE00515C01F01F01C840704720
:109BC80010B50C46202907D34DF62C40C0F60000EE
:109BD80040F2FC7101F0E8FA42F20050C4F20000D1
:069BE80050F8240010BD3E
:109BEE0070B515460E4604464FF4C05132462B460C
:109BFE00FDF72FFE68B9204631462A46FDF79BFE3B
:109C0E0038B920464FF4C06132462B46FDF721FE8F
:0E9C1E0020B1206E40F020002066032070BDB3
:109C2C0010B50446806AFF2808D94DF28900C0F6A9
:109C3C00000040F6AE4101F0B5FAA06A010715D557
:109C4C00A16B41F40040B0F5004F08D04DF28900F3
:109C5C00C0F6000040F6B34101F0A4FAA16B2268F3
:109C6C00A06A536823F4004319435160C10715D00F
:109C7C00E16A41F40030B0F5003F08D04DF28900A4
:109C8C00C0F6000040F6BA4101F08CFAE16A226895
:109C9C00A06A536823F4003319435160810715D52A
:109CAC00216B41F48030B0F5803F08D04DF2890033
:109CBC00C0F6000040F6C14101F074FA216B226835
:109CCC00A06A536823F4803319435160410715D5BA
:109CDC00616B41F48020B0F5802F08D04DF28900E3
:109CEC00C0F6000040F6C84101F05CFA616B2268D6
:109CFC00A06A536823F4802319435160C10615D51B
:109D0C00E16B41F48050B0F5805F08D04DF28900D2
:109D1C00C0F6000040F6CF4101F044FAE16B226836
:109D2C00A06A936823F4805319439160810615D57A
:109D3C00216C41F40050B0F5005F08D04DF2890061
:109D4C00C0F6000040F6D64101F02CFA216C2268D6
:109D5C00A06A936823F400531943916040064CD5D4
:109D6C00206844F6FF31C4F20001884209DD01315C
:109D7C00884216D001F58061884212D001F5684105
:109D8C0005E0A1F2FF7188420BD001F58061884299
:109D9C0007D04DF28900C0F6000040F6DD4101F01D
:109DAC0001FA616C41F48010B0F5801F08D04DF2BF
:109DBC008900C0F6000040F6DE4101F0F3F9616C59
:109DCC002068426822F480120A43B1F5801F426079
:109DDC0013D1A16C4FEA7152042A09D34DF28900B8
:109DEC00C0F6000040F6E34101F0DCF92068A16CFC
:109DFC00426822F4C0021143416094F82800000626
:109E0C0014D5E06C40F40021B1F5002F08D04DF2D0
:109E1C008900C0F6000040F6EB4101F0C3F9E06C9C
:0E9E2C0021684A6822F400221043486010BDED
:069E3A00806A00F02AB866
:109E400038B5846A2068D4F88810D4F88C508268B9
:109E5000120608D5212906D10020A4F85600204674
:109E6000F8F790FA20688068400607D5222D05D1C2
:109E70000020A4F85E002046FEF700F9D4F8900018
:109E800040F010012046C4F89010BDE8384002F0C0
:029E9000B1BB64
:029E9200704717
:029E9400704715
:029E9600704713
:029E9800704711
:109E9A00806A01210167C16E012904D1B0F85C1002
:0A9EAA004908FFF7F1BFFFF7F2BF10
:029EB4007047F5
:029EB6007047F3
:029EB8007047F1
:109EBA00416EF9B100B501684DF6BC7C8A688968C3
:109ECA00490FC0F6000CC2F342624DF6C47EC0F6DA
:109EDA00000E1CF801301EF80110DB00B3FBF1F193
:109EEA001CF802301EF802205DF804EBDB00B3FB1D
:109EFA00F2F201E001210122A0F86A10A0F868201C
:029F0A0070479E
:109F0C0010B50446006844F6FF71C4F200018842A3
:109F1C000ADCA1F6FF31884219D001F58061884234
:109F2C0015D001F5806108E0013188420FD001F5B0
:109F3C00405188420BD001F53841884207D04DF290
:109F4C005770C0F6000040F2362101F02BF994F85E
:109F5C008400012801D1022010BD2420C4F88800FF
:109F6C00216808680A6822F001020A6020F0005299
:109F7C00002060660A602021C4F8881084F88400F0
:029F8C0010BD06
:109F8E0070B50446006844F6FF72C4F200029042B7
:109F9E000D460ADCA2F6FF31884219D001F5806128
:109FAE00884215D001F5806108E0511C88420FD01F
:109FBE0001F5405188420BD001F53841884207D057
:109FCE004DF25770C0F6000040F2952101F0E9F80D
:109FDE004FEA7560062807D34DF25770C0F60000A1
:109FEE0040F2962101F0DDF894F88400012801D1A9
:109FFE00022070BD012084F884002420C4F888005B
:10A00E0020680668016821F001010160816821F075
:10A01E006061294381602046FFF748FF2068066093
:0EA02E002020C4F88800002084F8840070BD53
:10A03C0001460120A1F840000022A1F84020A1F81F
:0AA04C0044200020A1F850207047C6
:10A056000246D0F888019067B2F8CE00A2F87C00DC
:10A06600B2F8CC00A2F87E00D2F8D430C2F8803024
:0EA0760040F20000C1F20000002100F067B9C6
:10A084000246D0F8D400C2F88400D2F88400D2F892
:10A094008010401A41F2DC21C1F200014FF47A73BE
:10A0A4000968594391FBF0F340F20000C1F200004B
:0AA0B4000021C2F8883000F04AB91C
:10A0BE0040F20000C1F200004FF2F012C16DCFF677
:10A0CE00FF725143CB17C0E95813C16D4942C0F816
:10A0DE004011C16D5143CA17C0E97812C16D494292
:06A0EE00C0F8D811704714
:10A0F40010B582B040F25A04C1F200042088A4F8DA
:10A104002601B4F97200B4F91010884219DAB4F8CF
:10A1140072C0B4F97200B4F912108842D8BFB4F80E
:10A1240012C0B4F91200B4F91410B4F91020B4F93F
:10A1340000300FFA8CFCCDF800C002F02BF9A4F823
:06A14400260102B010BD6F
:10A14A0038B504464DF63050C0F6000000F080FCE9
:10A15A0040F2F835C1F2000505F1180040F2D811B5
:10A16A00C0F60001B822FAF739F8A8680130D02100
:10A17A00C5E9011001202870002000212A46D023B9
:0EA18A00FEF7BDFB2046BDE8384000F000B8EF
:10A19800F8B5054640F2F834C1F200040020002169
:10A1A8002246D023FEF756FBA0692861A08BA8821F
:10A1B800E08BE882208C2883608CA883A08CE883BD
:10A1C800E08C2884208D6884608DA5F87C00A08DA3
:10A1D800A5F87E00E08DA5F89800208EA5F89A00D5
:10A1E800608EA5F88C00A08EA5F8A000E08EA5F8DA
:10A1F800A80004F1380090E80F50D4E91467C5F8B6
:10A208008000C5F88410C5F88820C5F89030C5F8D6
:10A218009CC0C5F8A4E0C5F8AC60AF6704F158006D
:10A2280007C8C5F89400C5F8B010C5F8B420B4F84C
:10A238008800A5F85200B4F88A00A5F85000D4F8B0
:10A248008C00E865D4F890002866B4F89400A5F866
:10A258005400B4F89600A5F85600B4F89800A5F88C
:10A268005800B4F89A00A5F85A00B4F89C00A5F86C
:10A278006400B4F89E00A5F86800B4F8A000A886A9
:10A28800B4F8A200E886B4F8A4002887B4F8A600B9
:10A298006887B4F8A800A887B4F8AA00E887B4F8D3
:10A2A800AC00A5F84000B4F8AE00A5F84200B4F838
:10A2B800B000A5F84400B4F8B200A5F84600B4F818
:10A2C800B400A5F84800B4F8B600A5F84A00B4F8F8
:10A2D800B800A5F84C00B4F8BA00A5F84E00B4F8D8
:10A2E800BC00A5F86A00B4F8BE00A5F86C00B4F884
:10A2F800C000A5F86E00B4F8C200A5F87000B4F864
:10A30800C400A5F87200B4F8C600A5F8B800B4F8FF
:10A31800C800A5F8BA00B4F8CA00A5F8BC00B4F89B
:10A32800CC00A5F8BE00B4F8CE00A5F8C000E068DF
:10A338006860A088E188227880F0D000084382F025
:0AA348000101084318BF0120F8BD11
:10A352002DE9F041884604464DF64550C0F600000E
:10A3620000F07AFB40F2F836C1F200062069B061D3
:10A37200A08AB083E08AF083208B3084A08B708423
:10A38200E08BB084208CF084608C3085B4F87E0041
:10A39200B085B4F87C007085B4F89800F085B4F804
:10A3A2009A003086B4F88C007086B4F8A000B086AB
:10A3B200B4F8A800F086D4F88000D4F88410D4F859
:10A3C2008820D4F89030D4F89C50D4F8A470D4F8F3
:10A3D200ACC0D4F878E0C6E90E01C6E91023C6E99C
:10A3E2001257C6E914CED4F89400D4F8B010D4F8B9
:10A3F200B42006F1580307C3B4F85200A6F8880047
:10A40200B4F85000A6F88A00E06DC6F88C00206E01
:10A41200C6F89000B4F85400A6F89400B4F85600B8
:10A42200A6F89600B4F85800A6F89800B4F85A00B6
:10A43200A6F89A00B4F86400A6F89C00B4F8680084
:10A44200A6F89E00A08EA6F8A000E08EA6F8A200B4
:10A45200208FA6F8A400608FA6F8A600A08FA6F809
:10A46200A800E08FA6F8AA00B4F84000A6F8AC0055
:10A47200B4F84200A6F8AE00B4F84400A6F8B00062
:10A48200B4F84600A6F8B200B4F84800A6F8B40042
:10A49200B4F84A00A6F8B600B4F84C00A6F8B80022
:10A4A200B4F84E00A6F8BA00B4F86A00A6F8BC00E8
:10A4B200B4F86C00A6F8BE00B4F86E00A6F8C000AE
:10A4C200B4F87000A6F8C200B4F87200A6F8C4008E
:10A4D200B4F8B800A6F8C600B4F8BA00A6F8C800E6
:10A4E200B4F8BC00A6F8CA00B4F8BE00A6F8CC00C6
:10A4F200B4F8C000B168A6F8CE00481CD021C6E965
:10A5020001100120B8F1000F307007D04EF2780030
:10A51200C0F6000000F0A0FA6068F0603246002049
:10A522000021D023FEF7EFF92046BDE8F041FFF706
:02A5320032BE37
:0EA5340040F22600C2F20000002101707047C4
:10A5420038B50C460546F9F772FA0146A01C2953A4
:02A5520038BD12
:10A5540038B5044610F8275FD0F8011205290DD349
:10A5640002F0B4F8013009D035B140F20000C1F274
:10A574000000008BA84201D1022038BD0020C4F89D
:06A584002802207538BD1D
:10A58A0070B5044600260146C0F82C6211F8273F30
:10A59A0080F8273100F227152846012200F00DF82D
:10A5AA0001462846FFF7C8FFC4F82C02204602F0ED
:0AA5BA007EF8C4F82862267570BD13
:10A5C40091F801C0BCF1100F09D0BCF1060F04D002
:10A5D400BCF1030F05D1F9F743BA02F087B8F9F7D4
:10A5E40081BA8CF08001815481180123901C4B7036
:02A5F4007047AE
:10A5F60040F20410C1F200004FF0FF3141800180AB
:02A6060070479B
:10A6080070B540F2D804C1F2000441F2303534F894
:10A61800640CC1F2000528B134F8640C012817D184
:10A62800012218E0288800284FF6FF7018BFE0853F
:10A63800E18D11B1E18D814256D1206834F8A41C16
:10A64800884214DA01264DF6AE50C0F600003FE00D
:10A6580034F8640C002240F20040C4F600004FF4C5
:10A66800006101F075F934F8640C288070BDE06869
:10A6780034F99C1C4FF47A725143884205DA022659
:10A688004EF2B400C0F6000022E034F90A0C34F9A6
:10A69800901C884205DD03264DF64500C0F60000F3
:10A6A80016E034F90C0C34F9901C884205DD0426B8
:10A6B8004DF68D50C0F600000AE034F90A0C34F962
:10A6C8008C1C884247DA05264DF2C720C0F60000E8
:10A6D80000F0BFF9E68540F20040C4F600004FF4F0
:10A6E8000061002201F034F9E08D0028BBD0206819
:10A6F80034F8A21C8842B6DDE06834F99C1C4FF49B
:10A708007A7251438842AEDD34F90A0C34F98E1C52
:10A718008842A8DA34F90C0C34F98E1C8842A2DA83
:10A7280034F90A0C34F98A1C88429CDD34F90C0C83
:10A7380034F98A1C884296DDE08D022893D0E08D9A
:10A74800072890D04DF66700C0F6000000F081F9A8
:10A758000020E08564E734F90C0C34F98C1C88423D
:06A76800C2DA0626A4E798
:10A76E0070B540F2BC04C1F2000441F220352088DD
:10A77E00A0F10A062088A1690A308142C1F20005C3
:10A78E001BD9B4F8940041F26F71884215D828781D
:10A79E0098B94DF20D30C0F6000000F057F90120C7
:10A7AE002870A088B0FA80F0420940F60000C4F686
:10A7BE0000004FF4005101F0C8F8A069B04203D276
:10A7CE002878012808D070BDB4F8940041F2717158
:10A7DE00884217D32878A8B14EF20410C0F60000B4
:10A7EE0000F034F900202870A288002A18BF012238
:10A7FE0040F60000C4F600004FF40051BDE8704072
:06A80E0001F0A3B870BDCB
:10A8140038B540F2C004C1F2000441F22A30C1F25A
:10A824000000B4F90E10B0F90000A0F5FA708842E7
:10A834005ADBB4F90C10884256DB41F22830C1F2DD
:10A844000000B4F90E10B0F9000000F5FA70884267
:10A854004ADCB4F90C10884246DC41F22630C1F2DD
:10A864000000B4F90E10B0F90000A0F5FA708842A7
:10A874003ADBB4F90C10884236DB41F22230C1F2E3
:10A884000000B4F90E10B0F9000000F5FA70884227
:10A894002ADCB4F90C10884226DC41F22C30C1F2D7
:10A8A4000000616AB0F900204FF0FF334DF6F00567
:10A8B400CFF6FF754FF47A70C2FB00536A1A73EB3C
:10A8C400E17111DB616A41F21E33C1F200034FEA08
:10A8D400E17CB3F90030002542F21072C3FB00257D
:10A8E400881A7CEB05001CDA41F22435C1F200051C
:10A8F400287800B138BD4DF61160C0F6000000F0B4
:10A90400AAF8012028702088B0FA80F0420940F6A5
:10A914000000C4F600004FF40051BDE8384001F0D7
:10A9240019B841F22435C1F2000528780028E1D194
:10A934004DF6A500C0F6000000F08DF80020287048
:0AA944002288002AE3D00122E1E797
:10A94E0040F20000C1F200004FF46162016EA1FB03
:10A95E000212C0E95C120021C0E95A11C0F8481178
:06A96E00C0F82011704743
:02A97400FEE7FC
:02A97600FEE7FA
:02A97800FEE7F8
:02A97A00FEE7F6
:02A97C00FEE7F4
:02A97E00FEE7F2
:02A98000FEE7F0
:02A98200FEE7EE
:02A98400FEE7EC
:02A98600FEE7EA
:02A98800FEE7E8
:02A98A00FEE7E6
:02A98C00FEE7E4
:02A98E00FEE7E2
:02A99000FEE7E0
:02A99200FEE7DE
:02A99400FEE7DC
:02A99600FEE7DA
:02A99800FEE7D8
:02A99A00FEE7D6
:02A99C00FEE7D4
:02A99E00FEE7D2
:02A9A000FEE7D0
:02A9A200FEE7CE
:02A9A400FEE7CC
:02A9A600FEE7CA
:02A9A800FEE7C8
:02A9AA00FEE7C6
:02A9AC00FEE7C4
:02A9AE00FEE7C2
:02A9B000FEE7C0
:02A9B200FEE7BE
:02A9B400FEE7BC
:02A9B600FEE7BA
:02A9B800FEE7B8
:02A9BA00FEE7B6
:02A9BC00FEE7B4
:02A9BE00FEE7B2
:02A9C000FEE7B0
:02A9C200FEE7AE
:02A9C400FEE7AC
:02A9C600FEE7AA
:02A9C800FEE7A8
:02A9CA00FEE7A6
:02A9CC00FEE7A4
:02A9CE00FEE7A2
:02A9D000FEE7A0
:02A9D200FEE79E
:02A9D400FEE79C
:02A9D600FEE79A
:02A9D800FEE798
:02A9DA00FEE796
:02A9DC00FEE794
:02A9DE00FEE792
:02A9E000FEE790
:02A9E200FEE78E
:02A9E400FEE78C
:02A9E600FEE78A
:02A9E800FEE788
:02A9EA00FEE786
:02A9EC00FEE784
:02A9EE00FEE782
:02A9F000FEE780
:02A9F200FEE77E
:02A9F400FEE77C
:02A9F600FEE77A
:02A9F800FEE778
:02A9FA00FEE776
:02A9FC00FEE774
:02A9FE00FEE772
:02AA0000FEE76F
:02AA0200FEE76D
:02AA0400FEE76B
:02AA0600FEE769
:02AA0800FEE767
:02AA0A00FEE765
:02AA0C00FEE763
:02AA0E00FEE761
:02AA1000FEE75F
:02AA1200FEE75D
:02AA1400FEE75B
:02AA1600FEE759
:10AA18004EF68850CEF20000016841F470010160E2
:02AA2800704775
:0EAA2A0041F27471C1F20001096800F000B839
:10AA380080B50B468DF803000DF1030001210122BA
:10AA480000F01EF89DF80310002808BF411E0846B4
:02AA580008BD37
:10AA5A0038B541F27471C1F2000104460D6802F082
:10AA6A00E8F902462846214600F0A5F8013004D04C
:0EAA7A000A20BDE83840FFF7D3BFC04338BD07
:10AA8800F8B51D4617460C460646184602F034F936
:10AA9800002803D407FB04F2A24201D20020F8BD2B
:0EAAA8002846314600F088F8B0FBF4F0F8BD07
:10AAB60052EC10CBC2F30A5340F2FF718B4218BF1F
:10AAC600002B02D100210160704740F2FE3161F394
:0EAAD6001E52A3F2FE31016042EC10CB70471D
:10AAE4002DE9F8432DED028B8E1E00EBC6070D46B3
:10AAF40097ED008BD7E9022359EC108B4046494669
:10AB0400F9F72CFA53EC182BFDF7C6FF032D41EC93
:10AB1400100B12D3741E17ED028B083F53EC102B4D
:10AB240040464946F9F71AFA53EC182BFDF7B4FFDF
:10AB3400012E41EC100B2646ECD853EC102B40466A
:10AB44004946F9F70BFA41EC100BBDEC028BBDE85A
:02AB5400F88384
:10AB56002DE9F8430F46804600EBC10256EC109BE8
:10AB66007C1EA2F1080552E9022351EC100BFDF7F9
:10AB760092FF4A463346F9F7F0F9022F41EC100BE3
:10AB86002A462746ECD8D8E90023FDF784FF41EC96
:06AB9600100BBDE8F8837E
:10AB9C0042694AB110B50446036A002B1CBF2169F7
:0AABAC0098470020606110BD70475B
:0AABB600436A08460121FFF764BF5F
:06ABC000006800F036B849
:10ABC6000146C0680A6982426FEA000010449CBFD1
:06ABD60089680844704785
:10ABDC002DE9F843144688460546C7684FF000092E
:10ABEC002869F943B8420844A96898BF0844CE1BA9
:10ABFC00B04238BF06466868A64228BF264638448D
:10AC0C0041463246F9F7DAFAA868F1190F1A18BF5B
:10AC1C000F46A41BB144B044BFF35F8FEF60DFD18C
:06AC2C004846BDE8F88374
:10AC3200F8B540F6E413C1F2000314461B78002B6A
:10AC42000D46064608BF02F078F8EFF311874FF081
:10AC5200200181F3118830462946224602F0C1F8CC
:06AC620087F31188F8BD24
:10AC680084460020002918BF002A0ED0097848B26F
:10AC780000280BD4BCF1000F18BFCCF8001000213D
:10AC8800C3E90011002818BF012070476FF00100C8
:02AC9800704703
:0EAC9A007F298EBF6FF001000170012070470E
:10ACA80030B58BB000250A95CDE9085568462021B6
:10ACB800F9F7B4FA40F66454C1F200044FF0A0402A
:10ACC8002060201D1421F9F7A9FA0420A0614FF48F
:10ACD8008070A0830120206284F82450C4E90B55B9
:10ACE80084F838504FF48051E16384F840001C2107
:10ACF80061648021C4E9121520652046F9F7A4FF94
:10AD0800002818BFF9F7AAFD062408944FF400405C
:10AD1800CDE9090540F66450C1F2000008A900F029
:10AD2800FFFB002818BFF9F799FD0220C0F2304058
:10AD3800CDE90004012002900020C4F27F000390B6
:10AD48000420CDE9040540F66450C1F200006946CC
:10AD5800FAF702FC002818BFF9F780FD0BB030BDE8
:10AD6800F0B589B00025CDE9075540F6F844C1F2A1
:10AD7800000440F20010C5F200002060201D1421DC
:10AD8800F9F74CFA01270426A6614FF48070A083D6
:10AD9800276284F8245084F838504FF48050E063D8
:10ADA80084F840701C206064802004F14801A1C12F
:10ADB8002046F9F749FF002818BFF9F74FFD08208A
:10ADC800C0F6904001900620CDE902070020C4F2A9
:10ADD8007F00CDE904060695204601A9FAF7BCFBD9
:0CADE800002818BFF9F73AFD09B0F0BDD3
:10ADF40010B58CB000240B94CDE9094401A820219E
:10AE0400F9F70EFA40F68C40C1F2000040F200411E
:10AE1400C5F20001C0E90014C0E902440121C0E9FF
:10AE24000441082282614FF4807282830322026209
:10AE340080F82440C0E90B4480F838104FF4805265
:10AE4400C26380F840101C2242648022C0E91224AC
:10AE54000165F9F7FBFE002818BFF9F701FD099415
:10AE640040F68C40C1F2000009A900F05BFB002809
:10AE740018BFF9F7F5FC0220C0F23040019006201B
:10AE84000290072003907F2004900420CDE905045C
:10AE940040F68C40C1F2000001A9FAF75FFB0028DC
:10AEA40018BFF9F7DDFC41F20000C3F26020019005
:10AEB4000C20029040F68C40C1F2000001A9FAF780
:10AEC4004DFB002818BFF9F7CBFC2020C1F2F0405D
:10AED40001901220029040F68C40C1F2000001A9BA
:10AEE400FAF73CFB002818BFF9F7BAFC0CB010BD08
:10AEF40080B540F69860C1F2000046F60001C4F245
:10AF0400000101600021C0E90111C160C0F80F1007
:10AF1400102242610122C0E90622C0E90822C0E9E8
:10AF24000A22C0E90C21C0E90E11FBF777F90028C9
:0CAF340014BFBDE8084008BDF9F792BC4E
:10AF400080B540F63460C1F2000046F60041C4F21C
:10AF5000000101600021C0E90111C160C0F80F10BB
:10AF6000102242610122C0E90622C0E90822C0E99C
:10AF70000A22C0E90C21C0E90E11FBF751F90028A3
:0CAF800014BFBDE8084008BDF9F76CBC28
:10AF8C0010B541F29C14C1F2000448F20040C4F226
:10AF9C000000206048F2BE20C2F2B10060600020C8
:10AFAC00A0600120E06004F110001421F9F734F9DD
:10AFBC002046FDF7FAFF002818BFF9F74DFC204694
:10AFCC00002100F0D1FD002818BFF9F745FC204600
:10AFDC000021FEF71EFD002814BFBDE8104010BD77
:04AFEC00F9F73ABC7B
:10AFF00010B59CB0044617A81421F9F713F902A85C
:10B000005421F9F70FF9206848F20041C4F2000119
:10B01000884233D0A1F5406188425FD14FF48070FF
:10B02000029002A8F6F7AEFC002818BFF9F71AFC48
:10B0300041F24C04C4F2020417A9206840F0040055
:10B040002060206800F00400019001984FF44070E7
:10B050001790122018900020CDE9190008201B90AD
:10B0600040F60000C4F60000F6F7F8F8E06840F09B
:10B070008040E060E06800F080402DE04FF4003058
:10B08000029002A8F6F77EFC002818BFF9F7EAFB49
:10B0900041F24C04C4F2020417A9206840F00400F5
:10B0A0002060206800F0040001900198C0201790F3
:10B0B000122018900020CDE9190008201B9040F6BE
:10B0C0000000C4F60000F6F7C9F8206940F002005D
:10B0D0002061206900F00200019001981CB010BDB1
:10B0E00010B58EB001A83421F9F79CF801A8F5F746
:10B0F000FFFF06200190BB2005904FF4C44006904E
:10B100004FF4C040079000F007FC28B14CF6557092
:10B11000C0F60000FFF7A1FCFDF7ABFC28B14DF233
:10B12000E930C0F60000FFF798FC4DF61470C0F649
:10B130000000FFF792FC01A8FBF784FA040008D096
:10B140004DF6D110C0F60000FFF787FCFDF7C5FDF6
:10B1500015E0FDF7C2FD4DF62470C0F60000FFF7C4
:10B160007CFC00F0EDFB4DF2FF30C0F60000FFF775
:10B1700074FC4DF63C70C0F60000FFF76EFCB4FAAC
:08B1800084F040090EB010BD7F
:10B18800006800F130404FEA302006280BD87121C2
:10B19800C140C90707D040F6FC71C0F6000151F85C
:08B1A800200001210160704745
:10B1B0000A4601464DF6F900C0F6000001F08ABDCE
:10B1C00080B541F24420C1F2000042F60001C4F211
:10B1D0000001016000217F22C0E90112FF22C0E9C5
:10B1E0000321C0E905114FF08042C0E9072100F0BA
:10B1F00041FD002814BFBDE8084008BDF9F732BB87
:10B2000010B596B0044602A84C21F9F70BF8206857
:10B2100042F60001C4F2000188421DD14FF4002023
:10B2200001904FF48070159001A8F6F7ABFB002851
:10B2300018BFF9F717FB41F25800C4F20200816B06
:10B2400041F400418163016841F48061016000685C
:0CB2500000F480600090009816B010BD63
:10B25C0080B540F6D050C1F2000043F60041C4F274
:10B26C00000101604FF482714160002181604FF454
:10B27C00E062C0E90321012242614FF48022826125
:10B28C001022C0E90721C0E909110722C0E90B21EE
:10B29C00416300F0E3FD002814BFBDE8084008BD81
:04B2AC00F9F7DABA1A
:10B2B00000B583B041F25800C4F20200816841F049
:10B2C00001018160816801F0010102910299016828
:10B2D00041F080510160006800F0805001900198B9
:10B2E0000220FBF712FF00F0E9F803B05DF804EB71
:04B2F000FEF700BCA9
:04B2F400FBF789BE1D
:0CB2F80041F23C10C1F2000000F0BEBAB0
:0CB3040041F2DC00C1F2000000F0B8BA19
:0CB3100041F27C00C1F2000000F0B2BA73
:0CB31C0041F21C00C1F2000000F0ACBACD
:0CB3280040F6BC70C1F2000000F0A6BAB4
:0CB3340040F65C70C1F2000000F0A0BA0E
:0CB3400040F6FC60C1F2000000F09ABA78
:0CB34C0040F62030C1F20000FCF7D8BE33
:0CB3580040F68C20C1F20000FCF7D2BED1
:10B36400802808D0042805D141F2B020C1F20000A1
:10B3740001210160704740F25410C1F200000188BD
:0CB3840001310180418801314180704797
:10B3900010B540F68C24C1F2000444F20040C4F21F
:10B3A000000020604FF4964060604FF48050A06031
:10B3B0000020E0604FF4806020610C20606104F1A7
:10B3C00018001421F8F72EFF4FF40040A063204628
:10B3D00000F07EFE002818BFF9F744FA204600214D
:10B3E00000F020FF002818BFF9F73CFA20460021A2
:10B3F000FEF7CDFD002818BFF9F734FA2046FEF716
:10B4000085FD002814BFBDE8104010BDF9F72ABA29
:10B4100080B540F20850C1F2000045F60041C4F288
:10B42000000101604FF4027181800221C17100218D
:10B430008160FBF795FD002814BFBDE8084008BDFA
:04B44000F9F710BA4E
:10B4440080B5032000F034F90F2000F007F808B1AC
:0CB45400012008BDFFF72AFF002008BD02
:10B4600038B541F27071C1F200010968E9B10446D2
:10B470004FF47A70B0FBF1F041F28071C1F200013B
:10B480000968B1FBF0F0FCF7DEFF01250F2C0DD8A9
:10B4900060B921460022501E0025FCF7B2FD41F2A2
:10B4A0006C70C1F20000046000E00125284638BD40
:0CB4B00041F2A020C1F2000000687047CB
:10B4BC003020C4F20100016821F0010101607047E5
:10B4CC000146806AC26D12F0500FC26D05D0D206D3
:10B4DC000FD4406D426B0846104742F40071C165B1
:10B4EC0001680A681207CA6805D4910709D5FFF7E5
:10B4FC0045BEFCF73CBC12F4406FF8D1C968890416
:10B50C00F5D4C16D21F48071C165C16DC9045EBFF4
:0CB51C00C16D41F00101C165FFF730BEB8
:10B52800F0B583B00446006840F4806040F20046FD
:10B53800C5F20006B0420D4607D04DF6E610C0F63B
:10B54800000040F64C01FFF72FFE28680A280BD2AE
:10B5580040F2EF21C140C90706D041F24001C0F6D0
:10B56800000101EB800008E04DF6E610C0F600008F
:10B5780040F64D01FFF718FE2846006890B168684C
:10B58800002818BFB0F5004F22D1A8684FEA302034
:10B598000C2807D34DF6E610C0F6000040F651011E
:10B5A800FFF702FE94F85800012801D102207BE041
:10B5B8000020029001902368A6F57E70B3F1A04F99
:10B5C80000F1F80110D0B34239D100F59F620CE0C8
:10B5D800B0F5404FD9D04DF6E610C0F600004FF454
:10B5E8000561FFF7E1FDD0E70A4692689E6832439D
:10B5F800520724D48B4214BF4FF4E0614FF44071DA
:10B60800B3F1A04F08BF4FF44071D5F800E0465899
:10B6180026F46046BEF1000F43F4807300F1F80C85
:10B6280013D06A6894F8387042EA47323243634567
:10B63800425012D10268D0F80031134316E0E06D91
:10B6480040F02000E06501202BE06345465018D10A
:10B658000268D0F800311A431BE0D0F80024D0F873
:10B668000035D0F800761A4342EA0703DA0717D103
:10B678004258AF6840F61F739A433A4342EA0E02B3
:10B688000DE0D0F80024D0F80035D0F800761A4341
:10B698003A43D20704D1425840F61F739A434250A6
:0CB6A8000020002184F8581003B0F0BD11
:10B6B40010B504460338052806D34DF64720C0F6D6
:10B6C4000000A621FFF772FD4EF60C50CEF20000EA
:10B6D4004FF6FF020168114064F30A2141F08061D2
:08B6E40041F0FD71016010BD91
:04B6EC00F5F7BCFCB6
:10B6F0000179013940F60012C4F2020202EB810323
:10B700004032C0E9153201F01F01012202FA01F1B5
:04B71000C165704758
:10B7140010B58C46416DD0E913E4CEF804400029FD
:10B724001CBFD0E9164161608468102CD0E9101464
:10B73400006804F01F0E4FF0010404FA0EF44C608C
:10B744004360634604BF134662468360C26010BD13
:10B75400F8B51D4616460F46591E4FF6FF72C0F245
:10B7640003029142044607D34DF22350C0F6000071
:10B7740040F2AB11FFF71AFD94F82400012821D000
:10B78400012084F8240094F82500012817D1022010
:10B7940084F825000020E06320683246016821F027
:10B7A40001010160204639462B46FFF7B1FF216BAA
:10B7B40020680029016807D041F00E010AE000204A
:10B7C40084F824000220F8BD21F00401016001681E
:10B7D40041F00A010160A16C0A68D20342BF0A6801
:10B7E40042F480720A60616D00291EBF0A6842F447
:10B7F40080720A60016841F0010101600020F8BD17
:10B8040090F8251002292FD180B50168D0E910CE17
:10B81400826C0B6823F00E030B600B6823F00103AA
:10B824000B60116821F4807111600EF01F02012178
:10B8340001FA02F2CCF80420D0E913325A60426DC6
:10B8440032B1136823F480731360D0E91623536074
:10B8540080F82510826B002180F824100AB19047EB
:10B864000021BDE8084007E00421C163012180F8FC
:0CB874002510002280F8242008467047B0
:10B8800030B5D0E9103C02681968D2F800E00CF03D
:10B890001F0C042404FA0CF40C4218BF1EF004051B
:10B8A0001BD1022404FA0CF40C4218BF1EF002054E
:10B8B0001ED121FA0CF1090719D51EF0080116D086
:10B8C000116821F00E011160012101FA0CF25A6099
:10B8D000C16380F82510416B16E0116889065EBFD0
:10B8E000116821F0040111605C60016B89B930BD01
:10B8F0001168890606D4116821F00A01116001213E
:10B9000080F825105C60C16A0022002980F824209C
:08B91000EDD0BDE8304008470E
:10B9180042F20800C4F20200C168002901DB0020DD
:10B92800704740F22311C4F26751016001F1883178
:08B938000160C068C00F7047F8
:10B9400042F21400C4F20200016841F000410160BB
:08B950000068C043C00F7047FE
:10B9580070B516460C00054607D14CF6CB70C0F6FC
:10B9680000004FF4CD71FFF71FFC022E03D2182000
:10B9780056B9282008E04CF6CB70C0F6000040F21B
:0CB988009B11FFF711FC18202C5070BD23
:10B9940000688169890744BF002181628169C90700
:0CB9A40002BF816941F001018161704720
:10B9B0002DE9F84F1E4693468A46591E89B2022940
:10B9C000044607D34DF28150C0F6000040F66A21CC
:10B9D000FFF7EEFB94F8410020280AD1DDF828801B
:10B9E000B8F1000F07D00B9F2FB194F84000012849
:10B9F00006D1022514E04FF40070606401250FE0C9
:10BA0000012584F84050FFF753FD814620464FF44E
:10BA1000004101221923CDF80090FBF749F910B13C
:10BA20002846BDE8F88FDDF830C0222084F84100B8
:10BA3000402084F8420000256564C4F824806785AE
:10BA400042F20047C8F200076563A7F58068F2B2CA
:10BA5000204651460023CDF80080E046FDF70DFC5E
:10BA6000204641464A46F5F73FFDC0B9012E206801
:10BA700009D04FEA1B218162204641464A46F5F72C
:10BA800033FD60B920685FFA8BF181622046402166
:10BA900000224346CDF80090FBF70AF910B184F874
:10BAA0004050ABE7608DFF2804D9FF20FF224FF004
:10BAB000807303E0608DC2B24FF000732085204692
:10BAC00051460097FDF7D9FBFF26204604210022AE
:10BAD0004346CDF80090FBF7EBF800288ED12068A4
:10BAE000616A406A0870606A218D01306062481E98
:10BAF0002085618D01396185618DF1B100041CD112
:10BB00002046802100224346CDF80090FBF7D0F874
:10BB100000287FF473AF608DFF2804D92685FF22AB
:10BB20004FF0807304E0608D2085C2B24FF0007347
:10BB3000204651460095FDF7A0FB608D0028C4D13A
:10BB4000204641464A46FBF7B9F900287FF456AF34
:10BB500020682021C16142684EF60003CFF60063E1
:10BB60001A40426084F84110002584F8425084F85D
:04BB7000405055E705
:10BB740038B50446006847F2FF72C4F200029042EE
:10BB84000D4608DC45F20041C4F20001884210D0A1
:10BB940001F5806104E0511C88420AD001F540613E
:10BBA400884206D04DF60930C0F600006321FFF745
:10BBB400FDFA6FF48050054206D04DF60930C0F608
:10BBC40000006421FFF7F2FA94F84100202803D121
:10BBD40094F84000012801D1022038BD242084F8C3
:10BBE40041002068016821F001010160016821F42D
:10BBF40080510160016829430160016841F001013D
:10BC04000160202084F84100002084F8400038BD01
:10BC140010B582B004460020CAF6AA2004EA000146
:10BC2400814218BF14F47F0007D14DF60930C0F6E5
:10BC3400000040F23D11FFF7B9FA41F26000C4F28E
:10BC44000200016841F001010160006800F0010098
:10BC5400019001980420C4F20100016821430160AD
:04BC640002B010BD5D
:0CBC680001684AF6AA2200200A6070471A
:10BC740010B504002FD0606840F04000402807D081
:10BC84004DF29B60C0F6000040F23511FFF78EFACA
:10BC9400A068802807D34DF29B60C0F600004FF4E3
:10BCA4009B71FFF783FAE068B0F5004F07D34DF2BC
:10BCB4009B60C0F6000040F23711FFF777FA206965
:10BCC400B0F5800F09DB14D0B0F5C00F11D0B0F17E
:10BCD400806F06D10DE0012010BD50B1B0F5001FFA
:10BCE40007D04DF29B60C0F600004FF49C71FFF743
:10BCF4005DFA606940F00040B0F1004F07D04DF2AA
:10BD04009B60C0F6000040F23911FFF74FFAA069BA
:10BD140040F48010B0F5801F07D04DF29B60C0F650
:10BD240000004FF49D71FFF741FAE06940F0804054
:10BD3400B0F1804F07D04DF29B60C0F6000040F296
:10BD44003B11FFF733FA206A40F00050B0F1005F76
:10BD540007D04DF29B60C0F600004FF49E71FFF7D0
:10BD640025FA94F8250020B984F824002046FFF72A
:10BD740045FA022084F825002068C168C90634D435
:10BD8400CA214162532141622046F6F787F8C8B9B7
:10BD9400D4E9000CD4E90223816921F08E6121F0F9
:10BDA40040018161216943EA024E41EA0C01A36921
:10BDB4008269194311438161C0F810E0204600F004
:10BDC40019F818B12168FF224A6210BD2068D4F81E
:10BDD40014C0D4E90723816921F060411943114358
:10BDE40041EA0C018161FF214162012084F82500B0
:04BDF400002010BD5E
:10BDF80010B504460068C16821F08001C1608169FE
:10BE0800890607D42046F6F76BF810B1032084F8AA
:10BE1800250010BD816921F0200181612046F6F7D7
:10BE28005FF800281CBF032084F8250021688A6970
:08BE380042F020028A6110BDF6
:10BE400038B50C462029154607D34DF62C40C0F6D0
:10BE5000000040F2E471FFF7ABF942F20050C4F287
:08BE6000000040F8245038BD39
:10BE680038B504000FD0206842F6FF71C4F2010112
:10BE780088420ADC43F60001C4F20001884213D06C
:10BE880001F5806106E0012038BD013188420BD000
:10BE980001F54061884207D04DF2F960C0F6000014
:10BEA80040F24711FFF780F9606850B1B0F5827F22
:10BEB80007D04DF2F960C0F600004FF4A471FFF707
:10BEC80073F9A068002818BFB0F5806F40F086802D
:10BED800E068A0F540704FEA30200D2807D34DF2F6
:10BEE800F960C0F600004FF4A571FFF75DF9A0698D
:10BEF800002818BFB0F5007F7DD1606B40F00800C6
:10BF0800082807D04DF2F960C0F600004FF4A6717A
:10BF1800FFF74AF9E0694FEAF000082807D34DF225
:10BF2800F960C0F6000040F24D11FFF73DF9206AB4
:10BF380040F08000802807D04DF2F960C0F600007C
:10BF48004FF4A771FFF730F9606A40F0100110292B
:10BF580008D04DF2F960C0F6000040F24F11FFF72B
:10BF680023F9606A80B1E0694FEAF000082807D336
:10BF78004DF2F960C0F6000040F26111FFF714F9C4
:10BF88000020C4E9040045E0206940F002000228CE
:10BF980007D04DF2F960C0F600004FF4A971FFF721
:10BFA80003F96069022807D34DF2F960C0F6000072
:10BFB80040F25311FFF7F8F86068B0F5827F27D197
:10BFC800E0694FEAF000082824D34DF2F960C0F682
:10BFD800000040F25711FFF7E7F81BE0B0F5004FFB
:10BFE8003FF476AF4DF2F960C0F6000040F2491117
:10BFF800FFF7DAF86CE7B0F5802F3FF47EAF4DF22B
:10C00800F960C0F6000040F24B11FFF7CDF874E775
:10C018000020E0610025A56294F85D0020B984F84D
:10C028005C502046FAF737F8022084F85D00206853
:10C03800E168B1F5E06F026898BF012541F400633B
:10C04800B3F5706F22F0400202601CBF0022A262AA
:10C0580001F47061D4E9012341EA053C02F48272DB
:10C0680003F404431A44D4E90431A56903F0020334
:10C078001A4401F00101114405F40072114404222C
:10C08800E36902EA154203F03803256A194405F00A
:10C098008003A56A194405F4005319430160616AD5
:10C0A800636B42EA0C0201F01001114303F008022D
:10C0B80011434160C16921F40061C161002020661B
:08C0C800012184F85D1038BD70
:10C0D00010B5040042D0206844F6FF71C4F200019C
:10C0E00088420ADCA1F6FF3188421DD001F580614B
:10C0F000884219D001F5806108E00131884213D0EF
:10C1000001F5405188420FD001F5384188420BD0EB
:10C11000A0694FF49F71002808BF05314DF28900D6
:10C12000C0F60000FFF744F8D4F8880020B984F87E
:10C1300084002046FAF701FE2420C4F88800206815
:10C14000A16A0268002922F00101016002D02046A4
:10C15000FDF76CFD2046FBF755FC08B1012010BD32
:10C160002168486820F490404860886820F02A00E0
:10C170008860086840F0010220460A60BDE810406F
:04C18000F6F702B814
:0CC18400806A0021A0F85E1000F032BAC2
:10C1900038B50546006848F20002C4F20002904239
:10C1A00011D00C46B1F1807F08D34DF28900C0F662
:10C1B000000040F6AF21FEF7FBFF2868416901F05F
:08C1C0007F412143416138BDBC
:10C1C800016848F20002C4F20002914209D0D0F896
:10C1D8008820202A03D190F88420012A03D1022143
:10C1E8000EE001210CE02422C0F888204A6842F4BD
:10C1F80000024A602021C0F88810002180F88410CD
:04C20800084670472D
:10C20C00010002000400060008000A000C001000E7
:08C21C00200040008000000139
:10C2240070B50446006844F6FF72C4F200029042FE
:10C234000D460ADCA2F6FF31884219D001F580616F
:10C24400884215D001F5806108E0511C88420FD066
:10C2540001F5405188420BD001F53841884207D09E
:10C264004DF25770C0F600004FF41971FEF79EFFAF
:10C2740085F000404FEA7070072828D8012101FAA0
:10C2840000F010F0F30F22D094F88400012801D1BB
:10C29400022070BD012084F884002420C4F88800A2
:10C2A40020680668016821F001010160816821F0BD
:10C2B4006041294381602046FDF7FDFD206806604A
:10C2C4002020C4F88800002084F8840070BD4DF25A
:10C2D4005770C0F6000040F26521FEF767FFD3E710
:10C2E4000146B0F8400044F27F0202400020A1F869
:04C2F400402070472F
:10C2F80040F20000C1F200004FF47A73B0F8CC109D
:10C30800A0F88C10B0F98C10B0F97E20891A41F28F
:10C31800E422C1F2000212685A4392FBF1F20021B2
:08C32800C0F89020FEF711B8E7
:10C3300040F60000C4F6000001210122FFF70CBB0B
:04C34000F6F7BABB97
:10C3440040F20C11C1F20001486B0028BABF486BDF
:10C35400404200200A68002A02DD0A68D31702E07E
:10C3640051F8B02C002310B548F29F64C0F20104C8
:10C37400611C80FB0101FCF705FE221A00228A41A0
:10C3840004F10102A2EB0000B8BF0020002948BF5D
:04C39400104610BD82
:10C39800824201D1002015E090429446B8BF8446FD
:10C3A800101A48BF404299421A46B8BF0A46591A5D
:10C3B800009B48BF4942A3EB0C03424301FB032106
:08C3C80091FBF0F000B2704798
:10C3D00010B582B00DF10702002000210123FCF707
:10C3E0003DFA9DF80700411CC8B202280ED843F25E
:10C3F0004C52C0F60002C90052F82000C9B24FF4F6
:10C40000813222FA01F4FEF728FB00E00324E0B2B7
:04C4100002B010BDA9
:10C41400F8B504464DF28120C0F60000FEF71BFB80
:10C424002046FDF7B7FE40F2F832C1F20002B4F83C
:10C434007C005085B4F87E009085D4F880C0D4F890
:10C444008410D4F88830B4F88C005086D4F8900066
:10C45400D4F878E0D4F89450D4F8B060D4F8B47038
:10C46400C2E916561766B4F89850D585B4F89A50B0
:10C474001586D4F89C50B4F8A0609686D4F8A460CD
:10C48400B4F8A870D786D4F8AC70C2E90EC1C2E97A
:10C49400103002F1480080E8E0404FF496404FF439
:10C4A4008031C2E90601012010840021C2F826105F
:10C4B400C2F8221040F2DE31A2F8881047F20011CF
:10C4C400C0F202014FF4FA13C2E923130A21A2F8BD
:10C4D40094106921A2F88A100221C6F66051C2F8AC
:10C4E400961046F2E001A2F89A1000F5003145F6E4
:10C4F400C053C6F2A81347F2A037C6F660574FF6EA
:10C504008376C0F27D0641F27075C1F27C5502F16A
:10C514009C0C8CE88A00C2E92A654FF25421CFF6BC
:10C52400FF7101F57A73A2F8B0304FF63003C1F20F
:10C534007073C2F8B23041F27C53CFF25423C2F884
:10C54400B63001F5FA71A2F8BA103221A2F8BC1083
:10C554006FF0C701A2F8BE1044F62061C0F20701D3
:10C5640040F28433C0F201030127C6F64027642653
:10C5740002F1C00C8CE88A00C2F8CC60D021516072
:10C58400107010746068D06000200021D023FCF784
:0CC59400B9F92046BDE8F840FDF7FCBDF9
:10C5A00040F2B001C1F20001A0F500400860704700
:10C5B00010B582B09C4613460A460446ACF103000F
:10C5C00010F1020F049938BF4FF0010C022B80418B
:10C5D000C0F1090000EB0C0E2046CDE900CEF7F7C4
:10C5E000C7F90020A08484F82600E061C4F81F0089
:04C5F00002B010BDC8
:10C5F40010B5044640F20000C2F2000001210175AA
:10C60400002180F83112D4F880100968B4F85C2055
:10C614004968511AC0F82812D4F89000D4F8900050
:10C62400042805D14EF28400C0F6000000F050FB4F
:10C63400D4F89000012805D14EF29400C0F6000011
:10C6440000F046FBD4F89000022805D14EF2A40075
:10C65400C0F6000000F03CFBD4F89000102805D18F
:10C664004DF65A50C0F6000000F032FBD4F89000AA
:10C67400102805D14DF65A50C0F6000000F028FBF2
:10C68400D4F89000082805D14DF66B50C0F6000090
:10C6940000F01EFBA16D20464FF48072FBF784FC72
:10C6A40038B14DF2A020C0F60000BDE8104000F003
:04C6B4000FBB10BDEB
:10C6B80003464FF00C0C0068B3F82C2283F826C010
:08C6C80003F22711F5F7BABDDA
:10C6D00070B50C4605468E1E3146F7F7A9F9A95BE1
:0CC6E000814218BF4FF0FF34204670BDAF
:04C6EC00007D704716
:10C6F00070B540F2000CC1F2000CBCF81840002BE1
:10C7000018BFA3420AD18B7891F803E04EEA0324C4
:10C71000B4F5FE7F07D340F2862101E040F6863172
:10C720008152022010E00CEB44060D7975704D79B2
:10C730003570861806258554737086F802E00879EE
:0CC74000F070487930710520104470BD85
:10C74C0070B540F2D804C1F2000441F22E3534F831
:10C75C00620CC1F2000528B134F8620C012817D123
:10C76C00012218E0288800284FF6FF7018BFA0851A
:10C77C00A18D11B1A18D814262D1206834F8A01C29
:10C78C00884214DD01264EF2E400C0F600004BE0B6
:10C79C0034F8620C002240F20040C4F600004FF462
:10C7AC008051FFF7D3F834F8620C288070BDE06834
:10C7BC0034F99A1C4FF47A725143884205DD0226F3
:10C7CC004EF2CC00C0F600002EE034F90A0C34F91D
:10C7DC00981C884205DD03264DF67500C0F6000056
:10C7EC0022E034F90C0C34F9981C884205DD04263F
:10C7FC004DF6F050C0F6000016E034F90A0C34F98E
:10C80C00941C884205DA05264DF2EA20C0F6000099
:10C81C000AE034F90C0C34F9941C884210DA062620
:10C82C004DF6CF50C0F60000FEF711F9A68540F288
:10C83C000040C4F600004FF480510022FFF786F848
:10C84C00A08D0028AFD0206834F89E1C8842AADA4C
:10C85C00E06834F99A1C4FF47A7251438842A2DA98
:10C86C0034F90A0C34F9961C88429CDA34F90C0C15
:10C87C0034F9961C884296DA34F90A0C34F9921C75
:10C88C00884290DD34F90C0C34F9921C88427FF705
:10C89C008AAFA08D02283FF486AFA08D07283FF405
:10C8AC0082AF4DF69700C0F60000FEF7D0F80020DE
:04C8BC00A08555E717
:10C8C000F8B540F2BC05C1F200054FF47A77686C08
:10C8D00029887943884240F60004C4F6000441F2F6
:10C8E0001C36C1F2000612DD307880B94DF21830E6
:10C8F000C0F60000FEF7B1F801203070A888B0FA49
:10C9000080F0420920464FF40051FFF725F8686C8B
:10C9100069887943884214DA307890B14EF2101069
:10C92000C0F60000FEF799F800203070AA88002AAF
:10C9300018BF012220464FF40051BDE8F840FFF730
:04C940000BB8F8BD7B
:10C9440040F2E000C1F2000040F20A2120F8E01CAD
:10C95400002141640164CA438286C2620263828701
:10C96400C287028742874FF0010C20F8D8CC20F808
:10C97400D61C20F8D41C4FF000438360DB43C36013
:10C984004FF4004320F8103C013B20F80E3C5A1CA5
:10C99400CFF6FF7240F8042C0360A0F8A21020F830
:10C9A400BACC032120F8B81C052120F8B61C61215B
:10C9B40080F8C010622180F8C110792180F8D61067
:10C9C4007A2180F8D7104FF47A71A0F8F6107047E6
:10C9D40040F20000C1F200004FF2F012016ECFF6F7
:0CC9E400FF725143CA17C0E95A12704795
:10C9F00040F21010C1F20000816B826B002948BF29
:08CA00005242026000F000B890
:10CA080010B540F20004C1F20004D4F80C0100286B
:10CA18004FF0FF3011D4D4F80C11E26D91420AD2D4
:10CA2800E26D52B14FF47A70E26DA1FB0001002370
:10CA3800FCF788FB01E04FF47A70A4F8140110BDEC
:10CA480040F20000C1F20000026E8AB180B5D0E960
:10CA58005C0148F2A06CC0F2010CA0FB0C0301FBC6
:10CA68000C314FF46163A2FB0323FCF789FA08BD7C
:04CA780000207047E3
:10CA7C0040F21011C1F20001886B0028BABF886B1C
:10CA8C00404200200A68002A02DD0A68D31702E03F
:10CA9C0051F8B02C002310B548F29F64C0F2010489
:10CAAC00611C80FB0101FCF769FA221A00228A4101
:10CABC0004F10102A2EB0000B8BF0020002948BF1E
:04CACC00104610BD43
:10CAD00040F2D800C1F20000816B002905DD416BF6
:10CAE000826E11444FEAE17C05E050F87C1C826EB6
:10CAF00011444FF0000C70B50368B0F8A860856B66
:10CB0000012D02DB846BE51702E050F8784C00251C
:10CB1000981900EBD0735E10A1FB0602DB1701FB36
:10CB200003210CFB06114FF47A720023FCF72CFA58
:10CB300048F2A066C0F20106A0FB060201FB062136
:10CB400022462B46FCF720FA20EAE070B042A8BF4C
:04CB5000304670BD3E
:10CB540051EC102BC1F30A53002B1CBF40F2FF7C95
:10CB6400634514D01844604506DB0020C7F6F07016
:10CB740060F31E01002208E00028C7BF6FF31E51B6
:10CB840041EA005101F00041002241EC102B7047B2
:04CB9400F3F744BDB2
:10CB980010B582B0044600698DF8071078B1D4E961
:10CBA80000239A4231D26269531C63618154D4E9EB
:10CBB8000501884229D12046FDF7ECFF25E0E06811
:10CBC80050B1D4E9002C62451FD2531CB3EB0C03BF
:10CBD80018BF0B46835418E0A06858B1D4E9002C5C
:10CBE800624512D2531CB3EB0C0318BFCBB240F80A
:10CBF80022300AE0236A43B1D4E90001884204D212
:10CC08000DF1070120460122984720680130206075
:04CC180002B010BD99
:10CC1C00012A0CDBF8B514460D460646671E304655
:10CC2C002946FFF7B3FF012C3C46F7D8F8BD7047F7
:10CC3C00CB0606D43023890558BF20231946FFF7AD
:04CC4C00E7BF704787
:10CC500070B514460D460646F7F718FB01463046F8
:0CCC60002A462346BDE8704000F000B8F2
:10CC6C002DE9F04F03AF8DB047F83C3C91460C4694
:10CC7C00064600F05BF80546EB46073020F007004F
:10CC8C00ADEB0008C546A7F1380A50460021242216
:10CC9C00F7F7C6FA47E908546FF0004047F8340C30
:10CCAC004AF6B730C0F6000047F8288C47E906066C
:10CCBC005046494657F83C2CFCF744FBDD46A7F19F
:08CCCC000C04A546BDE8F08F41
:10CCD40083B000B582B0CDE9031241F2747CC1F295
:10CCE400000C059303AA01920146DCF80000FFF74B
:0CCCF400ADFF02B05DF804EB03B0704728
:10CD000041F27871C1F2000141F27472C1F2000285
:10CD10000968126841F27C73C1F20003411A1B6872
:10CD200018BF0121821A18BF01221140C01A18BF72
:08CD3000012008404042704759
:04CD380040207047E0
:10CD3C0040F6E410C1F2000003214DF63762C0F654
:10CD4C0000020161416141F23631C1F200018261A0
:10CD5C00C1614FF480610162002181624162C16254
:10CD6C0041F23673C1F200030266436610228266FA
:10CD7C000167C1664DF62662C0F600024167BFF33B
:10CD8C005F8F531ADB7B435401311029F9D1BFF368
:04CD9C005F8F7047EE
:10CDA0002DE9F04104468068E66815466268871BF5
:10CDB0009019BD4206D22A46F7F706FABFF35F8FF5
:10CDC00035440CE088463A46F7F7FEF9ED1B08EBD0
:10CDD000070160682A46F7F7F7F9BFF35F8FE56050
:04CDE000BDE8F08139
:10CDE40070B500EB400040F6E413C1F2000303EB1E
:10CDF400C00303F11806D86A022818D00D46144659
:10CE0400012807D020B93046FDF7DBFEA04207D247
:10CE140000240AE03046FDF7D4FEA04238BF0446A1
:10CE2400304629462246FFF7B9FF204670BD3046FA
:08CE3400BDE87040FDF7D0BE1F
:10CE3C00017889B14FF0013C0346194653F8042B95
:10CE4C00CCFA52F2002AF8D092FAA2F2B2FA82F29A
:0CCE5C0001EBD201081A7047002070475B
:10CE680000291CBF0278002A01D10020704700B5B4
:10CE78000429D0F800E0024609D34FF0013CCCFA6F
:10CE88005EF323B90439032952F804EFF7D84FF0B9
:10CE98000133C3FA5EF393FAA3F3B3FA83F3101AD8
:0CCEA800B1EBD30F88BFD908084400BDCF
:10CEB4007F280BD84EF25C12C0F600024DF6A16337
:10CEC400C0F60003105C595C0840704700207047AE
:0CCED400A0F161011A2938BF2038704716
:0CCEE000A0F141011A2938BF2030704732
:10CEEC007F280BD84EF25C12C0F600024DF6A163FF
:10CEFC00C0F60003105C595C084070470020704776
:0CCF0C00A0F161011A2938BF20387047DD
:0CCF1800A0F141011A2938BF20307047F9
:0FCF24005465737420646562756720696F0D0032
:10CF3300666163746F727920726573746F72652EA4
:03CF43002E2E008F
:0FCF46006572726F722068616E646C65720D00A7
:10CF5500466C61736820756E6C6F636B20657272C9
:03CF65006F7200E8
:10CF6800443A5C50726F6A656B74655C65637353B1
:10CF78006D61727450726F5C7472756E6B5C6677FB
:10CF88005F673437337263745C44726976657273B1
:10CF98005C53544D3332473478785F48414C5F4492
:10CFA80072697665725C5372635C73746D33326751
:10CFB8003478785F68616C5F666C6173685F657808
:03CFC8002E6300D5
:10CFCB00443A5C50726F6A656B74655C656373534E
:10CFDB006D61727450726F5C7472756E6B5C667798
:10CFEB005F673437337263745C447269766572734E
:10CFFB005C53544D3332473478785F48414C5F442F
:10D00B0072697665725C5372635C73746D333267ED
:0FD01B003478785F68616C5F6770696F2E6300AF
:10D02A00443A5C50726F6A656B74655C65637353EE
:10D03A006D61727450726F5C7472756E6B5C667738
:10D04A005F673437337263745C44726976657273EE
:10D05A005C53544D3332473478785F48414C5F44CF
:10D06A0072697665725C5372635C73746D3332678E
:0FD07A003478785F68616C5F697764672E630054
:10D08900443A5C50726F6A656B74655C656373538F
:10D099006D61727450726F5C7472756E6B5C6677D9
:10D0A9005F673437337263745C447269766572738F
:10D0B9005C53544D3332473478785F48414C5F4470
:10D0C90072697665725C5372635C73746D3332672F
:0FD0D9003478785F68616C5F756172742E6300E4
:0FD0E80049205265666572656E7A3D25660A00BD
:0BD0F700547368756E743D25660A00D6
:10D102002D2D2D204761696E20447269667420437B
:07D11200414C202D2D2D00E2
:0FD1190041637475616C20543D256620430A0004
:10D1280041637574616C20493D2566204128776903
:10D1380074686F7574206761696E2074656D7020FE
:10D14800647269667420636F7272656374696F6E66
:03D15800290A00A1
:10D15B004B6F7272656B74757266616B746F723D37
:10D16B002566205B2031202F2043656C7369757316
:03D17B005D0A004A
:10D17E004552524F52204144535F313236305F5345
:0BD18E006574446174615261746500B7
:10D199004552524F52204144535F313236305F532A
:0BD1A900657443686F704D6F64650093
:10D1B40054696D652025643A20456D707479206545
:10D1C40076656E742831292C20636E3D25642C20ED
:10D1D40063613D25642C20744469736368617267DC
:10D1E400653D25642C20753D25642C20693D25640E
:03D1F4000D0A0021
:10D1F70054696D652025643A20456D707479206502
:10D2070076656E742832292C20636E3D25642C20A8
:10D2170063613D25642C2074446973636861726798
:10D22700653D25642C20753D25642C20693D2564CA
:03D237000D0A00DD
:10D23A00454550524F4D20776173206368616E6790
:10D24A00656421205765206E65656420746F2070BF
:10D25A00726573657276652063616C696272617466
:10D26A00696F6E20616E642073657474696E67738A
:07D27A0020646174612100D2
:10D28100454550524F4D20464143544F525920522B
:0FD291004553544F52452F5550444154452100A9
:10D2A00055617274204572726F7220626569206EDA
:10D2B00065757374617274206E6163682046656879
:07D2C0006C6572200A0D00ED
:10D2C7004F5554505554535F4C56505F5348554E25
:10D2D700545F554E44455254454D5045524154555F
:03D2E700524500AD
:10D2EA004F5554505554535F4F56505F5348554EFF
:10D2FA00545F554E44455254454D5045524154553C
:03D30A0052450089
:0BD30D00486561746572206F6E0D00B2
:10D31800415558206F6E2028534F43204D6F646548
:03D32800290D00CC
:07D32B00286E756C6C2900EF
:10D332004A616E75617279004665627275617279D1
:10D34200004D6172636800417072696C004D6179D1
:10D35200004A756E65004A756C7900417567757390
:10D36200740053657074656D626572004F63746F0B
:10D37200626572004E6F76656D6265720044656328
:07D38200656D626572000099
:07D38900414D00504D000072
:0FD3900025612025622025652025542025590080
:10D39F0053797374656D20636F726520636C6F636F
:0AD3AF006B3A2025754D487A0A00FC
:10D3B9004261636B75705265676973746572446124
:0ED3C900746120617661696C61626C650D00B3
:10D3D7002E2E2E466C61736820756E6C6F636B65BD
:02D3E7006400E0
:10D3E900466C617368206F6220756E6C6F636B2089
:06D3F9006572726F720004
:0ED3FF00466C61736820206C6F636B65640080
:10D40D00443A5C50726F6A656B74655C6563735307
:10D41D006D61727450726F5C7472756E6B5C667751
:10D42D005F673437337263745C4472697665727307
:10D43D005C53544D3332473478785F48414C5F44E8
:10D44D0072697665725C5372635C73746D333267A7
:0AD45D003478785F68616C2E63007C
:10D46700443A5C50726F6A656B74655C65637353AD
:10D477006D61727450726F5C7472756E6B5C6677F7
:10D487005F673437337263745C44726976657273AD
:10D497005C53544D3332473478785F48414C5F448E
:10D4A70072697665725C5372635C73746D3332674D
:0ED4B7003478785F68616C5F6164632E630097
:10D4C500443A5C50726F6A656B74655C656373534F
:10D4D5006D61727450726F5C7472756E6B5C667799
:10D4E5005F673437337263745C447269766572734F
:10D4F5005C53544D3332473478785F48414C5F4430
:10D5050072697665725C5372635C73746D333267EE
:0ED515003478785F68616C5F6372632E630028
:10D52300443A5C50726F6A656B74655C65637353F0
:10D533006D61727450726F5C7472756E6B5C66773A
:10D543005F673437337263745C44726976657273F0
:10D553005C53544D3332473478785F48414C5F44D1
:10D5630072697665725C5372635C73746D33326790
:0ED573003478785F68616C5F646D612E6300D0
:10D58100443A5C50726F6A656B74655C6563735392
:10D591006D61727450726F5C7472756E6B5C6677DC
:10D5A1005F673437337263745C4472697665727392
:10D5B1005C53544D3332473478785F48414C5F4473
:10D5C10072697665725C5372635C73746D33326732
:0ED5D1003478785F68616C5F6932632E6300A6
:10D5DF00443A5C50726F6A656B74655C6563735334
:10D5EF006D61727450726F5C7472756E6B5C66777E
:10D5FF005F673437337263745C4472697665727334
:10D60F005C53544D3332473478785F48414C5F4414
:10D61F0072697665725C5372635C73746D333267D3
:0ED62F003478785F68616C5F7063642E63000E
:10D63D00443A5C50726F6A656B74655C65637353D5
:10D64D006D61727450726F5C7472756E6B5C66771F
:10D65D005F673437337263745C44726976657273D5
:10D66D005C53544D3332473478785F48414C5F44B6
:10D67D0072697665725C5372635C73746D33326775
:0ED68D003478785F68616C5F7263632E6300AF
:10D69B00443A5C50726F6A656B74655C6563735377
:10D6AB006D61727450726F5C7472756E6B5C6677C1
:10D6BB005F673437337263745C4472697665727377
:10D6CB005C53544D3332473478785F48414C5F4458
:10D6DB0072697665725C5372635C73746D33326717
:0ED6EB003478785F68616C5F7274632E630040
:10D6F900443A5C50726F6A656B74655C6563735319
:10D709006D61727450726F5C7472756E6B5C667762
:10D719005F673437337263745C4472697665727318
:10D729005C53544D3332473478785F48414C5F44F9
:10D7390072697665725C5372635C73746D333267B8
:0ED749003478785F68616C5F7370692E6300DE
:10D75700443A5C50726F6A656B74655C65637353BA
:10D767006D61727450726F5C7472756E6B5C667704
:10D777005F673437337263745C44726976657273BA
:10D787005C53544D3332473478785F48414C5F449B
:10D7970072697665725C5372635C73746D3332675A
:10D7A7003478785F68616C5F756172745F65782E35
:02D7B70063000D
:10D7B9002D2D2D204761696E202043414C202D2DB0
:02D7C9002D0031
:0AD7CB0054736869703D25660A007A
:10D7D5002D2D2D204761696E202043414C20454E5B
:06D7E50044452D2D2D002E
:0ED7EB0064656C746120543D256620430A007D
:0AD7F90052656620493D25660A00CE
:10D803004552524F52204144535F313236305F49C3
:0ED813006E7075744D757853656C65637400A6
:10D8210046697273742073746172742064657465DF
:06D8310063746564210030
:0ED8370075617274206572726F72200A0D00A6
:10D845004F5554505554535F4C56505F5348554EA1
:10D85500545F4F56455254454D50455241545552CB
:02D8650045007C
:0ED867004F5554505554204C5650204F4B00F6
:10D875004F5554505554535F4F56505F5348554E6E
:10D88500545F4F56455254454D504552415455529B
:02D8950045004C
:0ED897004F5554505554204F5650204F4B00C3
:10D8A500415558206F66662028416C61726D204D88
:06D8B5006F6465290D00FF
:10D8BB0053756E646179004D6F6E646179005475B8
:10D8CB006573646179005765646E65736461790093
:10D8DB00546875727364617900467269646179008A
:0AD8EB0053617475726461790000E6
:02D8F5004300EE
:02D8F7002E0001
:10D8F90057726F6E6720706172616D6574657273BE
:10D909002076616C75653A2066696C6520257320FF
:0DD919006F6E206C696E652025640D0A009C
:0DD926004144533132363020496E6974009F
:10D9330053484F52545F434952435549545F5052E1
:09D943004F54454354494F4E0076
:10D94C004A756D7020686173206661696C6564212D
:01D95C0000CA
:10D95D002E2E2E466C617368206F6220756E6C6F73
:05D96D00636B6564001E
:10D972002E2E2E44697361626C65206C6F636B207E
:10D9820070726F636573732066696E69736865642C
:01D992000094
:10D99300466C617368204F7074696F6E6279746549
:10D9A3002070726F6772616D6D206661696C65646A
:01D9B3000073
:10D9B4002E2E2E466C617368206C6F636B20616C35
:0DD9C40072656164792061637469766500A5
:10D9D1002E2E2E456E61626C65206C6F636B206527
:05D9E10072726F72007C
:10D9E600443A5C50726F6A656B74655C6563735329
:10D9F6006D61727450726F5C7472756E6B5C667773
:10DA06005F673437337263745C4472697665727328
:10DA16005C53544D3332473478785F48414C5F4409
:10DA260072697665725C5372635C73746D333267C8
:10DA36003478785F68616C5F6164635F65782E63D4
:01DA460000DF
:10DA4700443A5C50726F6A656B74655C65637353C7
:10DA57006D61727450726F5C7472756E6B5C667711
:10DA67005F673437337263745C44726976657273C7
:10DA77005C53544D3332473478785F48414C5F44A8
:10DA870072697665725C5372635C73746D33326767
:10DA97003478785F68616C5F636F727465782E6342
:01DAA700007E
:10DAA800443A5C50726F6A656B74655C6563735366
:10DAB8006D61727450726F5C7472756E6B5C6677B0
:10DAC8005F673437337263745C4472697665727366
:10DAD8005C53544D3332473478785F48414C5F4447
:10DAE80072697665725C5372635C73746D33326706
:10DAF8003478785F68616C5F6372635F65782E6302
:01DB0800001C
:10DB0900443A5C50726F6A656B74655C6563735304
:10DB19006D61727450726F5C7472756E6B5C66774E
:10DB29005F673437337263745C4472697665727304
:10DB39005C53544D3332473478785F48414C5F44E5
:10DB490072697665725C5372635C73746D333267A4
:10DB59003478785F68616C5F6932635F65782E63DA
:01DB690000BB
:10DB6A00443A5C50726F6A656B74655C65637353A3
:10DB7A006D61727450726F5C7472756E6B5C6677ED
:10DB8A005F673437337263745C44726976657273A3
:10DB9A005C53544D3332473478785F48414C5F4484
:10DBAA0072697665725C5372635C73746D33326743
:10DBBA003478785F68616C5F7077725F65782E631E
:01DBCA00005A
:10DBCB00443A5C50726F6A656B74655C6563735342
:10DBDB006D61727450726F5C7472756E6B5C66778C
:10DBEB005F673437337263745C4472697665727342
:10DBFB005C53544D3332473478785F48414C5F4423
:10DC0B0072697665725C5372635C73746D333267E1
:10DC1B003478785F68616C5F7263635F65782E63DD
:01DC2B0000F8
:10DC2C00443A5C50726F6A656B74655C65637353E0
:10DC3C006D61727450726F5C7472756E6B5C66772A
:10DC4C005F673437337263745C44726976657273E0
:10DC5C005C53544D3332473478785F48414C5F44C1
:10DC6C0072697665725C5372635C73746D33326780
:10DC7C003478785F68616C5F7274635F65782E636B
:01DC8C000097
:10DC8D00492028776974686F757420636F6D7065AE
:0DDC9D006E736174696F6E293D25660A0083
:10DCAA004144535F313236305F4261747465727930
:10DCBA0043757272656E744761696E43616C69621D
:10DCCA00726174696F6E53746172743A204552526C
:10DCDA004F5220494E2043414C4942524154494FE8
:10DCEA004E2C204E4F205245464552454E43452024
:09DCFA0043555252454E542100DD
:10DD03004E6F726D616C20737461727420776974E5
:10DD1300686F757420454550524F4D206368616E9E
:0DDD23006765732064657465637465640052
:10DD3000454550524F4D2046554C4C20524553546A
:05DD40004F52452100D7
:10DD4500454550524F4D2053544F524520434F4E59
:05DD55004649472100D2
:10DD5A004D4220444D41204572726F7221200A0DB6
:01DD6A0000B8
:10DD6B004D42204F5245204572726F7221200A0D91
:01DD7B0000A7
:10DD7C004552524F52205561727420494E49540DF0
:01DD8C000096
:10DD8D004F5554505554535F4C56505F434849506E
:10DD9D005F4F56455254454D50455241545552458D
:01DDAD000075
:10DDAE004F5554505554535F4C56505F4241545446
:10DDBE004552595F554E444552564F4C5441474576
:01DDCE000054
:10DDCF004F5554505554535F4F56505F4348495029
:10DDDF005F554E444554454D50455241545552455B
:01DDEF000033
:10DDF0004F5554505554535F4F56505F4348495008
:10DE00005F4F56455254454D504552415455524529
:01DE10000011
:10DE1100415558206F6E2028416C61726D204D6F05
:05DE21006465290D00FD
:10DE26000000000000005454522052454747455315
:01DE360000EB
:09DE37005465726D696E616C00A6
:09DE4000256D2F25642F257900C2
:09DE490025483A254D3A25530005
:10DE520053756E004D6F6E00547565005765640012
:0DDE62005468750046726900536174000039
:10DE6F004A616E00466562004D617200417072003A
:10DE7F004D6179004A756E004A756C0041756700F7
:10DE8F00536570004F6374004E6F760044656300F6
:01DE9F000082
:01DEA0000081
:0DDEA10000070320041702010857104080FD
:10DEB000AC420008AC420008AC420008AC4200088A
:04DEC000AC42000868
:04DEC400E1890008E8
:10DEC800554E4B4E4F574E20434F4D4D414E4400FB
:10DED800466C617368204F7074696F6E62797465FF
:0CDEE8002070726F6772616D6D656400E0
:10DEF400537461727420656E61626C652072656131
:10DF0400646F75742070726F74656374696F6E00EA
:10DF14002E2E2E466C61736820756E6C6F636B00D9
:10DF2400466C617368204F7074696F6E62797465B2
:08DF3400206C6F636B65640053
:10DF3C002E2E2E456E61626C65206C6F636B2070AB
:10DF4C00726F636573732066696E697368656400CC
:10DF5C00443A5C50726F6A656B74655C65637353AD
:10DF6C006D61727450726F5C7472756E6B5C6677F7
:10DF7C005F673437337263745C44726976657273AD
:10DF8C005C53544D3332473478785F48414C5F448E
:10DF9C0072697665725C5372635C73746D3332674D
:10DFAC003478785F68616C5F666463616E2E6300C1
:08DFBC0001010103070100004F
:08DFC400080402040801010138
:10DFCC004B6F7272656B74757266616B746F723DB8
:04DFDC0025660A00AC
:10DFE0002D2D2D204761696E20447269667420438F
:0CDFF000414C20454E4445202D2D2D00B5
:10DFFC004552524F52204144535F313236305F53B9
:10E00C006574496E7465726E616C52656665726595
:04E01C006E636500CA
:10E0200054696D652025643A204261747465726993
:10E03000652046756C6C206576656E74206D416850
:10E040004361726765643D25642C20744368617286
:10E0500067653D25642C2063656641683D25642C19
:10E060002063656657683D25642C20753D25642C2A
:08E0700020693D25640D0A0042
:0CE0780057726974696E6720534E2100D6
:10E084004D42204645204572726F7221200A0D00D0
:10E094004D42205045204572726F7221200A0D00B6
:10E0A4004D42204E45204572726F7221200A0D00A8
:10E0B4004F5554505554535F4C56505F4F5645522C
:08E0C40043555252454E540031
:10E0CC004F5554505554535F4F56505F4F56455211
:08E0DC0043555252454E540019
:10E0E4004F5554505554535F4F56505F424154540A
:10E0F4004552595F4F564552564F4C54414745007F
:0CE10400486561746572206F66660D004E
:10E11000415558206F66662028534F43204D6F6449
:04E1200065290D0060
:10E1240000000000000000000102030406070809C3
:08E134000000000001020304D9
:10E13C003031323334353637383941424344454631
:10E14C003031323334353637383961626364656661
:10E15C00202020202020202020682828282820204B
:10E16C0020202020202020202020202020202020A3
:10E17C00481010101010101010101010101010105B
:10E18C0084848484848484848484101010101010FB
:10E19C001081818181818101010101010101010154
:10E1AC000101010101010101010101101010101008
:10E1BC001082828282828202020202020202020225
:10E1CC0002020202020202020202021010101020CD
:10E1DC0000B506480649884205D00268043003B4ED
:10E1EC00904703BCF7E708BC18470000C4DE0008E2
:04E1FC00C8DE000871
:10E200009DE20008000000101D1300009DE20008C0
:10E210001E130010030000009DE2000822130010EE
:10E22000030000009DE200082613001020040000F7
:10E230009DE2000884170010040000009DE2000821
:10E24000000000205C030000AFE200088817001007
:10E2500070E2000814000000C3E200084C17001030
:10E2600084E2000838000000DDE10008273F0008D4
:10E27000AC420008AC420008AC420008AC420008C6
:10E28000AC420008FFFFFE01FFEE100144C4121073
:0CE29000C8121094CC121024F4000000FE
:10E29C00206861680834002200E04254491EFCD515
:02E2AC007047B9
:10E2AE0020686168A2680C3401E08B5C8354521EB6
:04E2BE00FBD57047D5
:10E2C20020686168A2680C340B78491C0826002576
:10E2D2005B0801D20D78491C0570401C521E02D009
:08E2E200761EF4D1F0E770474D
:0400000508003F317F
:00000001FF
